Archive member included to satisfy reference by file (symbol)

d:/psx/rj/mounriver_studio/toolchain/risc-v embedded gcc/bin/../lib/gcc/riscv-none-embed/8.2.0/rv32imacxw/ilp32\libgcc.a(adddf3.o)
                              ./App/src/mppt_control.o (__adddf3)
d:/psx/rj/mounriver_studio/toolchain/risc-v embedded gcc/bin/../lib/gcc/riscv-none-embed/8.2.0/rv32imacxw/ilp32\libgcc.a(gedf2.o)
                              ./App/src/mppt_control.o (__gedf2)
d:/psx/rj/mounriver_studio/toolchain/risc-v embedded gcc/bin/../lib/gcc/riscv-none-embed/8.2.0/rv32imacxw/ilp32\libgcc.a(ledf2.o)
                              ./App/src/mppt_control.o (__ledf2)
d:/psx/rj/mounriver_studio/toolchain/risc-v embedded gcc/bin/../lib/gcc/riscv-none-embed/8.2.0/rv32imacxw/ilp32\libgcc.a(muldf3.o)
                              ./App/src/collect_Conversion.o (__muldf3)
d:/psx/rj/mounriver_studio/toolchain/risc-v embedded gcc/bin/../lib/gcc/riscv-none-embed/8.2.0/rv32imacxw/ilp32\libgcc.a(subdf3.o)
                              ./App/src/collect_Conversion.o (__subdf3)
d:/psx/rj/mounriver_studio/toolchain/risc-v embedded gcc/bin/../lib/gcc/riscv-none-embed/8.2.0/rv32imacxw/ilp32\libgcc.a(floatsidf.o)
                              ./App/src/collect_Conversion.o (__floatsidf)
d:/psx/rj/mounriver_studio/toolchain/risc-v embedded gcc/bin/../lib/gcc/riscv-none-embed/8.2.0/rv32imacxw/ilp32\libgcc.a(addsf3.o)
                              ./App/src/mppt_control.o (__addsf3)
d:/psx/rj/mounriver_studio/toolchain/risc-v embedded gcc/bin/../lib/gcc/riscv-none-embed/8.2.0/rv32imacxw/ilp32\libgcc.a(divsf3.o)
                              ./App/src/mppt_control.o (__divsf3)
d:/psx/rj/mounriver_studio/toolchain/risc-v embedded gcc/bin/../lib/gcc/riscv-none-embed/8.2.0/rv32imacxw/ilp32\libgcc.a(eqsf2.o)
                              ./App/src/task.o (__eqsf2)
d:/psx/rj/mounriver_studio/toolchain/risc-v embedded gcc/bin/../lib/gcc/riscv-none-embed/8.2.0/rv32imacxw/ilp32\libgcc.a(gesf2.o)
                              ./App/src/mppt_control.o (__gesf2)
d:/psx/rj/mounriver_studio/toolchain/risc-v embedded gcc/bin/../lib/gcc/riscv-none-embed/8.2.0/rv32imacxw/ilp32\libgcc.a(lesf2.o)
                              ./App/src/mppt_control.o (__ltsf2)
d:/psx/rj/mounriver_studio/toolchain/risc-v embedded gcc/bin/../lib/gcc/riscv-none-embed/8.2.0/rv32imacxw/ilp32\libgcc.a(mulsf3.o)
                              ./Hardware/src/pwm.o (__mulsf3)
d:/psx/rj/mounriver_studio/toolchain/risc-v embedded gcc/bin/../lib/gcc/riscv-none-embed/8.2.0/rv32imacxw/ilp32\libgcc.a(subsf3.o)
                              ./App/src/mppt_control.o (__subsf3)
d:/psx/rj/mounriver_studio/toolchain/risc-v embedded gcc/bin/../lib/gcc/riscv-none-embed/8.2.0/rv32imacxw/ilp32\libgcc.a(fixsfsi.o)
                              ./App/src/mppt_control.o (__fixsfsi)
d:/psx/rj/mounriver_studio/toolchain/risc-v embedded gcc/bin/../lib/gcc/riscv-none-embed/8.2.0/rv32imacxw/ilp32\libgcc.a(fixunssfsi.o)
                              ./Hardware/src/pwm.o (__fixunssfsi)
d:/psx/rj/mounriver_studio/toolchain/risc-v embedded gcc/bin/../lib/gcc/riscv-none-embed/8.2.0/rv32imacxw/ilp32\libgcc.a(floatsisf.o)
                              ./App/src/task.o (__floatsisf)
d:/psx/rj/mounriver_studio/toolchain/risc-v embedded gcc/bin/../lib/gcc/riscv-none-embed/8.2.0/rv32imacxw/ilp32\libgcc.a(floatunsisf.o)
                              ./App/src/collect_Conversion.o (__floatunsisf)
d:/psx/rj/mounriver_studio/toolchain/risc-v embedded gcc/bin/../lib/gcc/riscv-none-embed/8.2.0/rv32imacxw/ilp32\libgcc.a(extendsfdf2.o)
                              ./Hardware/src/pwm.o (__extendsfdf2)
d:/psx/rj/mounriver_studio/toolchain/risc-v embedded gcc/bin/../lib/gcc/riscv-none-embed/8.2.0/rv32imacxw/ilp32\libgcc.a(truncdfsf2.o)
                              ./App/src/collect_Conversion.o (__truncdfsf2)
d:/psx/rj/mounriver_studio/toolchain/risc-v embedded gcc/bin/../lib/gcc/riscv-none-embed/8.2.0/rv32imacxw/ilp32\libgcc.a(save-restore.o)
                              ./App/src/sl_protocol.o (__riscv_save_12)
d:/psx/rj/mounriver_studio/toolchain/risc-v embedded gcc/bin/../lib/gcc/riscv-none-embed/8.2.0/rv32imacxw/ilp32\libgcc.a(_clzsi2.o)
                              d:/psx/rj/mounriver_studio/toolchain/risc-v embedded gcc/bin/../lib/gcc/riscv-none-embed/8.2.0/rv32imacxw/ilp32\libgcc.a(adddf3.o) (__clzsi2)
d:/psx/rj/mounriver_studio/toolchain/risc-v embedded gcc/bin/../lib/gcc/riscv-none-embed/8.2.0/rv32imacxw/ilp32\libgcc.a(_clz.o)
                              d:/psx/rj/mounriver_studio/toolchain/risc-v embedded gcc/bin/../lib/gcc/riscv-none-embed/8.2.0/rv32imacxw/ilp32\libgcc.a(_clzsi2.o) (__clz_tab)
d:/psx/rj/mounriver_studio/toolchain/risc-v embedded gcc/bin/../lib/gcc/riscv-none-embed/8.2.0/../../../../riscv-none-embed/lib/rv32imacxw/ilp32\libg_nano.a(lib_a-memcpy.o)
                              ./Hardware/src/flash.o (memcpy)
d:/psx/rj/mounriver_studio/toolchain/risc-v embedded gcc/bin/../lib/gcc/riscv-none-embed/8.2.0/../../../../riscv-none-embed/lib/rv32imacxw/ilp32\libg_nano.a(lib_a-memset.o)
                              ./Hardware/src/adc.o (memset)
d:/psx/rj/mounriver_studio/toolchain/risc-v embedded gcc/bin/../lib/gcc/riscv-none-embed/8.2.0/../../../../riscv-none-embed/lib/rv32imacxw/ilp32\libg_nano.a(lib_a-printf.o)
                              ./User/main.o (printf)
d:/psx/rj/mounriver_studio/toolchain/risc-v embedded gcc/bin/../lib/gcc/riscv-none-embed/8.2.0/../../../../riscv-none-embed/lib/rv32imacxw/ilp32\libg_nano.a(lib_a-putchar.o)
                              ./App/src/mppt_control.o (putchar)
d:/psx/rj/mounriver_studio/toolchain/risc-v embedded gcc/bin/../lib/gcc/riscv-none-embed/8.2.0/../../../../riscv-none-embed/lib/rv32imacxw/ilp32\libg_nano.a(lib_a-puts.o)
                              ./Hardware/src/flash.o (puts)
d:/psx/rj/mounriver_studio/toolchain/risc-v embedded gcc/bin/../lib/gcc/riscv-none-embed/8.2.0/../../../../riscv-none-embed/lib/rv32imacxw/ilp32\libg_nano.a(lib_a-rand.o)
                              ./App/src/sl_protocol.o (srand)
d:/psx/rj/mounriver_studio/toolchain/risc-v embedded gcc/bin/../lib/gcc/riscv-none-embed/8.2.0/../../../../riscv-none-embed/lib/rv32imacxw/ilp32\libg_nano.a(lib_a-wbuf.o)
                              d:/psx/rj/mounriver_studio/toolchain/risc-v embedded gcc/bin/../lib/gcc/riscv-none-embed/8.2.0/../../../../riscv-none-embed/lib/rv32imacxw/ilp32\libg_nano.a(lib_a-puts.o) (__swbuf_r)
d:/psx/rj/mounriver_studio/toolchain/risc-v embedded gcc/bin/../lib/gcc/riscv-none-embed/8.2.0/../../../../riscv-none-embed/lib/rv32imacxw/ilp32\libg_nano.a(lib_a-wsetup.o)
                              d:/psx/rj/mounriver_studio/toolchain/risc-v embedded gcc/bin/../lib/gcc/riscv-none-embed/8.2.0/../../../../riscv-none-embed/lib/rv32imacxw/ilp32\libg_nano.a(lib_a-puts.o) (__swsetup_r)
d:/psx/rj/mounriver_studio/toolchain/risc-v embedded gcc/bin/../lib/gcc/riscv-none-embed/8.2.0/../../../../riscv-none-embed/lib/rv32imacxw/ilp32\libg_nano.a(lib_a-fflush.o)
                              d:/psx/rj/mounriver_studio/toolchain/risc-v embedded gcc/bin/../lib/gcc/riscv-none-embed/8.2.0/../../../../riscv-none-embed/lib/rv32imacxw/ilp32\libg_nano.a(lib_a-wbuf.o) (_fflush_r)
d:/psx/rj/mounriver_studio/toolchain/risc-v embedded gcc/bin/../lib/gcc/riscv-none-embed/8.2.0/../../../../riscv-none-embed/lib/rv32imacxw/ilp32\libg_nano.a(lib_a-findfp.o)
                              d:/psx/rj/mounriver_studio/toolchain/risc-v embedded gcc/bin/../lib/gcc/riscv-none-embed/8.2.0/../../../../riscv-none-embed/lib/rv32imacxw/ilp32\libg_nano.a(lib_a-printf.o) (__sinit)
d:/psx/rj/mounriver_studio/toolchain/risc-v embedded gcc/bin/../lib/gcc/riscv-none-embed/8.2.0/../../../../riscv-none-embed/lib/rv32imacxw/ilp32\libg_nano.a(lib_a-fwalk.o)
                              d:/psx/rj/mounriver_studio/toolchain/risc-v embedded gcc/bin/../lib/gcc/riscv-none-embed/8.2.0/../../../../riscv-none-embed/lib/rv32imacxw/ilp32\libg_nano.a(lib_a-findfp.o) (_fwalk)
d:/psx/rj/mounriver_studio/toolchain/risc-v embedded gcc/bin/../lib/gcc/riscv-none-embed/8.2.0/../../../../riscv-none-embed/lib/rv32imacxw/ilp32\libg_nano.a(lib_a-impure.o)
                              d:/psx/rj/mounriver_studio/toolchain/risc-v embedded gcc/bin/../lib/gcc/riscv-none-embed/8.2.0/../../../../riscv-none-embed/lib/rv32imacxw/ilp32\libg_nano.a(lib_a-fflush.o) (_global_impure_ptr)
d:/psx/rj/mounriver_studio/toolchain/risc-v embedded gcc/bin/../lib/gcc/riscv-none-embed/8.2.0/../../../../riscv-none-embed/lib/rv32imacxw/ilp32\libg_nano.a(lib_a-makebuf.o)
                              d:/psx/rj/mounriver_studio/toolchain/risc-v embedded gcc/bin/../lib/gcc/riscv-none-embed/8.2.0/../../../../riscv-none-embed/lib/rv32imacxw/ilp32\libg_nano.a(lib_a-wsetup.o) (__smakebuf_r)
d:/psx/rj/mounriver_studio/toolchain/risc-v embedded gcc/bin/../lib/gcc/riscv-none-embed/8.2.0/../../../../riscv-none-embed/lib/rv32imacxw/ilp32\libg_nano.a(lib_a-malloc.o)
                              d:/psx/rj/mounriver_studio/toolchain/risc-v embedded gcc/bin/../lib/gcc/riscv-none-embed/8.2.0/../../../../riscv-none-embed/lib/rv32imacxw/ilp32\libg_nano.a(lib_a-rand.o) (malloc)
d:/psx/rj/mounriver_studio/toolchain/risc-v embedded gcc/bin/../lib/gcc/riscv-none-embed/8.2.0/../../../../riscv-none-embed/lib/rv32imacxw/ilp32\libg_nano.a(lib_a-nano-freer.o)
                              d:/psx/rj/mounriver_studio/toolchain/risc-v embedded gcc/bin/../lib/gcc/riscv-none-embed/8.2.0/../../../../riscv-none-embed/lib/rv32imacxw/ilp32\libg_nano.a(lib_a-wsetup.o) (_free_r)
d:/psx/rj/mounriver_studio/toolchain/risc-v embedded gcc/bin/../lib/gcc/riscv-none-embed/8.2.0/../../../../riscv-none-embed/lib/rv32imacxw/ilp32\libg_nano.a(lib_a-nano-mallocr.o)
                              d:/psx/rj/mounriver_studio/toolchain/risc-v embedded gcc/bin/../lib/gcc/riscv-none-embed/8.2.0/../../../../riscv-none-embed/lib/rv32imacxw/ilp32\libg_nano.a(lib_a-findfp.o) (_malloc_r)
d:/psx/rj/mounriver_studio/toolchain/risc-v embedded gcc/bin/../lib/gcc/riscv-none-embed/8.2.0/../../../../riscv-none-embed/lib/rv32imacxw/ilp32\libg_nano.a(lib_a-nano-vfprintf.o)
                              d:/psx/rj/mounriver_studio/toolchain/risc-v embedded gcc/bin/../lib/gcc/riscv-none-embed/8.2.0/../../../../riscv-none-embed/lib/rv32imacxw/ilp32\libg_nano.a(lib_a-printf.o) (_vfprintf_r)
d:/psx/rj/mounriver_studio/toolchain/risc-v embedded gcc/bin/../lib/gcc/riscv-none-embed/8.2.0/../../../../riscv-none-embed/lib/rv32imacxw/ilp32\libg_nano.a(lib_a-nano-vfprintf_i.o)
                              d:/psx/rj/mounriver_studio/toolchain/risc-v embedded gcc/bin/../lib/gcc/riscv-none-embed/8.2.0/../../../../riscv-none-embed/lib/rv32imacxw/ilp32\libg_nano.a(lib_a-nano-vfprintf.o) (_printf_i)
d:/psx/rj/mounriver_studio/toolchain/risc-v embedded gcc/bin/../lib/gcc/riscv-none-embed/8.2.0/../../../../riscv-none-embed/lib/rv32imacxw/ilp32\libg_nano.a(lib_a-putc.o)
                              d:/psx/rj/mounriver_studio/toolchain/risc-v embedded gcc/bin/../lib/gcc/riscv-none-embed/8.2.0/../../../../riscv-none-embed/lib/rv32imacxw/ilp32\libg_nano.a(lib_a-putchar.o) (_putc_r)
d:/psx/rj/mounriver_studio/toolchain/risc-v embedded gcc/bin/../lib/gcc/riscv-none-embed/8.2.0/../../../../riscv-none-embed/lib/rv32imacxw/ilp32\libg_nano.a(lib_a-sbrkr.o)
                              d:/psx/rj/mounriver_studio/toolchain/risc-v embedded gcc/bin/../lib/gcc/riscv-none-embed/8.2.0/../../../../riscv-none-embed/lib/rv32imacxw/ilp32\libg_nano.a(lib_a-nano-mallocr.o) (_sbrk_r)
d:/psx/rj/mounriver_studio/toolchain/risc-v embedded gcc/bin/../lib/gcc/riscv-none-embed/8.2.0/../../../../riscv-none-embed/lib/rv32imacxw/ilp32\libg_nano.a(lib_a-stdio.o)
                              d:/psx/rj/mounriver_studio/toolchain/risc-v embedded gcc/bin/../lib/gcc/riscv-none-embed/8.2.0/../../../../riscv-none-embed/lib/rv32imacxw/ilp32\libg_nano.a(lib_a-findfp.o) (__sread)
d:/psx/rj/mounriver_studio/toolchain/risc-v embedded gcc/bin/../lib/gcc/riscv-none-embed/8.2.0/../../../../riscv-none-embed/lib/rv32imacxw/ilp32\libg_nano.a(lib_a-writer.o)
                              d:/psx/rj/mounriver_studio/toolchain/risc-v embedded gcc/bin/../lib/gcc/riscv-none-embed/8.2.0/../../../../riscv-none-embed/lib/rv32imacxw/ilp32\libg_nano.a(lib_a-stdio.o) (_write_r)
d:/psx/rj/mounriver_studio/toolchain/risc-v embedded gcc/bin/../lib/gcc/riscv-none-embed/8.2.0/../../../../riscv-none-embed/lib/rv32imacxw/ilp32\libg_nano.a(lib_a-closer.o)
                              d:/psx/rj/mounriver_studio/toolchain/risc-v embedded gcc/bin/../lib/gcc/riscv-none-embed/8.2.0/../../../../riscv-none-embed/lib/rv32imacxw/ilp32\libg_nano.a(lib_a-stdio.o) (_close_r)
d:/psx/rj/mounriver_studio/toolchain/risc-v embedded gcc/bin/../lib/gcc/riscv-none-embed/8.2.0/../../../../riscv-none-embed/lib/rv32imacxw/ilp32\libg_nano.a(lib_a-fstatr.o)
                              d:/psx/rj/mounriver_studio/toolchain/risc-v embedded gcc/bin/../lib/gcc/riscv-none-embed/8.2.0/../../../../riscv-none-embed/lib/rv32imacxw/ilp32\libg_nano.a(lib_a-makebuf.o) (_fstat_r)
d:/psx/rj/mounriver_studio/toolchain/risc-v embedded gcc/bin/../lib/gcc/riscv-none-embed/8.2.0/../../../../riscv-none-embed/lib/rv32imacxw/ilp32\libg_nano.a(lib_a-fvwrite.o)
                              d:/psx/rj/mounriver_studio/toolchain/risc-v embedded gcc/bin/../lib/gcc/riscv-none-embed/8.2.0/../../../../riscv-none-embed/lib/rv32imacxw/ilp32\libg_nano.a(lib_a-nano-vfprintf.o) (__sfvwrite_r)
d:/psx/rj/mounriver_studio/toolchain/risc-v embedded gcc/bin/../lib/gcc/riscv-none-embed/8.2.0/../../../../riscv-none-embed/lib/rv32imacxw/ilp32\libg_nano.a(lib_a-isattyr.o)
                              d:/psx/rj/mounriver_studio/toolchain/risc-v embedded gcc/bin/../lib/gcc/riscv-none-embed/8.2.0/../../../../riscv-none-embed/lib/rv32imacxw/ilp32\libg_nano.a(lib_a-makebuf.o) (_isatty_r)
d:/psx/rj/mounriver_studio/toolchain/risc-v embedded gcc/bin/../lib/gcc/riscv-none-embed/8.2.0/../../../../riscv-none-embed/lib/rv32imacxw/ilp32\libg_nano.a(lib_a-lseekr.o)
                              d:/psx/rj/mounriver_studio/toolchain/risc-v embedded gcc/bin/../lib/gcc/riscv-none-embed/8.2.0/../../../../riscv-none-embed/lib/rv32imacxw/ilp32\libg_nano.a(lib_a-stdio.o) (_lseek_r)
d:/psx/rj/mounriver_studio/toolchain/risc-v embedded gcc/bin/../lib/gcc/riscv-none-embed/8.2.0/../../../../riscv-none-embed/lib/rv32imacxw/ilp32\libg_nano.a(lib_a-memchr.o)
                              d:/psx/rj/mounriver_studio/toolchain/risc-v embedded gcc/bin/../lib/gcc/riscv-none-embed/8.2.0/../../../../riscv-none-embed/lib/rv32imacxw/ilp32\libg_nano.a(lib_a-nano-vfprintf.o) (memchr)
d:/psx/rj/mounriver_studio/toolchain/risc-v embedded gcc/bin/../lib/gcc/riscv-none-embed/8.2.0/../../../../riscv-none-embed/lib/rv32imacxw/ilp32\libg_nano.a(lib_a-memmove.o)
                              d:/psx/rj/mounriver_studio/toolchain/risc-v embedded gcc/bin/../lib/gcc/riscv-none-embed/8.2.0/../../../../riscv-none-embed/lib/rv32imacxw/ilp32\libg_nano.a(lib_a-fvwrite.o) (memmove)
d:/psx/rj/mounriver_studio/toolchain/risc-v embedded gcc/bin/../lib/gcc/riscv-none-embed/8.2.0/../../../../riscv-none-embed/lib/rv32imacxw/ilp32\libg_nano.a(lib_a-mlock.o)
                              d:/psx/rj/mounriver_studio/toolchain/risc-v embedded gcc/bin/../lib/gcc/riscv-none-embed/8.2.0/../../../../riscv-none-embed/lib/rv32imacxw/ilp32\libg_nano.a(lib_a-nano-freer.o) (__malloc_lock)
d:/psx/rj/mounriver_studio/toolchain/risc-v embedded gcc/bin/../lib/gcc/riscv-none-embed/8.2.0/../../../../riscv-none-embed/lib/rv32imacxw/ilp32\libg_nano.a(lib_a-nano-reallocr.o)
                              d:/psx/rj/mounriver_studio/toolchain/risc-v embedded gcc/bin/../lib/gcc/riscv-none-embed/8.2.0/../../../../riscv-none-embed/lib/rv32imacxw/ilp32\libg_nano.a(lib_a-fvwrite.o) (_realloc_r)
d:/psx/rj/mounriver_studio/toolchain/risc-v embedded gcc/bin/../lib/gcc/riscv-none-embed/8.2.0/../../../../riscv-none-embed/lib/rv32imacxw/ilp32\libg_nano.a(lib_a-readr.o)
                              d:/psx/rj/mounriver_studio/toolchain/risc-v embedded gcc/bin/../lib/gcc/riscv-none-embed/8.2.0/../../../../riscv-none-embed/lib/rv32imacxw/ilp32\libg_nano.a(lib_a-stdio.o) (_read_r)
d:/psx/rj/mounriver_studio/toolchain/risc-v embedded gcc/bin/../lib/gcc/riscv-none-embed/8.2.0/../../../../riscv-none-embed/lib/rv32imacxw/ilp32\libg_nano.a(lib_a-reent.o)
                              d:/psx/rj/mounriver_studio/toolchain/risc-v embedded gcc/bin/../lib/gcc/riscv-none-embed/8.2.0/../../../../riscv-none-embed/lib/rv32imacxw/ilp32\libg_nano.a(lib_a-sbrkr.o) (errno)
d:/psx/rj/mounriver_studio/toolchain/risc-v embedded gcc/bin/../lib/gcc/riscv-none-embed/8.2.0/../../../../riscv-none-embed/lib/rv32imacxw/ilp32\libg_nano.a(lib_a-nano-msizer.o)
                              d:/psx/rj/mounriver_studio/toolchain/risc-v embedded gcc/bin/../lib/gcc/riscv-none-embed/8.2.0/../../../../riscv-none-embed/lib/rv32imacxw/ilp32\libg_nano.a(lib_a-nano-reallocr.o) (_malloc_usable_size_r)
d:/psx/rj/mounriver_studio/toolchain/risc-v embedded gcc/bin/../lib/gcc/riscv-none-embed/8.2.0/../../../../riscv-none-embed/lib/rv32imacxw/ilp32\libnosys.a(close.o)
                              d:/psx/rj/mounriver_studio/toolchain/risc-v embedded gcc/bin/../lib/gcc/riscv-none-embed/8.2.0/../../../../riscv-none-embed/lib/rv32imacxw/ilp32\libg_nano.a(lib_a-closer.o) (_close)
d:/psx/rj/mounriver_studio/toolchain/risc-v embedded gcc/bin/../lib/gcc/riscv-none-embed/8.2.0/../../../../riscv-none-embed/lib/rv32imacxw/ilp32\libnosys.a(fstat.o)
                              d:/psx/rj/mounriver_studio/toolchain/risc-v embedded gcc/bin/../lib/gcc/riscv-none-embed/8.2.0/../../../../riscv-none-embed/lib/rv32imacxw/ilp32\libg_nano.a(lib_a-fstatr.o) (_fstat)
d:/psx/rj/mounriver_studio/toolchain/risc-v embedded gcc/bin/../lib/gcc/riscv-none-embed/8.2.0/../../../../riscv-none-embed/lib/rv32imacxw/ilp32\libnosys.a(isatty.o)
                              d:/psx/rj/mounriver_studio/toolchain/risc-v embedded gcc/bin/../lib/gcc/riscv-none-embed/8.2.0/../../../../riscv-none-embed/lib/rv32imacxw/ilp32\libg_nano.a(lib_a-isattyr.o) (_isatty)
d:/psx/rj/mounriver_studio/toolchain/risc-v embedded gcc/bin/../lib/gcc/riscv-none-embed/8.2.0/../../../../riscv-none-embed/lib/rv32imacxw/ilp32\libnosys.a(lseek.o)
                              d:/psx/rj/mounriver_studio/toolchain/risc-v embedded gcc/bin/../lib/gcc/riscv-none-embed/8.2.0/../../../../riscv-none-embed/lib/rv32imacxw/ilp32\libg_nano.a(lib_a-lseekr.o) (_lseek)
d:/psx/rj/mounriver_studio/toolchain/risc-v embedded gcc/bin/../lib/gcc/riscv-none-embed/8.2.0/../../../../riscv-none-embed/lib/rv32imacxw/ilp32\libnosys.a(read.o)
                              d:/psx/rj/mounriver_studio/toolchain/risc-v embedded gcc/bin/../lib/gcc/riscv-none-embed/8.2.0/../../../../riscv-none-embed/lib/rv32imacxw/ilp32\libg_nano.a(lib_a-readr.o) (_read)

Allocating common symbols
Common symbol       size              file

errno               0x4               d:/psx/rj/mounriver_studio/toolchain/risc-v embedded gcc/bin/../lib/gcc/riscv-none-embed/8.2.0/../../../../riscv-none-embed/lib/rv32imacxw/ilp32\libg_nano.a(lib_a-reent.o)

Discarded input sections

 .text          0x0000000000000000        0x0 ./User/ch32l103_it.o
 .data          0x0000000000000000        0x0 ./User/ch32l103_it.o
 .bss           0x0000000000000000        0x0 ./User/ch32l103_it.o
 .text          0x0000000000000000        0x0 ./User/main.o
 .data          0x0000000000000000        0x0 ./User/main.o
 .bss           0x0000000000000000        0x0 ./User/main.o
 .text          0x0000000000000000        0x0 ./User/system_ch32l103.o
 .data          0x0000000000000000        0x0 ./User/system_ch32l103.o
 .bss           0x0000000000000000        0x0 ./User/system_ch32l103.o
 .text          0x0000000000000000        0x0 ./Startup/startup_ch32l103.o
 .data          0x0000000000000000        0x0 ./Startup/startup_ch32l103.o
 .bss           0x0000000000000000        0x0 ./Startup/startup_ch32l103.o
 .text          0x0000000000000000        0x0 ./Peripheral/src/ch32l103_adc.o
 .data          0x0000000000000000        0x0 ./Peripheral/src/ch32l103_adc.o
 .bss           0x0000000000000000        0x0 ./Peripheral/src/ch32l103_adc.o
 .text.ADC_StructInit
                0x0000000000000000       0x1a ./Peripheral/src/ch32l103_adc.o
 .text.ADC_ITConfig
                0x0000000000000000       0x16 ./Peripheral/src/ch32l103_adc.o
 .text.ADC_GetSoftwareStartConvStatus
                0x0000000000000000        0x8 ./Peripheral/src/ch32l103_adc.o
 .text.ADC_DiscModeChannelCountConfig
                0x0000000000000000       0x12 ./Peripheral/src/ch32l103_adc.o
 .text.ADC_DiscModeCmd
                0x0000000000000000       0x1a ./Peripheral/src/ch32l103_adc.o
 .text.ADC_ExternalTrigConvCmd
                0x0000000000000000       0x18 ./Peripheral/src/ch32l103_adc.o
 .text.ADC_GetDualModeConversionValue
                0x0000000000000000        0xa ./Peripheral/src/ch32l103_adc.o
 .text.ADC_AutoInjectedConvCmd
                0x0000000000000000       0x12 ./Peripheral/src/ch32l103_adc.o
 .text.ADC_InjectedDiscModeCmd
                0x0000000000000000       0x14 ./Peripheral/src/ch32l103_adc.o
 .text.ADC_ExternalTrigInjectedConvConfig
                0x0000000000000000        0xe ./Peripheral/src/ch32l103_adc.o
 .text.ADC_ExternalTrigInjectedConvCmd
                0x0000000000000000       0x14 ./Peripheral/src/ch32l103_adc.o
 .text.ADC_SoftwareStartInjectedConvCmd
                0x0000000000000000       0x18 ./Peripheral/src/ch32l103_adc.o
 .text.ADC_GetSoftwareStartInjectedConvCmdStatus
                0x0000000000000000        0x8 ./Peripheral/src/ch32l103_adc.o
 .text.ADC_InjectedChannelConfig
                0x0000000000000000       0x7a ./Peripheral/src/ch32l103_adc.o
 .text.ADC_InjectedSequencerLengthConfig
                0x0000000000000000       0x14 ./Peripheral/src/ch32l103_adc.o
 .text.ADC_SetInjectedOffset
                0x0000000000000000       0x14 ./Peripheral/src/ch32l103_adc.o
 .text.ADC_GetInjectedConversionValue
                0x0000000000000000       0x1c ./Peripheral/src/ch32l103_adc.o
 .text.ADC_AnalogWatchdogCmd
                0x0000000000000000       0x12 ./Peripheral/src/ch32l103_adc.o
 .text.ADC_AnalogWatchdogThresholdsConfig
                0x0000000000000000        0x6 ./Peripheral/src/ch32l103_adc.o
 .text.ADC_AnalogWatchdogSingleChannelConfig
                0x0000000000000000        0xa ./Peripheral/src/ch32l103_adc.o
 .text.ADC_TempSensorVrefintCmd
                0x0000000000000000       0x20 ./Peripheral/src/ch32l103_adc.o
 .text.ADC_ClearFlag
                0x0000000000000000        0x8 ./Peripheral/src/ch32l103_adc.o
 .text.ADC_GetITStatus
                0x0000000000000000       0x1c ./Peripheral/src/ch32l103_adc.o
 .text.ADC_ClearITPendingBit
                0x0000000000000000        0xa ./Peripheral/src/ch32l103_adc.o
 .text.TempSensor_Volt_To_Temper
                0x0000000000000000       0x28 ./Peripheral/src/ch32l103_adc.o
 .text.ADC_TKey_WakeUpCmd
                0x0000000000000000       0x2c ./Peripheral/src/ch32l103_adc.o
 .text.ADC_TKey_ChannelxMulShieldCmd
                0x0000000000000000       0x1a ./Peripheral/src/ch32l103_adc.o
 .text.ADC_TKey_MulShieldCmd
                0x0000000000000000       0x12 ./Peripheral/src/ch32l103_adc.o
 .text.ADC_OffsetCalibrationConfig
                0x0000000000000000       0x22 ./Peripheral/src/ch32l103_adc.o
 .text.ADC_AnalogWatchdogResetCmd
                0x0000000000000000       0x10 ./Peripheral/src/ch32l103_adc.o
 .text          0x0000000000000000        0x0 ./Peripheral/src/ch32l103_bkp.o
 .data          0x0000000000000000        0x0 ./Peripheral/src/ch32l103_bkp.o
 .bss           0x0000000000000000        0x0 ./Peripheral/src/ch32l103_bkp.o
 .text.BKP_DeInit
                0x0000000000000000       0x24 ./Peripheral/src/ch32l103_bkp.o
 .text.BKP_TamperPinLevelConfig
                0x0000000000000000       0x20 ./Peripheral/src/ch32l103_bkp.o
 .text.BKP_TamperPinCmd
                0x0000000000000000       0x20 ./Peripheral/src/ch32l103_bkp.o
 .text.BKP_ITConfig
                0x0000000000000000       0x20 ./Peripheral/src/ch32l103_bkp.o
 .text.BKP_RTCOutputConfig
                0x0000000000000000       0x18 ./Peripheral/src/ch32l103_bkp.o
 .text.BKP_SetRTCCalibrationValue
                0x0000000000000000       0x18 ./Peripheral/src/ch32l103_bkp.o
 .text.BKP_WriteBackupRegister
                0x0000000000000000       0x1c ./Peripheral/src/ch32l103_bkp.o
 .text.BKP_ReadBackupRegister
                0x0000000000000000       0x1c ./Peripheral/src/ch32l103_bkp.o
 .text.BKP_GetFlagStatus
                0x0000000000000000        0xe ./Peripheral/src/ch32l103_bkp.o
 .text.BKP_ClearFlag
                0x0000000000000000       0x12 ./Peripheral/src/ch32l103_bkp.o
 .text.BKP_GetITStatus
                0x0000000000000000        0xe ./Peripheral/src/ch32l103_bkp.o
 .text.BKP_ClearITPendingBit
                0x0000000000000000       0x12 ./Peripheral/src/ch32l103_bkp.o
 .debug_info    0x0000000000000000      0xdc5 ./Peripheral/src/ch32l103_bkp.o
 .debug_abbrev  0x0000000000000000      0x2cc ./Peripheral/src/ch32l103_bkp.o
 .debug_loc     0x0000000000000000       0xd8 ./Peripheral/src/ch32l103_bkp.o
 .debug_aranges
                0x0000000000000000       0x78 ./Peripheral/src/ch32l103_bkp.o
 .debug_ranges  0x0000000000000000       0x68 ./Peripheral/src/ch32l103_bkp.o
 .debug_line    0x0000000000000000      0x614 ./Peripheral/src/ch32l103_bkp.o
 .debug_str     0x0000000000000000      0x876 ./Peripheral/src/ch32l103_bkp.o
 .comment       0x0000000000000000       0x34 ./Peripheral/src/ch32l103_bkp.o
 .debug_frame   0x0000000000000000       0xec ./Peripheral/src/ch32l103_bkp.o
 .text          0x0000000000000000        0x0 ./Peripheral/src/ch32l103_can.o
 .data          0x0000000000000000        0x0 ./Peripheral/src/ch32l103_can.o
 .bss           0x0000000000000000        0x0 ./Peripheral/src/ch32l103_can.o
 .text.CAN_DeInit
                0x0000000000000000       0x3a ./Peripheral/src/ch32l103_can.o
 .text.CAN_Init
                0x0000000000000000       0xee ./Peripheral/src/ch32l103_can.o
 .text.CAN_FilterInit
                0x0000000000000000       0xee ./Peripheral/src/ch32l103_can.o
 .text.CAN_StructInit
                0x0000000000000000       0x24 ./Peripheral/src/ch32l103_can.o
 .text.CAN_SlaveStartBank
                0x0000000000000000       0x38 ./Peripheral/src/ch32l103_can.o
 .text.CAN_DBGFreeze
                0x0000000000000000       0x14 ./Peripheral/src/ch32l103_can.o
 .text.CAN_TTComModeCmd
                0x0000000000000000       0x58 ./Peripheral/src/ch32l103_can.o
 .text.CAN_Transmit
                0x0000000000000000       0xc2 ./Peripheral/src/ch32l103_can.o
 .text.CAN_TransmitStatus
                0x0000000000000000       0x62 ./Peripheral/src/ch32l103_can.o
 .text.CAN_CancelTransmit
                0x0000000000000000       0x2a ./Peripheral/src/ch32l103_can.o
 .text.CAN_Receive
                0x0000000000000000       0x8c ./Peripheral/src/ch32l103_can.o
 .text.CAN_FIFORelease
                0x0000000000000000       0x16 ./Peripheral/src/ch32l103_can.o
 .text.CAN_MessagePending
                0x0000000000000000       0x16 ./Peripheral/src/ch32l103_can.o
 .text.CAN_OperatingModeRequest
                0x0000000000000000       0x72 ./Peripheral/src/ch32l103_can.o
 .text.CAN_Sleep
                0x0000000000000000       0x16 ./Peripheral/src/ch32l103_can.o
 .text.CAN_WakeUp
                0x0000000000000000       0x1e ./Peripheral/src/ch32l103_can.o
 .text.CAN_GetLastErrorCode
                0x0000000000000000        0x8 ./Peripheral/src/ch32l103_can.o
 .text.CAN_GetReceiveErrorCounter
                0x0000000000000000        0x6 ./Peripheral/src/ch32l103_can.o
 .text.CAN_GetLSBTransmitErrorCounter
                0x0000000000000000        0xa ./Peripheral/src/ch32l103_can.o
 .text.CAN_ITConfig
                0x0000000000000000       0x12 ./Peripheral/src/ch32l103_can.o
 .text.CAN_GetFlagStatus
                0x0000000000000000       0x56 ./Peripheral/src/ch32l103_can.o
 .text.CAN_ClearFlag
                0x0000000000000000       0x40 ./Peripheral/src/ch32l103_can.o
 .text.CAN_GetITStatus
                0x0000000000000000       0xd0 ./Peripheral/src/ch32l103_can.o
 .text.CAN_ClearITPendingBit
                0x0000000000000000       0x94 ./Peripheral/src/ch32l103_can.o
 .text.CAN_BS1_ModeConfig
                0x0000000000000000       0x36 ./Peripheral/src/ch32l103_can.o
 .text.CAN_BusOff_ErrCntConfig
                0x0000000000000000       0x10 ./Peripheral/src/ch32l103_can.o
 .text.CANFD_Restrict_ModeCmd
                0x0000000000000000       0x12 ./Peripheral/src/ch32l103_can.o
 .text.CANFD_Init
                0x0000000000000000      0x1a2 ./Peripheral/src/ch32l103_can.o
 .text.CANFD_StructInit
                0x0000000000000000       0x48 ./Peripheral/src/ch32l103_can.o
 .text.CANFD_Transmit
                0x0000000000000000       0xac ./Peripheral/src/ch32l103_can.o
 .text.CANFD_Receive
                0x0000000000000000       0xd6 ./Peripheral/src/ch32l103_can.o
 .text.CANFD_GetTransmitDelayOffsetVal
                0x0000000000000000        0xa ./Peripheral/src/ch32l103_can.o
 .text.CANFD_TransmitMailbox_DMAAdr
                0x0000000000000000        0xa ./Peripheral/src/ch32l103_can.o
 .text.CANFD_ReceiveFIFO_DMAAdr
                0x0000000000000000        0xa ./Peripheral/src/ch32l103_can.o
 .debug_info    0x0000000000000000     0x1df4 ./Peripheral/src/ch32l103_can.o
 .debug_abbrev  0x0000000000000000      0x402 ./Peripheral/src/ch32l103_can.o
 .debug_loc     0x0000000000000000      0xcb1 ./Peripheral/src/ch32l103_can.o
 .debug_aranges
                0x0000000000000000      0x128 ./Peripheral/src/ch32l103_can.o
 .debug_ranges  0x0000000000000000      0x148 ./Peripheral/src/ch32l103_can.o
 .debug_line    0x0000000000000000     0x266d ./Peripheral/src/ch32l103_can.o
 .debug_str     0x0000000000000000      0xe78 ./Peripheral/src/ch32l103_can.o
 .comment       0x0000000000000000       0x34 ./Peripheral/src/ch32l103_can.o
 .debug_frame   0x0000000000000000      0x23c ./Peripheral/src/ch32l103_can.o
 .text          0x0000000000000000        0x0 ./Peripheral/src/ch32l103_crc.o
 .data          0x0000000000000000        0x0 ./Peripheral/src/ch32l103_crc.o
 .bss           0x0000000000000000        0x0 ./Peripheral/src/ch32l103_crc.o
 .text.CRC_ResetDR
                0x0000000000000000        0xa ./Peripheral/src/ch32l103_crc.o
 .text.CRC_CalcCRC
                0x0000000000000000        0xa ./Peripheral/src/ch32l103_crc.o
 .text.CRC_CalcBlockCRC
                0x0000000000000000       0x20 ./Peripheral/src/ch32l103_crc.o
 .text.CRC_GetCRC
                0x0000000000000000        0x8 ./Peripheral/src/ch32l103_crc.o
 .text.CRC_SetIDRegister
                0x0000000000000000        0x8 ./Peripheral/src/ch32l103_crc.o
 .text.CRC_GetIDRegister
                0x0000000000000000        0x8 ./Peripheral/src/ch32l103_crc.o
 .debug_info    0x0000000000000000      0xadc ./Peripheral/src/ch32l103_crc.o
 .debug_abbrev  0x0000000000000000      0x25f ./Peripheral/src/ch32l103_crc.o
 .debug_loc     0x0000000000000000       0x75 ./Peripheral/src/ch32l103_crc.o
 .debug_aranges
                0x0000000000000000       0x48 ./Peripheral/src/ch32l103_crc.o
 .debug_ranges  0x0000000000000000       0x38 ./Peripheral/src/ch32l103_crc.o
 .debug_line    0x0000000000000000      0x38a ./Peripheral/src/ch32l103_crc.o
 .debug_str     0x0000000000000000      0x673 ./Peripheral/src/ch32l103_crc.o
 .comment       0x0000000000000000       0x34 ./Peripheral/src/ch32l103_crc.o
 .debug_frame   0x0000000000000000       0x70 ./Peripheral/src/ch32l103_crc.o
 .text          0x0000000000000000        0x0 ./Peripheral/src/ch32l103_dbgmcu.o
 .data          0x0000000000000000        0x0 ./Peripheral/src/ch32l103_dbgmcu.o
 .bss           0x0000000000000000        0x0 ./Peripheral/src/ch32l103_dbgmcu.o
 .text.DBGMCU_GetREVID
                0x0000000000000000        0xa ./Peripheral/src/ch32l103_dbgmcu.o
 .text.DBGMCU_GetDEVID
                0x0000000000000000        0xa ./Peripheral/src/ch32l103_dbgmcu.o
 .text.__get_DEBUG_CR
                0x0000000000000000        0x6 ./Peripheral/src/ch32l103_dbgmcu.o
 .text.__set_DEBUG_CR
                0x0000000000000000        0x6 ./Peripheral/src/ch32l103_dbgmcu.o
 .text.DBGMCU_Config
                0x0000000000000000       0x14 ./Peripheral/src/ch32l103_dbgmcu.o
 .text          0x0000000000000000        0x0 ./Peripheral/src/ch32l103_dma.o
 .data          0x0000000000000000        0x0 ./Peripheral/src/ch32l103_dma.o
 .bss           0x0000000000000000        0x0 ./Peripheral/src/ch32l103_dma.o
 .text.DMA_StructInit
                0x0000000000000000       0x2e ./Peripheral/src/ch32l103_dma.o
 .text.DMA_SetCurrDataCounter
                0x0000000000000000        0x4 ./Peripheral/src/ch32l103_dma.o
 .text.DMA_GetCurrDataCounter
                0x0000000000000000        0x8 ./Peripheral/src/ch32l103_dma.o
 .text.DMA_ClearFlag
                0x0000000000000000        0x8 ./Peripheral/src/ch32l103_dma.o
 .text          0x0000000000000000        0x0 ./Peripheral/src/ch32l103_exti.o
 .data          0x0000000000000000        0x0 ./Peripheral/src/ch32l103_exti.o
 .bss           0x0000000000000000        0x0 ./Peripheral/src/ch32l103_exti.o
 .text.EXTI_DeInit
                0x0000000000000000       0x22 ./Peripheral/src/ch32l103_exti.o
 .text.EXTI_StructInit
                0x0000000000000000       0x12 ./Peripheral/src/ch32l103_exti.o
 .text.EXTI_GenerateSWInterrupt
                0x0000000000000000       0x10 ./Peripheral/src/ch32l103_exti.o
 .text.EXTI_GetFlagStatus
                0x0000000000000000       0x12 ./Peripheral/src/ch32l103_exti.o
 .text.EXTI_ClearFlag
                0x0000000000000000        0xa ./Peripheral/src/ch32l103_exti.o
 .text          0x0000000000000000        0x0 ./Peripheral/src/ch32l103_flash.o
 .data          0x0000000000000000        0x0 ./Peripheral/src/ch32l103_flash.o
 .bss           0x0000000000000000        0x0 ./Peripheral/src/ch32l103_flash.o
 .text.ROM_ERASE
                0x0000000000000000       0xba ./Peripheral/src/ch32l103_flash.o
 .text.FLASH_SetLatency
                0x0000000000000000        0xe ./Peripheral/src/ch32l103_flash.o
 .text.FLASH_Unlock
                0x0000000000000000       0x1a ./Peripheral/src/ch32l103_flash.o
 .text.FLASH_Lock
                0x0000000000000000        0xe ./Peripheral/src/ch32l103_flash.o
 .text.FLASH_GetUserOptionByte
                0x0000000000000000        0xa ./Peripheral/src/ch32l103_flash.o
 .text.FLASH_GetWriteProtectionOptionByte
                0x0000000000000000        0x8 ./Peripheral/src/ch32l103_flash.o
 .text.FLASH_GetReadOutProtectionStatus
                0x0000000000000000        0xc ./Peripheral/src/ch32l103_flash.o
 .text.FLASH_ITConfig
                0x0000000000000000       0x1e ./Peripheral/src/ch32l103_flash.o
 .text.FLASH_GetFlagStatus
                0x0000000000000000       0x1e ./Peripheral/src/ch32l103_flash.o
 .text.FLASH_ClearFlag
                0x0000000000000000        0x8 ./Peripheral/src/ch32l103_flash.o
 .text.FLASH_GetStatus
                0x0000000000000000       0x18 ./Peripheral/src/ch32l103_flash.o
 .text.FLASH_GetBank1Status
                0x0000000000000000       0x18 ./Peripheral/src/ch32l103_flash.o
 .text.FLASH_WaitForLastOperation
                0x0000000000000000       0x34 ./Peripheral/src/ch32l103_flash.o
 .text.FLASH_ErasePage
                0x0000000000000000       0x58 ./Peripheral/src/ch32l103_flash.o
 .text.FLASH_EraseAllPages
                0x0000000000000000       0x54 ./Peripheral/src/ch32l103_flash.o
 .text.FLASH_EraseOptionBytes
                0x0000000000000000       0x82 ./Peripheral/src/ch32l103_flash.o
 .text.FLASH_WaitForLastBank1Operation
                0x0000000000000000       0x18 ./Peripheral/src/ch32l103_flash.o
 .text.FLASH_Unlock_Fast
                0x0000000000000000       0x1e ./Peripheral/src/ch32l103_flash.o
 .text.FLASH_Lock_Fast
                0x0000000000000000        0xe ./Peripheral/src/ch32l103_flash.o
 .text.FLASH_BufReset
                0x0000000000000000       0x34 ./Peripheral/src/ch32l103_flash.o
 .text.FLASH_BufLoad
                0x0000000000000000       0x36 ./Peripheral/src/ch32l103_flash.o
 .text.FLASH_ErasePage_Fast
                0x0000000000000000       0x36 ./Peripheral/src/ch32l103_flash.o
 .text.FLASH_EraseBlock_32K_Fast
                0x0000000000000000       0x3c ./Peripheral/src/ch32l103_flash.o
 .text.FLASH_ProgramPage_Fast
                0x0000000000000000       0x34 ./Peripheral/src/ch32l103_flash.o
 .text.FLASH_OptionBytePR
                0x0000000000000000       0x60 ./Peripheral/src/ch32l103_flash.o
 .text.FLASH_EnableWriteProtection
                0x0000000000000000       0xa6 ./Peripheral/src/ch32l103_flash.o
 .text.FLASH_EnableReadOutProtection
                0x0000000000000000       0x64 ./Peripheral/src/ch32l103_flash.o
 .text.FLASH_UserOptionByteConfig
                0x0000000000000000       0x62 ./Peripheral/src/ch32l103_flash.o
 .text.FLASH_ROM_ERASE
                0x0000000000000000      0x1ae ./Peripheral/src/ch32l103_flash.o
 .text.FLASH_ROM_WRITE
                0x0000000000000000       0xf8 ./Peripheral/src/ch32l103_flash.o
 .debug_info    0x0000000000000000     0x1407 ./Peripheral/src/ch32l103_flash.o
 .debug_abbrev  0x0000000000000000      0x488 ./Peripheral/src/ch32l103_flash.o
 .debug_loc     0x0000000000000000      0xad7 ./Peripheral/src/ch32l103_flash.o
 .debug_aranges
                0x0000000000000000      0x100 ./Peripheral/src/ch32l103_flash.o
 .debug_ranges  0x0000000000000000       0xf0 ./Peripheral/src/ch32l103_flash.o
 .debug_line    0x0000000000000000     0x1aeb ./Peripheral/src/ch32l103_flash.o
 .debug_str     0x0000000000000000      0xa67 ./Peripheral/src/ch32l103_flash.o
 .comment       0x0000000000000000       0x34 ./Peripheral/src/ch32l103_flash.o
 .debug_frame   0x0000000000000000      0x2c8 ./Peripheral/src/ch32l103_flash.o
 .text          0x0000000000000000        0x0 ./Peripheral/src/ch32l103_gpio.o
 .data          0x0000000000000000        0x0 ./Peripheral/src/ch32l103_gpio.o
 .bss           0x0000000000000000        0x0 ./Peripheral/src/ch32l103_gpio.o
 .text.GPIO_DeInit
                0x0000000000000000       0x82 ./Peripheral/src/ch32l103_gpio.o
 .text.GPIO_AFIODeInit
                0x0000000000000000       0x28 ./Peripheral/src/ch32l103_gpio.o
 .text.GPIO_StructInit
                0x0000000000000000        0xe ./Peripheral/src/ch32l103_gpio.o
 .text.GPIO_ReadInputData
                0x0000000000000000        0x8 ./Peripheral/src/ch32l103_gpio.o
 .text.GPIO_ReadOutputData
                0x0000000000000000        0x8 ./Peripheral/src/ch32l103_gpio.o
 .text.GPIO_ResetBits
                0x0000000000000000        0x4 ./Peripheral/src/ch32l103_gpio.o
 .text.GPIO_Write
                0x0000000000000000        0x4 ./Peripheral/src/ch32l103_gpio.o
 .text.GPIO_PinLockConfig
                0x0000000000000000       0x10 ./Peripheral/src/ch32l103_gpio.o
 .text.GPIO_EventOutputConfig
                0x0000000000000000       0x18 ./Peripheral/src/ch32l103_gpio.o
 .text.GPIO_EventOutputCmd
                0x0000000000000000       0x16 ./Peripheral/src/ch32l103_gpio.o
 .text          0x0000000000000000        0x0 ./Peripheral/src/ch32l103_i2c.o
 .data          0x0000000000000000        0x0 ./Peripheral/src/ch32l103_i2c.o
 .bss           0x0000000000000000        0x0 ./Peripheral/src/ch32l103_i2c.o
 .text.I2C_DeInit
                0x0000000000000000       0x4c ./Peripheral/src/ch32l103_i2c.o
 .text.I2C_Init
                0x0000000000000000      0x10c ./Peripheral/src/ch32l103_i2c.o
 .text.I2C_StructInit
                0x0000000000000000       0x18 ./Peripheral/src/ch32l103_i2c.o
 .text.I2C_Cmd  0x0000000000000000       0x18 ./Peripheral/src/ch32l103_i2c.o
 .text.I2C_DMACmd
                0x0000000000000000       0x1e ./Peripheral/src/ch32l103_i2c.o
 .text.I2C_DMALastTransferCmd
                0x0000000000000000       0x16 ./Peripheral/src/ch32l103_i2c.o
 .text.I2C_GenerateSTART
                0x0000000000000000       0x1a ./Peripheral/src/ch32l103_i2c.o
 .text.I2C_GenerateSTOP
                0x0000000000000000       0x1a ./Peripheral/src/ch32l103_i2c.o
 .text.I2C_AcknowledgeConfig
                0x0000000000000000       0x1a ./Peripheral/src/ch32l103_i2c.o
 .text.I2C_OwnAddress2Config
                0x0000000000000000       0x14 ./Peripheral/src/ch32l103_i2c.o
 .text.I2C_DualAddressCmd
                0x0000000000000000       0x18 ./Peripheral/src/ch32l103_i2c.o
 .text.I2C_GeneralCallCmd
                0x0000000000000000       0x1a ./Peripheral/src/ch32l103_i2c.o
 .text.I2C_ITConfig
                0x0000000000000000       0x12 ./Peripheral/src/ch32l103_i2c.o
 .text.I2C_SendData
                0x0000000000000000        0x4 ./Peripheral/src/ch32l103_i2c.o
 .text.I2C_ReceiveData
                0x0000000000000000        0x8 ./Peripheral/src/ch32l103_i2c.o
 .text.I2C_Send7bitAddress
                0x0000000000000000       0x12 ./Peripheral/src/ch32l103_i2c.o
 .text.I2C_ReadRegister
                0x0000000000000000       0x14 ./Peripheral/src/ch32l103_i2c.o
 .text.I2C_SoftwareResetCmd
                0x0000000000000000       0x12 ./Peripheral/src/ch32l103_i2c.o
 .text.I2C_NACKPositionConfig
                0x0000000000000000       0x22 ./Peripheral/src/ch32l103_i2c.o
 .text.I2C_SMBusAlertConfig
                0x0000000000000000       0x1a ./Peripheral/src/ch32l103_i2c.o
 .text.I2C_TransmitPEC
                0x0000000000000000       0x16 ./Peripheral/src/ch32l103_i2c.o
 .text.I2C_PECPositionConfig
                0x0000000000000000       0x18 ./Peripheral/src/ch32l103_i2c.o
 .text.I2C_CalculatePEC
                0x0000000000000000       0x1a ./Peripheral/src/ch32l103_i2c.o
 .text.I2C_GetPEC
                0x0000000000000000        0x6 ./Peripheral/src/ch32l103_i2c.o
 .text.I2C_ARPCmd
                0x0000000000000000       0x18 ./Peripheral/src/ch32l103_i2c.o
 .text.I2C_StretchClockCmd
                0x0000000000000000       0x1a ./Peripheral/src/ch32l103_i2c.o
 .text.I2C_FastModeDutyCycleConfig
                0x0000000000000000       0x1a ./Peripheral/src/ch32l103_i2c.o
 .text.I2C_CheckEvent
                0x0000000000000000       0x16 ./Peripheral/src/ch32l103_i2c.o
 .text.I2C_GetLastEvent
                0x0000000000000000        0xe ./Peripheral/src/ch32l103_i2c.o
 .text.I2C_GetFlagStatus
                0x0000000000000000       0x32 ./Peripheral/src/ch32l103_i2c.o
 .text.I2C_ClearFlag
                0x0000000000000000        0xc ./Peripheral/src/ch32l103_i2c.o
 .text.I2C_GetITStatus
                0x0000000000000000       0x20 ./Peripheral/src/ch32l103_i2c.o
 .text.I2C_ClearITPendingBit
                0x0000000000000000        0xc ./Peripheral/src/ch32l103_i2c.o
 .debug_info    0x0000000000000000     0x14af ./Peripheral/src/ch32l103_i2c.o
 .debug_abbrev  0x0000000000000000      0x3a7 ./Peripheral/src/ch32l103_i2c.o
 .debug_loc     0x0000000000000000      0x6cc ./Peripheral/src/ch32l103_i2c.o
 .debug_aranges
                0x0000000000000000      0x110 ./Peripheral/src/ch32l103_i2c.o
 .debug_ranges  0x0000000000000000      0x100 ./Peripheral/src/ch32l103_i2c.o
 .debug_line    0x0000000000000000     0x10e7 ./Peripheral/src/ch32l103_i2c.o
 .debug_str     0x0000000000000000      0xad7 ./Peripheral/src/ch32l103_i2c.o
 .comment       0x0000000000000000       0x34 ./Peripheral/src/ch32l103_i2c.o
 .debug_frame   0x0000000000000000      0x264 ./Peripheral/src/ch32l103_i2c.o
 .text          0x0000000000000000        0x0 ./Peripheral/src/ch32l103_iwdg.o
 .data          0x0000000000000000        0x0 ./Peripheral/src/ch32l103_iwdg.o
 .bss           0x0000000000000000        0x0 ./Peripheral/src/ch32l103_iwdg.o
 .text.IWDG_WriteAccessCmd
                0x0000000000000000        0x8 ./Peripheral/src/ch32l103_iwdg.o
 .text.IWDG_SetPrescaler
                0x0000000000000000        0x8 ./Peripheral/src/ch32l103_iwdg.o
 .text.IWDG_SetReload
                0x0000000000000000        0x8 ./Peripheral/src/ch32l103_iwdg.o
 .text.IWDG_ReloadCounter
                0x0000000000000000        0xe ./Peripheral/src/ch32l103_iwdg.o
 .text.IWDG_Enable
                0x0000000000000000       0x14 ./Peripheral/src/ch32l103_iwdg.o
 .text.IWDG_GetFlagStatus
                0x0000000000000000        0xe ./Peripheral/src/ch32l103_iwdg.o
 .debug_info    0x0000000000000000      0xb96 ./Peripheral/src/ch32l103_iwdg.o
 .debug_abbrev  0x0000000000000000      0x282 ./Peripheral/src/ch32l103_iwdg.o
 .debug_loc     0x0000000000000000       0x68 ./Peripheral/src/ch32l103_iwdg.o
 .debug_aranges
                0x0000000000000000       0x48 ./Peripheral/src/ch32l103_iwdg.o
 .debug_ranges  0x0000000000000000       0x38 ./Peripheral/src/ch32l103_iwdg.o
 .debug_line    0x0000000000000000      0x37f ./Peripheral/src/ch32l103_iwdg.o
 .debug_str     0x0000000000000000      0x6f0 ./Peripheral/src/ch32l103_iwdg.o
 .comment       0x0000000000000000       0x34 ./Peripheral/src/ch32l103_iwdg.o
 .debug_frame   0x0000000000000000       0x70 ./Peripheral/src/ch32l103_iwdg.o
 .text          0x0000000000000000        0x0 ./Peripheral/src/ch32l103_lptim.o
 .data          0x0000000000000000        0x0 ./Peripheral/src/ch32l103_lptim.o
 .bss           0x0000000000000000        0x0 ./Peripheral/src/ch32l103_lptim.o
 .text.LPTIM_DeInit
                0x0000000000000000       0x2c ./Peripheral/src/ch32l103_lptim.o
 .text.LPTIM_TimeBaseInit
                0x0000000000000000       0x7e ./Peripheral/src/ch32l103_lptim.o
 .text.LPTIM_TimeBaseStructInit
                0x0000000000000000       0x52 ./Peripheral/src/ch32l103_lptim.o
 .text.LPTIM_CounterDirIndicat_Cmd
                0x0000000000000000       0x18 ./Peripheral/src/ch32l103_lptim.o
 .text.LPTIM_OutCmd
                0x0000000000000000       0x18 ./Peripheral/src/ch32l103_lptim.o
 .text.LPTIM_Cmd
                0x0000000000000000       0x18 ./Peripheral/src/ch32l103_lptim.o
 .text.LPTIM_GetCounter
                0x0000000000000000        0xa ./Peripheral/src/ch32l103_lptim.o
 .text.LPTIM_SetAutoreload
                0x0000000000000000        0xa ./Peripheral/src/ch32l103_lptim.o
 .text.LPTIM_SetCompare
                0x0000000000000000        0xa ./Peripheral/src/ch32l103_lptim.o
 .text.LPTIM_GetCapture
                0x0000000000000000        0xa ./Peripheral/src/ch32l103_lptim.o
 .text.LPTIM_ITConfig
                0x0000000000000000       0x1a ./Peripheral/src/ch32l103_lptim.o
 .text.LPTIM_GetFlagStatus
                0x0000000000000000       0x10 ./Peripheral/src/ch32l103_lptim.o
 .text.LPTIM_ClearFlag
                0x0000000000000000       0x10 ./Peripheral/src/ch32l103_lptim.o
 .text.LPTIM_GetITStatus
                0x0000000000000000       0x18 ./Peripheral/src/ch32l103_lptim.o
 .text.LPTIM_ClearITPendingBit
                0x0000000000000000       0x18 ./Peripheral/src/ch32l103_lptim.o
 .debug_info    0x0000000000000000      0xe5e ./Peripheral/src/ch32l103_lptim.o
 .debug_abbrev  0x0000000000000000      0x361 ./Peripheral/src/ch32l103_lptim.o
 .debug_loc     0x0000000000000000      0x13a ./Peripheral/src/ch32l103_lptim.o
 .debug_aranges
                0x0000000000000000       0x78 ./Peripheral/src/ch32l103_lptim.o
 .debug_ranges  0x0000000000000000       0x68 ./Peripheral/src/ch32l103_lptim.o
 .debug_line    0x0000000000000000      0x75e ./Peripheral/src/ch32l103_lptim.o
 .debug_str     0x0000000000000000      0x953 ./Peripheral/src/ch32l103_lptim.o
 .comment       0x0000000000000000       0x34 ./Peripheral/src/ch32l103_lptim.o
 .debug_frame   0x0000000000000000      0x130 ./Peripheral/src/ch32l103_lptim.o
 .text          0x0000000000000000        0x0 ./Peripheral/src/ch32l103_misc.o
 .data          0x0000000000000000        0x0 ./Peripheral/src/ch32l103_misc.o
 .bss           0x0000000000000000        0x0 ./Peripheral/src/ch32l103_misc.o
 .text          0x0000000000000000        0x0 ./Peripheral/src/ch32l103_opa.o
 .data          0x0000000000000000        0x0 ./Peripheral/src/ch32l103_opa.o
 .bss           0x0000000000000000        0x0 ./Peripheral/src/ch32l103_opa.o
 .text.OPCM_Unlock
                0x0000000000000000       0x1a ./Peripheral/src/ch32l103_opa.o
 .text.OPCM_Lock
                0x0000000000000000        0xe ./Peripheral/src/ch32l103_opa.o
 .text.OPA_Init
                0x0000000000000000       0x8a ./Peripheral/src/ch32l103_opa.o
 .text.OPA_StructInit
                0x0000000000000000       0x36 ./Peripheral/src/ch32l103_opa.o
 .text.OPA_Cmd  0x0000000000000000       0x28 ./Peripheral/src/ch32l103_opa.o
 .text.OPA_LP_Cmd
                0x0000000000000000       0x20 ./Peripheral/src/ch32l103_opa.o
 .text.OPA_CMP_Init
                0x0000000000000000       0x72 ./Peripheral/src/ch32l103_opa.o
 .text.OPA_CMP_StructInit
                0x0000000000000000       0x12 ./Peripheral/src/ch32l103_opa.o
 .text.OPA_CMP_Cmd
                0x0000000000000000       0x2e ./Peripheral/src/ch32l103_opa.o
 .text.OPA_CMP_LP_Cmd
                0x0000000000000000       0x24 ./Peripheral/src/ch32l103_opa.o
 .text.OPA_CMP_WakeUp_ModeConfig
                0x0000000000000000       0x18 ./Peripheral/src/ch32l103_opa.o
 .text.OPA_GetFlagStatus
                0x0000000000000000        0xe ./Peripheral/src/ch32l103_opa.o
 .text.OPA_ClearFlag
                0x0000000000000000       0x10 ./Peripheral/src/ch32l103_opa.o
 .sbss.CTLR2_tmp
                0x0000000000000000        0x4 ./Peripheral/src/ch32l103_opa.o
 .debug_info    0x0000000000000000     0x10f2 ./Peripheral/src/ch32l103_opa.o
 .debug_abbrev  0x0000000000000000      0x2b9 ./Peripheral/src/ch32l103_opa.o
 .debug_loc     0x0000000000000000      0x23a ./Peripheral/src/ch32l103_opa.o
 .debug_aranges
                0x0000000000000000       0x80 ./Peripheral/src/ch32l103_opa.o
 .debug_ranges  0x0000000000000000       0x70 ./Peripheral/src/ch32l103_opa.o
 .debug_line    0x0000000000000000      0x9c3 ./Peripheral/src/ch32l103_opa.o
 .debug_str     0x0000000000000000      0xb21 ./Peripheral/src/ch32l103_opa.o
 .comment       0x0000000000000000       0x34 ./Peripheral/src/ch32l103_opa.o
 .debug_frame   0x0000000000000000       0xe0 ./Peripheral/src/ch32l103_opa.o
 .text          0x0000000000000000        0x0 ./Peripheral/src/ch32l103_pwr.o
 .data          0x0000000000000000        0x0 ./Peripheral/src/ch32l103_pwr.o
 .bss           0x0000000000000000        0x0 ./Peripheral/src/ch32l103_pwr.o
 .text.PWR_DeInit
                0x0000000000000000       0x2c ./Peripheral/src/ch32l103_pwr.o
 .text.PWR_BackupAccessCmd
                0x0000000000000000       0x16 ./Peripheral/src/ch32l103_pwr.o
 .text.PWR_PVDCmd
                0x0000000000000000       0x14 ./Peripheral/src/ch32l103_pwr.o
 .text.PWR_PVDLevelConfig
                0x0000000000000000       0x10 ./Peripheral/src/ch32l103_pwr.o
 .text.PWR_WakeUpPinCmd
                0x0000000000000000       0x16 ./Peripheral/src/ch32l103_pwr.o
 .text.PWR_EnterSTOPMode
                0x0000000000000000       0x96 ./Peripheral/src/ch32l103_pwr.o
 .text.PWR_EnterSTANDBYMode
                0x0000000000000000       0x38 ./Peripheral/src/ch32l103_pwr.o
 .text.PWR_GetFlagStatus
                0x0000000000000000        0xe ./Peripheral/src/ch32l103_pwr.o
 .text.PWR_ClearFlag
                0x0000000000000000        0xe ./Peripheral/src/ch32l103_pwr.o
 .text.PWR_EnterSTANDBYMode_RAM
                0x0000000000000000       0x3a ./Peripheral/src/ch32l103_pwr.o
 .text.PWR_EnterSTANDBYMode_RAM_LV
                0x0000000000000000       0x3a ./Peripheral/src/ch32l103_pwr.o
 .text.PWR_EnterSTANDBYMode_RAM_VBAT_EN
                0x0000000000000000       0x3a ./Peripheral/src/ch32l103_pwr.o
 .text.PWR_EnterSTANDBYMode_RAM_LV_VBAT_EN
                0x0000000000000000       0x3a ./Peripheral/src/ch32l103_pwr.o
 .text.PWR_EnterSTOPMode_RAM_LV
                0x0000000000000000       0x9e ./Peripheral/src/ch32l103_pwr.o
 .text.PWR_LDO_LP_Cmd
                0x0000000000000000       0x20 ./Peripheral/src/ch32l103_pwr.o
 .text.PWR_STOPMode_Auto_LDO_LP_Cmd
                0x0000000000000000       0x20 ./Peripheral/src/ch32l103_pwr.o
 .text.PWR_FLASH_LP_Cmd
                0x0000000000000000       0x22 ./Peripheral/src/ch32l103_pwr.o
 .debug_info    0x0000000000000000     0x10d0 ./Peripheral/src/ch32l103_pwr.o
 .debug_abbrev  0x0000000000000000      0x399 ./Peripheral/src/ch32l103_pwr.o
 .debug_loc     0x0000000000000000      0x2fa ./Peripheral/src/ch32l103_pwr.o
 .debug_aranges
                0x0000000000000000       0xa0 ./Peripheral/src/ch32l103_pwr.o
 .debug_ranges  0x0000000000000000      0x110 ./Peripheral/src/ch32l103_pwr.o
 .debug_line    0x0000000000000000      0xc67 ./Peripheral/src/ch32l103_pwr.o
 .debug_str     0x0000000000000000      0x88b ./Peripheral/src/ch32l103_pwr.o
 .comment       0x0000000000000000       0x34 ./Peripheral/src/ch32l103_pwr.o
 .debug_frame   0x0000000000000000      0x12c ./Peripheral/src/ch32l103_pwr.o
 .text          0x0000000000000000        0x0 ./Peripheral/src/ch32l103_rcc.o
 .data          0x0000000000000000        0x0 ./Peripheral/src/ch32l103_rcc.o
 .bss           0x0000000000000000        0x0 ./Peripheral/src/ch32l103_rcc.o
 .text.RCC_DeInit
                0x0000000000000000       0x42 ./Peripheral/src/ch32l103_rcc.o
 .text.RCC_HSEConfig
                0x0000000000000000       0x3c ./Peripheral/src/ch32l103_rcc.o
 .text.RCC_AdjustHSICalibrationValue
                0x0000000000000000       0x12 ./Peripheral/src/ch32l103_rcc.o
 .text.RCC_HSICmd
                0x0000000000000000       0x14 ./Peripheral/src/ch32l103_rcc.o
 .text.RCC_PLLConfig
                0x0000000000000000       0x16 ./Peripheral/src/ch32l103_rcc.o
 .text.RCC_PLLCmd
                0x0000000000000000       0x24 ./Peripheral/src/ch32l103_rcc.o
 .text.RCC_SYSCLKConfig
                0x0000000000000000        0xe ./Peripheral/src/ch32l103_rcc.o
 .text.RCC_GetSYSCLKSource
                0x0000000000000000        0xa ./Peripheral/src/ch32l103_rcc.o
 .text.RCC_HCLKConfig
                0x0000000000000000       0x10 ./Peripheral/src/ch32l103_rcc.o
 .text.RCC_PCLK1Config
                0x0000000000000000       0x10 ./Peripheral/src/ch32l103_rcc.o
 .text.RCC_PCLK2Config
                0x0000000000000000       0x16 ./Peripheral/src/ch32l103_rcc.o
 .text.RCC_ITConfig
                0x0000000000000000       0x16 ./Peripheral/src/ch32l103_rcc.o
 .text.RCC_USBCLKConfig
                0x0000000000000000       0x18 ./Peripheral/src/ch32l103_rcc.o
 .text.RCC_LSEConfig
                0x0000000000000000       0x28 ./Peripheral/src/ch32l103_rcc.o
 .text.RCC_LSICmd
                0x0000000000000000       0x14 ./Peripheral/src/ch32l103_rcc.o
 .text.RCC_RTCCLKConfig
                0x0000000000000000        0xc ./Peripheral/src/ch32l103_rcc.o
 .text.RCC_RTCCLKCmd
                0x0000000000000000       0x20 ./Peripheral/src/ch32l103_rcc.o
 .text.RCC_PB1PeriphResetCmd
                0x0000000000000000       0x1e ./Peripheral/src/ch32l103_rcc.o
 .text.RCC_BackupResetCmd
                0x0000000000000000       0x20 ./Peripheral/src/ch32l103_rcc.o
 .text.RCC_ClockSecuritySystemCmd
                0x0000000000000000       0x24 ./Peripheral/src/ch32l103_rcc.o
 .text.RCC_MCOConfig
                0x0000000000000000        0x8 ./Peripheral/src/ch32l103_rcc.o
 .text.RCC_GetFlagStatus
                0x0000000000000000       0x2e ./Peripheral/src/ch32l103_rcc.o
 .text.RCC_WaitForHSEStartUp
                0x0000000000000000       0x42 ./Peripheral/src/ch32l103_rcc.o
 .text.RCC_ClearFlag
                0x0000000000000000       0x10 ./Peripheral/src/ch32l103_rcc.o
 .text.RCC_GetITStatus
                0x0000000000000000        0xe ./Peripheral/src/ch32l103_rcc.o
 .text.RCC_ClearITPendingBit
                0x0000000000000000        0x8 ./Peripheral/src/ch32l103_rcc.o
 .text.RCC_ADCCLKDutyCycleConfig
                0x0000000000000000       0x18 ./Peripheral/src/ch32l103_rcc.o
 .text.RCC_HSE_LP_Cmd
                0x0000000000000000       0x24 ./Peripheral/src/ch32l103_rcc.o
 .text.RCC_HSI_LP_Cmd
                0x0000000000000000       0x14 ./Peripheral/src/ch32l103_rcc.o
 .text          0x0000000000000000        0x0 ./Peripheral/src/ch32l103_rtc.o
 .data          0x0000000000000000        0x0 ./Peripheral/src/ch32l103_rtc.o
 .bss           0x0000000000000000        0x0 ./Peripheral/src/ch32l103_rtc.o
 .text.RTC_ITConfig
                0x0000000000000000       0x1a ./Peripheral/src/ch32l103_rtc.o
 .text.RTC_EnterConfigMode
                0x0000000000000000       0x12 ./Peripheral/src/ch32l103_rtc.o
 .text.RTC_ExitConfigMode
                0x0000000000000000       0x18 ./Peripheral/src/ch32l103_rtc.o
 .text.RTC_GetCounter
                0x0000000000000000       0x36 ./Peripheral/src/ch32l103_rtc.o
 .text.RTC_SetCounter
                0x0000000000000000       0x3c ./Peripheral/src/ch32l103_rtc.o
 .text.RTC_SetPrescaler
                0x0000000000000000       0x3e ./Peripheral/src/ch32l103_rtc.o
 .text.RTC_SetAlarm
                0x0000000000000000       0x3c ./Peripheral/src/ch32l103_rtc.o
 .text.RTC_GetDivider
                0x0000000000000000       0x18 ./Peripheral/src/ch32l103_rtc.o
 .text.RTC_WaitForLastTask
                0x0000000000000000       0x10 ./Peripheral/src/ch32l103_rtc.o
 .text.RTC_WaitForSynchro
                0x0000000000000000       0x24 ./Peripheral/src/ch32l103_rtc.o
 .text.RTC_GetFlagStatus
                0x0000000000000000       0x12 ./Peripheral/src/ch32l103_rtc.o
 .text.RTC_ClearFlag
                0x0000000000000000       0x14 ./Peripheral/src/ch32l103_rtc.o
 .text.RTC_GetITStatus
                0x0000000000000000       0x20 ./Peripheral/src/ch32l103_rtc.o
 .text.RTC_ClearITPendingBit
                0x0000000000000000       0x18 ./Peripheral/src/ch32l103_rtc.o
 .debug_info    0x0000000000000000      0xd7f ./Peripheral/src/ch32l103_rtc.o
 .debug_abbrev  0x0000000000000000      0x2c0 ./Peripheral/src/ch32l103_rtc.o
 .debug_loc     0x0000000000000000      0x272 ./Peripheral/src/ch32l103_rtc.o
 .debug_aranges
                0x0000000000000000       0x80 ./Peripheral/src/ch32l103_rtc.o
 .debug_ranges  0x0000000000000000       0x70 ./Peripheral/src/ch32l103_rtc.o
 .debug_line    0x0000000000000000      0x751 ./Peripheral/src/ch32l103_rtc.o
 .debug_str     0x0000000000000000      0x7e4 ./Peripheral/src/ch32l103_rtc.o
 .comment       0x0000000000000000       0x34 ./Peripheral/src/ch32l103_rtc.o
 .debug_frame   0x0000000000000000      0x12c ./Peripheral/src/ch32l103_rtc.o
 .text          0x0000000000000000        0x0 ./Peripheral/src/ch32l103_spi.o
 .data          0x0000000000000000        0x0 ./Peripheral/src/ch32l103_spi.o
 .bss           0x0000000000000000        0x0 ./Peripheral/src/ch32l103_spi.o
 .text.SPI_I2S_DeInit
                0x0000000000000000       0x56 ./Peripheral/src/ch32l103_spi.o
 .text.SPI_StructInit
                0x0000000000000000       0x22 ./Peripheral/src/ch32l103_spi.o
 .text.SPI_I2S_ITConfig
                0x0000000000000000       0x1e ./Peripheral/src/ch32l103_spi.o
 .text.SPI_I2S_DMACmd
                0x0000000000000000       0x12 ./Peripheral/src/ch32l103_spi.o
 .text.SPI_NSSInternalSoftwareConfig
                0x0000000000000000       0x24 ./Peripheral/src/ch32l103_spi.o
 .text.SPI_SSOutputCmd
                0x0000000000000000       0x18 ./Peripheral/src/ch32l103_spi.o
 .text.SPI_DataSizeConfig
                0x0000000000000000       0x14 ./Peripheral/src/ch32l103_spi.o
 .text.SPI_TransmitCRC
                0x0000000000000000        0xa ./Peripheral/src/ch32l103_spi.o
 .text.SPI_CalculateCRC
                0x0000000000000000       0x16 ./Peripheral/src/ch32l103_spi.o
 .text.SPI_GetCRC
                0x0000000000000000       0x12 ./Peripheral/src/ch32l103_spi.o
 .text.SPI_GetCRCPolynomial
                0x0000000000000000        0x4 ./Peripheral/src/ch32l103_spi.o
 .text.SPI_BiDirectionalLineConfig
                0x0000000000000000       0x1a ./Peripheral/src/ch32l103_spi.o
 .text.SPI_I2S_ClearFlag
                0x0000000000000000        0xc ./Peripheral/src/ch32l103_spi.o
 .text.SPI_I2S_GetITStatus
                0x0000000000000000       0x28 ./Peripheral/src/ch32l103_spi.o
 .text.SPI_I2S_ClearITPendingBit
                0x0000000000000000       0x14 ./Peripheral/src/ch32l103_spi.o
 .text.SPI_HighSpeedRead_Cmd
                0x0000000000000000       0x18 ./Peripheral/src/ch32l103_spi.o
 .text          0x0000000000000000        0x0 ./Peripheral/src/ch32l103_tim.o
 .data          0x0000000000000000        0x0 ./Peripheral/src/ch32l103_tim.o
 .bss           0x0000000000000000        0x0 ./Peripheral/src/ch32l103_tim.o
 .text.TI1_Config
                0x0000000000000000       0x62 ./Peripheral/src/ch32l103_tim.o
 .text.TI2_Config
                0x0000000000000000       0x7a ./Peripheral/src/ch32l103_tim.o
 .text.TIM_DeInit
                0x0000000000000000       0x94 ./Peripheral/src/ch32l103_tim.o
 .text.TIM_OC2Init
                0x0000000000000000       0xa8 ./Peripheral/src/ch32l103_tim.o
 .text.TIM_OC3Init
                0x0000000000000000       0xa6 ./Peripheral/src/ch32l103_tim.o
 .text.TIM_BDTRConfig
                0x0000000000000000       0x20 ./Peripheral/src/ch32l103_tim.o
 .text.TIM_TimeBaseStructInit
                0x0000000000000000       0x14 ./Peripheral/src/ch32l103_tim.o
 .text.TIM_OCStructInit
                0x0000000000000000       0x16 ./Peripheral/src/ch32l103_tim.o
 .text.TIM_ICStructInit
                0x0000000000000000       0x16 ./Peripheral/src/ch32l103_tim.o
 .text.TIM_BDTRStructInit
                0x0000000000000000       0x1e ./Peripheral/src/ch32l103_tim.o
 .text.TIM_GenerateEvent
                0x0000000000000000        0x4 ./Peripheral/src/ch32l103_tim.o
 .text.TIM_DMAConfig
                0x0000000000000000        0x8 ./Peripheral/src/ch32l103_tim.o
 .text.TIM_DMACmd
                0x0000000000000000       0x18 ./Peripheral/src/ch32l103_tim.o
 .text.TIM_InternalClockConfig
                0x0000000000000000       0x10 ./Peripheral/src/ch32l103_tim.o
 .text.TIM_ITRxExternalClockConfig
                0x0000000000000000       0x18 ./Peripheral/src/ch32l103_tim.o
 .text.TIM_TIxExternalClockConfig
                0x0000000000000000       0x48 ./Peripheral/src/ch32l103_tim.o
 .text.TIM_ETRConfig
                0x0000000000000000       0x16 ./Peripheral/src/ch32l103_tim.o
 .text.TIM_ETRClockMode1Config
                0x0000000000000000       0x2a ./Peripheral/src/ch32l103_tim.o
 .text.TIM_ETRClockMode2Config
                0x0000000000000000       0x22 ./Peripheral/src/ch32l103_tim.o
 .text.TIM_PrescalerConfig
                0x0000000000000000        0x6 ./Peripheral/src/ch32l103_tim.o
 .text.TIM_CounterModeConfig
                0x0000000000000000       0x10 ./Peripheral/src/ch32l103_tim.o
 .text.TIM_SelectInputTrigger
                0x0000000000000000       0x10 ./Peripheral/src/ch32l103_tim.o
 .text.TIM_EncoderInterfaceConfig
                0x0000000000000000       0x3c ./Peripheral/src/ch32l103_tim.o
 .text.TIM_ForcedOC1Config
                0x0000000000000000       0x10 ./Peripheral/src/ch32l103_tim.o
 .text.TIM_ForcedOC2Config
                0x0000000000000000       0x14 ./Peripheral/src/ch32l103_tim.o
 .text.TIM_ForcedOC3Config
                0x0000000000000000       0x10 ./Peripheral/src/ch32l103_tim.o
 .text.TIM_ForcedOC4Config
                0x0000000000000000       0x14 ./Peripheral/src/ch32l103_tim.o
 .text.TIM_SelectCOM
                0x0000000000000000       0x18 ./Peripheral/src/ch32l103_tim.o
 .text.TIM_SelectCCDMA
                0x0000000000000000       0x18 ./Peripheral/src/ch32l103_tim.o
 .text.TIM_CCPreloadControl
                0x0000000000000000       0x18 ./Peripheral/src/ch32l103_tim.o
 .text.TIM_OC2PreloadConfig
                0x0000000000000000       0x16 ./Peripheral/src/ch32l103_tim.o
 .text.TIM_OC3PreloadConfig
                0x0000000000000000        0xe ./Peripheral/src/ch32l103_tim.o
 .text.TIM_OC1FastConfig
                0x0000000000000000        0xe ./Peripheral/src/ch32l103_tim.o
 .text.TIM_OC2FastConfig
                0x0000000000000000       0x16 ./Peripheral/src/ch32l103_tim.o
 .text.TIM_OC3FastConfig
                0x0000000000000000        0xe ./Peripheral/src/ch32l103_tim.o
 .text.TIM_OC4FastConfig
                0x0000000000000000       0x16 ./Peripheral/src/ch32l103_tim.o
 .text.TIM_ClearOC1Ref
                0x0000000000000000       0x10 ./Peripheral/src/ch32l103_tim.o
 .text.TIM_ClearOC2Ref
                0x0000000000000000       0x12 ./Peripheral/src/ch32l103_tim.o
 .text.TIM_ClearOC3Ref
                0x0000000000000000       0x10 ./Peripheral/src/ch32l103_tim.o
 .text.TIM_ClearOC4Ref
                0x0000000000000000       0x12 ./Peripheral/src/ch32l103_tim.o
 .text.TIM_OC1PolarityConfig
                0x0000000000000000        0xe ./Peripheral/src/ch32l103_tim.o
 .text.TIM_OC1NPolarityConfig
                0x0000000000000000        0xe ./Peripheral/src/ch32l103_tim.o
 .text.TIM_OC2PolarityConfig
                0x0000000000000000       0x16 ./Peripheral/src/ch32l103_tim.o
 .text.TIM_OC2NPolarityConfig
                0x0000000000000000       0x16 ./Peripheral/src/ch32l103_tim.o
 .text.TIM_OC3PolarityConfig
                0x0000000000000000       0x16 ./Peripheral/src/ch32l103_tim.o
 .text.TIM_OC3NPolarityConfig
                0x0000000000000000       0x16 ./Peripheral/src/ch32l103_tim.o
 .text.TIM_OC4PolarityConfig
                0x0000000000000000       0x14 ./Peripheral/src/ch32l103_tim.o
 .text.TIM_CCxCmd
                0x0000000000000000       0x20 ./Peripheral/src/ch32l103_tim.o
 .text.TIM_CCxNCmd
                0x0000000000000000       0x20 ./Peripheral/src/ch32l103_tim.o
 .text.TIM_SelectOCxM
                0x0000000000000000       0x4c ./Peripheral/src/ch32l103_tim.o
 .text.TIM_UpdateDisableConfig
                0x0000000000000000       0x18 ./Peripheral/src/ch32l103_tim.o
 .text.TIM_UpdateRequestConfig
                0x0000000000000000       0x18 ./Peripheral/src/ch32l103_tim.o
 .text.TIM_SelectHallSensor
                0x0000000000000000       0x1a ./Peripheral/src/ch32l103_tim.o
 .text.TIM_SelectOnePulseMode
                0x0000000000000000       0x16 ./Peripheral/src/ch32l103_tim.o
 .text.TIM_SelectOutputTrigger
                0x0000000000000000       0x18 ./Peripheral/src/ch32l103_tim.o
 .text.TIM_SelectSlaveMode
                0x0000000000000000       0x16 ./Peripheral/src/ch32l103_tim.o
 .text.TIM_SelectMasterSlaveMode
                0x0000000000000000       0x18 ./Peripheral/src/ch32l103_tim.o
 .text.TIM_SetCounter
                0x0000000000000000       0x18 ./Peripheral/src/ch32l103_tim.o
 .text.TIM_SetAutoreload
                0x0000000000000000       0x18 ./Peripheral/src/ch32l103_tim.o
 .text.TIM_SetCompare1
                0x0000000000000000       0x16 ./Peripheral/src/ch32l103_tim.o
 .text.TIM_SetCompare2
                0x0000000000000000       0x16 ./Peripheral/src/ch32l103_tim.o
 .text.TIM_SetCompare3
                0x0000000000000000       0x16 ./Peripheral/src/ch32l103_tim.o
 .text.TIM_SetIC1Prescaler
                0x0000000000000000       0x16 ./Peripheral/src/ch32l103_tim.o
 .text.TIM_SetIC2Prescaler
                0x0000000000000000       0x1a ./Peripheral/src/ch32l103_tim.o
 .text.TIM_PWMIConfig
                0x0000000000000000       0x92 ./Peripheral/src/ch32l103_tim.o
 .text.TIM_SetIC3Prescaler
                0x0000000000000000       0x16 ./Peripheral/src/ch32l103_tim.o
 .text.TIM_SetIC4Prescaler
                0x0000000000000000       0x1a ./Peripheral/src/ch32l103_tim.o
 .text.TIM_ICInit
                0x0000000000000000      0x172 ./Peripheral/src/ch32l103_tim.o
 .text.TIM_SetClockDivision
                0x0000000000000000       0x18 ./Peripheral/src/ch32l103_tim.o
 .text.TIM_GetCapture1
                0x0000000000000000        0x4 ./Peripheral/src/ch32l103_tim.o
 .text.TIM_GetCapture2
                0x0000000000000000        0x4 ./Peripheral/src/ch32l103_tim.o
 .text.TIM_GetCapture3
                0x0000000000000000        0x4 ./Peripheral/src/ch32l103_tim.o
 .text.TIM_GetCapture4
                0x0000000000000000        0x4 ./Peripheral/src/ch32l103_tim.o
 .text.TIM_GetCounter
                0x0000000000000000       0x18 ./Peripheral/src/ch32l103_tim.o
 .text.TIM_GetPrescaler
                0x0000000000000000        0x4 ./Peripheral/src/ch32l103_tim.o
 .text.TIM_GetFlagStatus
                0x0000000000000000        0xa ./Peripheral/src/ch32l103_tim.o
 .text.TIM_ClearFlag
                0x0000000000000000        0xc ./Peripheral/src/ch32l103_tim.o
 .text.TIM_CaptureLevelIndicate_Cmd
                0x0000000000000000       0x12 ./Peripheral/src/ch32l103_tim.o
 .text.TIM_CaptureModeConfig
                0x0000000000000000       0x1a ./Peripheral/src/ch32l103_tim.o
 .text          0x0000000000000000        0x0 ./Peripheral/src/ch32l103_usart.o
 .data          0x0000000000000000        0x0 ./Peripheral/src/ch32l103_usart.o
 .bss           0x0000000000000000        0x0 ./Peripheral/src/ch32l103_usart.o
 .text.USART_DeInit
                0x0000000000000000       0x9e ./Peripheral/src/ch32l103_usart.o
 .text.USART_StructInit
                0x0000000000000000       0x18 ./Peripheral/src/ch32l103_usart.o
 .text.USART_ClockInit
                0x0000000000000000       0x1e ./Peripheral/src/ch32l103_usart.o
 .text.USART_ClockStructInit
                0x0000000000000000       0x12 ./Peripheral/src/ch32l103_usart.o
 .text.USART_DMACmd
                0x0000000000000000       0x12 ./Peripheral/src/ch32l103_usart.o
 .text.USART_SetAddress
                0x0000000000000000       0x16 ./Peripheral/src/ch32l103_usart.o
 .text.USART_WakeUpConfig
                0x0000000000000000       0x14 ./Peripheral/src/ch32l103_usart.o
 .text.USART_ReceiverWakeUpCmd
                0x0000000000000000       0x18 ./Peripheral/src/ch32l103_usart.o
 .text.USART_LINBreakDetectLengthConfig
                0x0000000000000000       0x18 ./Peripheral/src/ch32l103_usart.o
 .text.USART_LINCmd
                0x0000000000000000       0x16 ./Peripheral/src/ch32l103_usart.o
 .text.USART_SendBreak
                0x0000000000000000        0xa ./Peripheral/src/ch32l103_usart.o
 .text.USART_SetGuardTime
                0x0000000000000000       0x12 ./Peripheral/src/ch32l103_usart.o
 .text.USART_SetPrescaler
                0x0000000000000000       0x18 ./Peripheral/src/ch32l103_usart.o
 .text.USART_SmartCardCmd
                0x0000000000000000       0x1a ./Peripheral/src/ch32l103_usart.o
 .text.USART_SmartCardNACKCmd
                0x0000000000000000       0x18 ./Peripheral/src/ch32l103_usart.o
 .text.USART_HalfDuplexCmd
                0x0000000000000000       0x18 ./Peripheral/src/ch32l103_usart.o
 .text.USART_OverSampling8Cmd
                0x0000000000000000       0x12 ./Peripheral/src/ch32l103_usart.o
 .text.USART_OneBitMethodCmd
                0x0000000000000000       0x1e ./Peripheral/src/ch32l103_usart.o
 .text.USART_IrDAConfig
                0x0000000000000000       0x16 ./Peripheral/src/ch32l103_usart.o
 .text.USART_IrDACmd
                0x0000000000000000       0x18 ./Peripheral/src/ch32l103_usart.o
 .text.USART_ClearFlag
                0x0000000000000000        0xc ./Peripheral/src/ch32l103_usart.o
 .text.USART_ClearITPendingBit
                0x0000000000000000       0x14 ./Peripheral/src/ch32l103_usart.o
 .text          0x0000000000000000        0x0 ./Peripheral/src/ch32l103_wwdg.o
 .data          0x0000000000000000        0x0 ./Peripheral/src/ch32l103_wwdg.o
 .bss           0x0000000000000000        0x0 ./Peripheral/src/ch32l103_wwdg.o
 .text.WWDG_DeInit
                0x0000000000000000       0x2e ./Peripheral/src/ch32l103_wwdg.o
 .text.WWDG_SetPrescaler
                0x0000000000000000       0x14 ./Peripheral/src/ch32l103_wwdg.o
 .text.WWDG_SetWindowValue
                0x0000000000000000       0x26 ./Peripheral/src/ch32l103_wwdg.o
 .text.WWDG_EnableIT
                0x0000000000000000       0x12 ./Peripheral/src/ch32l103_wwdg.o
 .text.WWDG_SetCounter
                0x0000000000000000        0xe ./Peripheral/src/ch32l103_wwdg.o
 .text.WWDG_Enable
                0x0000000000000000        0xe ./Peripheral/src/ch32l103_wwdg.o
 .text.WWDG_GetFlagStatus
                0x0000000000000000        0xa ./Peripheral/src/ch32l103_wwdg.o
 .text.WWDG_ClearFlag
                0x0000000000000000        0xa ./Peripheral/src/ch32l103_wwdg.o
 .debug_info    0x0000000000000000      0xb6f ./Peripheral/src/ch32l103_wwdg.o
 .debug_abbrev  0x0000000000000000      0x29d ./Peripheral/src/ch32l103_wwdg.o
 .debug_loc     0x0000000000000000       0xae ./Peripheral/src/ch32l103_wwdg.o
 .debug_aranges
                0x0000000000000000       0x58 ./Peripheral/src/ch32l103_wwdg.o
 .debug_ranges  0x0000000000000000       0x48 ./Peripheral/src/ch32l103_wwdg.o
 .debug_line    0x0000000000000000      0x443 ./Peripheral/src/ch32l103_wwdg.o
 .debug_str     0x0000000000000000      0x6bd ./Peripheral/src/ch32l103_wwdg.o
 .comment       0x0000000000000000       0x34 ./Peripheral/src/ch32l103_wwdg.o
 .debug_frame   0x0000000000000000       0xa4 ./Peripheral/src/ch32l103_wwdg.o
 .text          0x0000000000000000        0x0 ./Hardware/src/adc.o
 .data          0x0000000000000000        0x0 ./Hardware/src/adc.o
 .bss           0x0000000000000000        0x0 ./Hardware/src/adc.o
 .text.Get_ConversionVal1
                0x0000000000000000       0x2e ./Hardware/src/adc.o
 .text          0x0000000000000000        0x0 ./Hardware/src/flash.o
 .data          0x0000000000000000        0x0 ./Hardware/src/flash.o
 .bss           0x0000000000000000        0x0 ./Hardware/src/flash.o
 .text.SPI_Flash_ReadSR
                0x0000000000000000       0x4e ./Hardware/src/flash.o
 .text.SPI_FLASH_Write_SR
                0x0000000000000000       0x4a ./Hardware/src/flash.o
 .text.SPI_Flash_Wait_Busy
                0x0000000000000000       0x1c ./Hardware/src/flash.o
 .text.SPI_FLASH_Write_Enable
                0x0000000000000000       0x3e ./Hardware/src/flash.o
 .text.SPI_FLASH_Write_Disable
                0x0000000000000000       0x3e ./Hardware/src/flash.o
 .text.SPI_Flash_ReadID
                0x0000000000000000       0x86 ./Hardware/src/flash.o
 .text.SPI_Flash_Erase_Sector
                0x0000000000000000       0x86 ./Hardware/src/flash.o
 .text.SPI_Flash_Write_Page
                0x0000000000000000       0xa2 ./Hardware/src/flash.o
 .text.SPI_Flash_Write_NoCheck
                0x0000000000000000       0x60 ./Hardware/src/flash.o
 .text.SPI_Flash_Write
                0x0000000000000000       0xd8 ./Hardware/src/flash.o
 .text.SPI_Flash_Erase_Chip
                0x0000000000000000       0x58 ./Hardware/src/flash.o
 .text.SPI_Flash_PowerDown
                0x0000000000000000       0x4a ./Hardware/src/flash.o
 .text.SPI_Flash_WAKEUP
                0x0000000000000000       0x4a ./Hardware/src/flash.o
 .text.SPI_Flash_TEST
                0x0000000000000000      0x166 ./Hardware/src/flash.o
 .rodata.SPI_Flash_TEST
                0x0000000000000000       0x14 ./Hardware/src/flash.o
 .rodata        0x0000000000000000       0x64 ./Hardware/src/flash.o
 .bss.SPI_FLASH_BUF
                0x0000000000000000     0x1000 ./Hardware/src/flash.o
 .rodata.SPI_Flash_TEST.str1.4
                0x0000000000000000       0xe2 ./Hardware/src/flash.o
 .text          0x0000000000000000        0x0 ./Hardware/src/gpio.o
 .data          0x0000000000000000        0x0 ./Hardware/src/gpio.o
 .bss           0x0000000000000000        0x0 ./Hardware/src/gpio.o
 .text.G_FFMOS_CON_Init
                0x0000000000000000       0x7c ./Hardware/src/gpio.o
 .text.BEEP_Init
                0x0000000000000000       0x3e ./Hardware/src/gpio.o
 .text.EnPowerSupply_Init
                0x0000000000000000       0x4e ./Hardware/src/gpio.o
 .text          0x0000000000000000        0x0 ./Hardware/src/pwm.o
 .data          0x0000000000000000        0x0 ./Hardware/src/pwm.o
 .bss           0x0000000000000000        0x0 ./Hardware/src/pwm.o
 .text          0x0000000000000000        0x0 ./Hardware/src/rs485.o
 .data          0x0000000000000000        0x0 ./Hardware/src/rs485.o
 .bss           0x0000000000000000        0x0 ./Hardware/src/rs485.o
 .text.USARTx_SendByte
                0x0000000000000000       0x2a ./Hardware/src/rs485.o
 .text.USARTx_ITSendstr
                0x0000000000000000       0x26 ./Hardware/src/rs485.o
 .text          0x0000000000000000        0x0 ./Hardware/src/tim.o
 .data          0x0000000000000000        0x0 ./Hardware/src/tim.o
 .bss           0x0000000000000000        0x0 ./Hardware/src/tim.o
 .text.TIM3_Int_Init
                0x0000000000000000       0x78 ./Hardware/src/tim.o
 .text.TIM3_Init
                0x0000000000000000       0x3c ./Hardware/src/tim.o
 .text.Systick_Init
                0x0000000000000000       0x3e ./Hardware/src/tim.o
 .text.TIM1_Int_Init
                0x0000000000000000       0x7c ./Hardware/src/tim.o
 .text.TIM1_Init
                0x0000000000000000       0x36 ./Hardware/src/tim.o
 .text          0x0000000000000000        0x0 ./Drivers/TimeSliceOffset/timeSliceOffset.o
 .data          0x0000000000000000        0x0 ./Drivers/TimeSliceOffset/timeSliceOffset.o
 .bss           0x0000000000000000        0x0 ./Drivers/TimeSliceOffset/timeSliceOffset.o
 .text          0x0000000000000000        0x0 ./Drivers/RingQueue/ring_queue.o
 .data          0x0000000000000000        0x0 ./Drivers/RingQueue/ring_queue.o
 .bss           0x0000000000000000        0x0 ./Drivers/RingQueue/ring_queue.o
 .text.ShowRingQueue
                0x0000000000000000        0xc ./Drivers/RingQueue/ring_queue.o
 .text.OutRingQueue
                0x0000000000000000       0x26 ./Drivers/RingQueue/ring_queue.o
 .text.RingQueueLength
                0x0000000000000000       0x10 ./Drivers/RingQueue/ring_queue.o
 .text          0x0000000000000000        0x0 ./Debug/debug.o
 .data          0x0000000000000000        0x0 ./Debug/debug.o
 .bss           0x0000000000000000        0x0 ./Debug/debug.o
 .text.Delay_Us
                0x0000000000000000       0x42 ./Debug/debug.o
 .text.Delay_Ms
                0x0000000000000000       0x3a ./Debug/debug.o
 .text          0x0000000000000000        0x0 ./Core/core_riscv.o
 .data          0x0000000000000000        0x0 ./Core/core_riscv.o
 .bss           0x0000000000000000        0x0 ./Core/core_riscv.o
 .text.__get_MSTATUS
                0x0000000000000000        0x6 ./Core/core_riscv.o
 .text.__set_MSTATUS
                0x0000000000000000        0x6 ./Core/core_riscv.o
 .text.__get_MISA
                0x0000000000000000        0x6 ./Core/core_riscv.o
 .text.__set_MISA
                0x0000000000000000        0x6 ./Core/core_riscv.o
 .text.__get_MTVEC
                0x0000000000000000        0x6 ./Core/core_riscv.o
 .text.__set_MTVEC
                0x0000000000000000        0x6 ./Core/core_riscv.o
 .text.__get_MSCRATCH
                0x0000000000000000        0x6 ./Core/core_riscv.o
 .text.__set_MSCRATCH
                0x0000000000000000        0x6 ./Core/core_riscv.o
 .text.__get_MEPC
                0x0000000000000000        0x6 ./Core/core_riscv.o
 .text.__set_MEPC
                0x0000000000000000        0x6 ./Core/core_riscv.o
 .text.__get_MCAUSE
                0x0000000000000000        0x6 ./Core/core_riscv.o
 .text.__set_MCAUSE
                0x0000000000000000        0x6 ./Core/core_riscv.o
 .text.__get_MTVAL
                0x0000000000000000        0x6 ./Core/core_riscv.o
 .text.__set_MTVAL
                0x0000000000000000        0x6 ./Core/core_riscv.o
 .text.__get_MVENDORID
                0x0000000000000000        0x6 ./Core/core_riscv.o
 .text.__get_MARCHID
                0x0000000000000000        0x6 ./Core/core_riscv.o
 .text.__get_MIMPID
                0x0000000000000000        0x6 ./Core/core_riscv.o
 .text.__get_MHARTID
                0x0000000000000000        0x6 ./Core/core_riscv.o
 .text.__get_SP
                0x0000000000000000        0x4 ./Core/core_riscv.o
 .debug_info    0x0000000000000000      0x376 ./Core/core_riscv.o
 .debug_abbrev  0x0000000000000000       0xe0 ./Core/core_riscv.o
 .debug_aranges
                0x0000000000000000       0xb0 ./Core/core_riscv.o
 .debug_ranges  0x0000000000000000       0xa0 ./Core/core_riscv.o
 .debug_line    0x0000000000000000      0x440 ./Core/core_riscv.o
 .debug_str     0x0000000000000000      0x274 ./Core/core_riscv.o
 .comment       0x0000000000000000       0x34 ./Core/core_riscv.o
 .debug_frame   0x0000000000000000      0x140 ./Core/core_riscv.o
 .text          0x0000000000000000        0x0 ./App/src/collect_Conversion.o
 .data          0x0000000000000000        0x0 ./App/src/collect_Conversion.o
 .bss           0x0000000000000000        0x0 ./App/src/collect_Conversion.o
 .text.get_aftercalculationAdc1
                0x0000000000000000       0x18 ./App/src/collect_Conversion.o
 .text.get_SYS_VOLT_IN
                0x0000000000000000       0x32 ./App/src/collect_Conversion.o
 .text.get_PV2_VOLT_IN
                0x0000000000000000        0x6 ./App/src/collect_Conversion.o
 .sdata2.P_CHG_CURR
                0x0000000000000000        0x4 ./App/src/collect_Conversion.o
 .sdata2.P_DSG_CURR
                0x0000000000000000        0x4 ./App/src/collect_Conversion.o
 .sdata2.P_PV1_VOLT_IN
                0x0000000000000000        0x4 ./App/src/collect_Conversion.o
 .sdata2.P_PV2_VOLT_IN
                0x0000000000000000        0x4 ./App/src/collect_Conversion.o
 .sdata2.P_PV_VOLT_IN1
                0x0000000000000000        0x4 ./App/src/collect_Conversion.o
 .sdata2.P_PV_VOLT_OUT
                0x0000000000000000        0x4 ./App/src/collect_Conversion.o
 .text          0x0000000000000000        0x0 ./App/src/inflash.o
 .data          0x0000000000000000        0x0 ./App/src/inflash.o
 .bss           0x0000000000000000        0x0 ./App/src/inflash.o
 .text.save_config_info
                0x0000000000000000       0x1e ./App/src/inflash.o
 .text.read_config_info1
                0x0000000000000000       0x8e ./App/src/inflash.o
 .text          0x0000000000000000        0x0 ./App/src/mppt_control.o
 .data          0x0000000000000000        0x0 ./App/src/mppt_control.o
 .bss           0x0000000000000000        0x0 ./App/src/mppt_control.o
 .text.Get_OutputPower
                0x0000000000000000       0xaa ./App/src/mppt_control.o
 .text.mppt_readJust
                0x0000000000000000      0x10e ./App/src/mppt_control.o
 .text.printf_data
                0x0000000000000000       0x24 ./App/src/mppt_control.o
 .text.mppt_constantVoltage
                0x0000000000000000       0x8e ./App/src/mppt_control.o
 .text.mppt_constantVoltageB
                0x0000000000000000       0x8a ./App/src/mppt_control.o
 .text.mppt_constantVoltageO
                0x0000000000000000       0x8a ./App/src/mppt_control.o
 .text.mppt_constantCurrentO
                0x0000000000000000       0x8a ./App/src/mppt_control.o
 .text.NoBatteryCharge
                0x0000000000000000       0x20 ./App/src/mppt_control.o
 .text.MpptContorl
                0x0000000000000000      0x132 ./App/src/mppt_control.o
 .text.MpptMode
                0x0000000000000000      0x3a2 ./App/src/mppt_control.o
 .text.findMiNDutyRatio
                0x0000000000000000       0x6c ./App/src/mppt_control.o
 .rodata.Get_OutputPower.cst4
                0x0000000000000000        0x8 ./App/src/mppt_control.o
 .rodata.Get_OutputPower.str1.4
                0x0000000000000000       0x35 ./App/src/mppt_control.o
 .rodata.MpptContorl.cst4
                0x0000000000000000        0x4 ./App/src/mppt_control.o
 .rodata.MpptMode.cst4
                0x0000000000000000        0x8 ./App/src/mppt_control.o
 .rodata.MpptMode.cst8
                0x0000000000000000       0x18 ./App/src/mppt_control.o
 .rodata.MpptMode.str1.4
                0x0000000000000000       0x1c ./App/src/mppt_control.o
 .rodata.NoBatteryCharge.cst4
                0x0000000000000000        0x4 ./App/src/mppt_control.o
 .rodata.findMiNDutyRatio.str1.4
                0x0000000000000000       0x1a ./App/src/mppt_control.o
 .rodata.mppt_constantCurrentO.cst4
                0x0000000000000000        0x4 ./App/src/mppt_control.o
 .rodata.mppt_constantVoltage.cst4
                0x0000000000000000        0x4 ./App/src/mppt_control.o
 .rodata.mppt_readJust.str1.4
                0x0000000000000000       0x6b ./App/src/mppt_control.o
 .sbss.ConstantCurrentV.5848
                0x0000000000000000        0x4 ./App/src/mppt_control.o
 .sbss.ConstantVoltageChargeV.5826
                0x0000000000000000        0x4 ./App/src/mppt_control.o
 .sbss.ConstantVoltageV.5849
                0x0000000000000000        0x4 ./App/src/mppt_control.o
 .sbss.FloatChargeV.5831
                0x0000000000000000        0x4 ./App/src/mppt_control.o
 .sbss.FloatI.5850
                0x0000000000000000        0x4 ./App/src/mppt_control.o
 .sbss.OutputPower.5768
                0x0000000000000000        0x4 ./App/src/mppt_control.o
 .sbss.StopSolarOpenCircuitV.5851
                0x0000000000000000        0x4 ./App/src/mppt_control.o
 .sbss.TrickleChargeC.5818
                0x0000000000000000        0x4 ./App/src/mppt_control.o
 .sbss.V_out.5769
                0x0000000000000000        0x4 ./App/src/mppt_control.o
 .sbss.last_OutputPower.5777
                0x0000000000000000        0x4 ./App/src/mppt_control.o
 .sdata.last_duty_ratio.5776
                0x0000000000000000        0x4 ./App/src/mppt_control.o
 .sdata.num.5856
                0x0000000000000000        0x1 ./App/src/mppt_control.o
 .sdata.onlyOnce.5819
                0x0000000000000000        0x1 ./App/src/mppt_control.o
 .sdata.onlyOnce.5827
                0x0000000000000000        0x1 ./App/src/mppt_control.o
 .sdata.onlyOnce.5832
                0x0000000000000000        0x1 ./App/src/mppt_control.o
 .sdata.only_once.5852
                0x0000000000000000        0x1 ./App/src/mppt_control.o
 .sdata.step_pwm.5779
                0x0000000000000000        0x4 ./App/src/mppt_control.o
 .sdata2.step1_pwm
                0x0000000000000000        0x4 ./App/src/mppt_control.o
 .sdata2.step2_pwm
                0x0000000000000000        0x4 ./App/src/mppt_control.o
 .text          0x0000000000000000        0x0 ./App/src/sl_protocol.o
 .data          0x0000000000000000        0x0 ./App/src/sl_protocol.o
 .bss           0x0000000000000000        0x0 ./App/src/sl_protocol.o
 .text.SL_ReadRegisterMPPTMode
                0x0000000000000000       0x3a ./App/src/sl_protocol.o
 .text.SL_ReadRegisterDischargMosState
                0x0000000000000000       0x34 ./App/src/sl_protocol.o
 .text.SL_ReadRegisterHighSideMosTemperature
                0x0000000000000000       0x56 ./App/src/sl_protocol.o
 .text.SL_ReadRegisterSolarOpenCircuitVoltage
                0x0000000000000000       0x56 ./App/src/sl_protocol.o
 .text.SL_ReadRegisterDischargCurrent
                0x0000000000000000       0x54 ./App/src/sl_protocol.o
 .text.SL_ReadRegisterChargCurrent
                0x0000000000000000       0x54 ./App/src/sl_protocol.o
 .text.SL_ReadRegisterBatteryVoltage
                0x0000000000000000       0x54 ./App/src/sl_protocol.o
 .text.SL_MsgProcFunc_Registration_request
                0x0000000000000000       0x7c ./App/src/sl_protocol.o
 .text.SL_MsgProcFunc_Broadcast_Scan
                0x0000000000000000       0x50 ./App/src/sl_protocol.o
 .text.SL_MsgProcFunc_Write_Register
                0x0000000000000000       0x66 ./App/src/sl_protocol.o
 .text.CheckFunc
                0x0000000000000000       0x3e ./App/src/sl_protocol.o
 .text.randomDelay
                0x0000000000000000       0x40 ./App/src/sl_protocol.o
 .text.Check_485_bus_busy
                0x0000000000000000       0x9a ./App/src/sl_protocol.o
 .text.SL_MsgProcFunc_Remote_Upgrade
                0x0000000000000000       0xc2 ./App/src/sl_protocol.o
 .text.SL_MsgProcFunc_Update_Profile
                0x0000000000000000       0xc2 ./App/src/sl_protocol.o
 .text.SL_MsgProcFunc_Read_Register
                0x0000000000000000      0x1c0 ./App/src/sl_protocol.o
 .text.FRT_MsgHandler
                0x0000000000000000       0x3a ./App/src/sl_protocol.o
 .text.read_and_process_uart_data
                0x0000000000000000      0x322 ./App/src/sl_protocol.o
 .bss.g_RegTblW
                0x0000000000000000        0x0 ./App/src/sl_protocol.o
 .bss.rs485_buff
                0x0000000000000000       0x32 ./App/src/sl_protocol.o
 .data.g_MsgTbl
                0x0000000000000000       0x30 ./App/src/sl_protocol.o
 .data.g_RegTblR
                0x0000000000000000       0x38 ./App/src/sl_protocol.o
 .rodata.SL_MsgProcFunc_Registration_request.str1.4
                0x0000000000000000       0x29 ./App/src/sl_protocol.o
 .rodata.SL_MsgProcFunc_Write_Register.str1.4
                0x0000000000000000       0x7b ./App/src/sl_protocol.o
 .rodata.SL_ReadRegisterBatteryVoltage.str1.4
                0x0000000000000000       0x31 ./App/src/sl_protocol.o
 .rodata.SL_ReadRegisterChargCurrent.str1.4
                0x0000000000000000       0x2f ./App/src/sl_protocol.o
 .rodata.SL_ReadRegisterDischargCurrent.str1.4
                0x0000000000000000       0x32 ./App/src/sl_protocol.o
 .rodata.SL_ReadRegisterDischargMosState.str1.4
                0x0000000000000000       0x33 ./App/src/sl_protocol.o
 .rodata.SL_ReadRegisterHighSideMosTemperature.cst4
                0x0000000000000000        0x4 ./App/src/sl_protocol.o
 .rodata.SL_ReadRegisterHighSideMosTemperature.str1.4
                0x0000000000000000       0x39 ./App/src/sl_protocol.o
 .rodata.SL_ReadRegisterMPPTMode.str1.4
                0x0000000000000000       0x2b ./App/src/sl_protocol.o
 .rodata.SL_ReadRegisterSolarOpenCircuitVoltage.str1.4
                0x0000000000000000       0x3a ./App/src/sl_protocol.o
 .rodata.read_and_process_uart_data.str1.4
                0x0000000000000000      0x164 ./App/src/sl_protocol.o
 .text          0x0000000000000000        0x0 ./App/src/task.o
 .data          0x0000000000000000        0x0 ./App/src/task.o
 .bss           0x0000000000000000        0x0 ./App/src/task.o
 .text.stop_mpptWork
                0x0000000000000000       0x44 ./App/src/task.o
 .text.start_mpptWork
                0x0000000000000000       0x34 ./App/src/task.o
 .text.Task_softStart
                0x0000000000000000      0x1a0 ./App/src/task.o
 .text.Task_impedanceCalculation
                0x0000000000000000      0x1d6 ./App/src/task.o
 .text.Task_startMpptControl
                0x0000000000000000      0x118 ./App/src/task.o
 .text.Task_usart
                0x0000000000000000       0x20 ./App/src/task.o
 .text.Task_refreshRegister
                0x0000000000000000      0x38a ./App/src/task.o
 .text.Task_recvbroadcast
                0x0000000000000000      0x19e ./App/src/task.o
 .text.Task_sensorEnableBroadcast
                0x0000000000000000       0x64 ./App/src/task.o
 .bss.m_impedanceCalculation
                0x0000000000000000       0x10 ./App/src/task.o
 .bss.m_recvbroadcast
                0x0000000000000000       0x10 ./App/src/task.o
 .bss.m_refreshRegister
                0x0000000000000000       0x10 ./App/src/task.o
 .bss.m_sensorEnableBroadcast
                0x0000000000000000       0x10 ./App/src/task.o
 .bss.m_softStart
                0x0000000000000000       0x10 ./App/src/task.o
 .bss.m_startMpptControl
                0x0000000000000000       0x10 ./App/src/task.o
 .bss.m_usart   0x0000000000000000       0x10 ./App/src/task.o
 .rodata.Task_impedanceCalculation.cst8
                0x0000000000000000        0x8 ./App/src/task.o
 .rodata.Task_refreshRegister.cst4
                0x0000000000000000        0x8 ./App/src/task.o
 .rodata.Task_refreshRegister.cst8
                0x0000000000000000       0x10 ./App/src/task.o
 .rodata.Task_softStart.cst8
                0x0000000000000000       0x10 ./App/src/task.o
 .rodata.stop_mpptWork.cst4
                0x0000000000000000        0x4 ./App/src/task.o
 .sbss.RegistrationRequestFlag
                0x0000000000000000        0x1 ./App/src/task.o
 .sbss.checkRegisterRefreshTimeFlag.6467
                0x0000000000000000        0x2 ./App/src/task.o
 .sbss.checkSolarOpenCircuitVTimeFlag.6444
                0x0000000000000000        0x2 ./App/src/task.o
 .sbss.currOne.6492
                0x0000000000000000        0x4 ./App/src/task.o
 .sbss.currTwo.6494
                0x0000000000000000        0x4 ./App/src/task.o
 .sbss.dutyRatio.6451
                0x0000000000000000        0x4 ./App/src/task.o
 .sbss.enabBroadcastTimeFlag.6515
                0x0000000000000000        0x4 ./App/src/task.o
 .sbss.g_batteryState
                0x0000000000000000        0x1 ./App/src/task.o
 .sbss.g_recvBroadcastDevice
                0x0000000000000000        0x4 ./App/src/task.o
 .sbss.g_recvBroadcastRegisterNumber
                0x0000000000000000        0x1 ./App/src/task.o
 .sbss.num.6450
                0x0000000000000000        0x2 ./App/src/task.o
 .sbss.num.6491
                0x0000000000000000        0x1 ./App/src/task.o
 .sbss.overTemperature
                0x0000000000000000        0x1 ./App/src/task.o
 .sbss.recvbroadcast_flag
                0x0000000000000000        0x1 ./App/src/task.o
 .sbss.run_number.6477
                0x0000000000000000        0x1 ./App/src/task.o
 .sbss.voltOne.6493
                0x0000000000000000        0x4 ./App/src/task.o
 .sdata.only_once.6445
                0x0000000000000000        0x1 ./App/src/task.o
 .sdata.run_Broadcast
                0x0000000000000000        0x1 ./App/src/task.o
 .text          0x0000000000000000        0x0 ./App/src/uart_dev.o
 .data          0x0000000000000000        0x0 ./App/src/uart_dev.o
 .bss           0x0000000000000000        0x0 ./App/src/uart_dev.o
 .text.uart_putchar
                0x0000000000000000       0x56 ./App/src/uart_dev.o
 .text.bat485_tx_enabla
                0x0000000000000000       0x26 ./App/src/uart_dev.o
 .text.bat485_tx_disenabla
                0x0000000000000000       0x26 ./App/src/uart_dev.o
 .text.gw485_tx_enabla
                0x0000000000000000       0x24 ./App/src/uart_dev.o
 .text.gw485_tx_disenabla
                0x0000000000000000       0x24 ./App/src/uart_dev.o
 .text.uart_sendstr
                0x0000000000000000       0x8e ./App/src/uart_dev.o
 .text.uart_dev_write
                0x0000000000000000       0x8e ./App/src/uart_dev.o
 .text.uart_dev_char_present
                0x0000000000000000       0x18 ./App/src/uart_dev.o
 .text.uart_dev_in_char
                0x0000000000000000       0x38 ./App/src/uart_dev.o
 .text.ring_queue_dev_char_present
                0x0000000000000000        0xe ./App/src/uart_dev.o
 .text.ring_queue_dev_in_char
                0x0000000000000000       0x30 ./App/src/uart_dev.o
 .text.ring_queue_length
                0x0000000000000000       0x1a ./App/src/uart_dev.o
 .bss.rs485_out_buff
                0x0000000000000000       0x64 ./App/src/uart_dev.o
 .text          0x0000000000000000        0x0 d:/psx/rj/mounriver_studio/toolchain/risc-v embedded gcc/bin/../lib/gcc/riscv-none-embed/8.2.0/rv32imacxw/ilp32\libgcc.a(adddf3.o)
 .data          0x0000000000000000        0x0 d:/psx/rj/mounriver_studio/toolchain/risc-v embedded gcc/bin/../lib/gcc/riscv-none-embed/8.2.0/rv32imacxw/ilp32\libgcc.a(adddf3.o)
 .bss           0x0000000000000000        0x0 d:/psx/rj/mounriver_studio/toolchain/risc-v embedded gcc/bin/../lib/gcc/riscv-none-embed/8.2.0/rv32imacxw/ilp32\libgcc.a(adddf3.o)
 .text.__adddf3
                0x0000000000000000      0x738 d:/psx/rj/mounriver_studio/toolchain/risc-v embedded gcc/bin/../lib/gcc/riscv-none-embed/8.2.0/rv32imacxw/ilp32\libgcc.a(adddf3.o)
 .debug_frame   0x0000000000000000       0x44 d:/psx/rj/mounriver_studio/toolchain/risc-v embedded gcc/bin/../lib/gcc/riscv-none-embed/8.2.0/rv32imacxw/ilp32\libgcc.a(adddf3.o)
 .text          0x0000000000000000        0x0 d:/psx/rj/mounriver_studio/toolchain/risc-v embedded gcc/bin/../lib/gcc/riscv-none-embed/8.2.0/rv32imacxw/ilp32\libgcc.a(gedf2.o)
 .data          0x0000000000000000        0x0 d:/psx/rj/mounriver_studio/toolchain/risc-v embedded gcc/bin/../lib/gcc/riscv-none-embed/8.2.0/rv32imacxw/ilp32\libgcc.a(gedf2.o)
 .bss           0x0000000000000000        0x0 d:/psx/rj/mounriver_studio/toolchain/risc-v embedded gcc/bin/../lib/gcc/riscv-none-embed/8.2.0/rv32imacxw/ilp32\libgcc.a(gedf2.o)
 .text          0x0000000000000000        0x0 d:/psx/rj/mounriver_studio/toolchain/risc-v embedded gcc/bin/../lib/gcc/riscv-none-embed/8.2.0/rv32imacxw/ilp32\libgcc.a(ledf2.o)
 .data          0x0000000000000000        0x0 d:/psx/rj/mounriver_studio/toolchain/risc-v embedded gcc/bin/../lib/gcc/riscv-none-embed/8.2.0/rv32imacxw/ilp32\libgcc.a(ledf2.o)
 .bss           0x0000000000000000        0x0 d:/psx/rj/mounriver_studio/toolchain/risc-v embedded gcc/bin/../lib/gcc/riscv-none-embed/8.2.0/rv32imacxw/ilp32\libgcc.a(ledf2.o)
 .text          0x0000000000000000        0x0 d:/psx/rj/mounriver_studio/toolchain/risc-v embedded gcc/bin/../lib/gcc/riscv-none-embed/8.2.0/rv32imacxw/ilp32\libgcc.a(muldf3.o)
 .data          0x0000000000000000        0x0 d:/psx/rj/mounriver_studio/toolchain/risc-v embedded gcc/bin/../lib/gcc/riscv-none-embed/8.2.0/rv32imacxw/ilp32\libgcc.a(muldf3.o)
 .bss           0x0000000000000000        0x0 d:/psx/rj/mounriver_studio/toolchain/risc-v embedded gcc/bin/../lib/gcc/riscv-none-embed/8.2.0/rv32imacxw/ilp32\libgcc.a(muldf3.o)
 .text          0x0000000000000000        0x0 d:/psx/rj/mounriver_studio/toolchain/risc-v embedded gcc/bin/../lib/gcc/riscv-none-embed/8.2.0/rv32imacxw/ilp32\libgcc.a(subdf3.o)
 .data          0x0000000000000000        0x0 d:/psx/rj/mounriver_studio/toolchain/risc-v embedded gcc/bin/../lib/gcc/riscv-none-embed/8.2.0/rv32imacxw/ilp32\libgcc.a(subdf3.o)
 .bss           0x0000000000000000        0x0 d:/psx/rj/mounriver_studio/toolchain/risc-v embedded gcc/bin/../lib/gcc/riscv-none-embed/8.2.0/rv32imacxw/ilp32\libgcc.a(subdf3.o)
 .text          0x0000000000000000        0x0 d:/psx/rj/mounriver_studio/toolchain/risc-v embedded gcc/bin/../lib/gcc/riscv-none-embed/8.2.0/rv32imacxw/ilp32\libgcc.a(floatsidf.o)
 .data          0x0000000000000000        0x0 d:/psx/rj/mounriver_studio/toolchain/risc-v embedded gcc/bin/../lib/gcc/riscv-none-embed/8.2.0/rv32imacxw/ilp32\libgcc.a(floatsidf.o)
 .bss           0x0000000000000000        0x0 d:/psx/rj/mounriver_studio/toolchain/risc-v embedded gcc/bin/../lib/gcc/riscv-none-embed/8.2.0/rv32imacxw/ilp32\libgcc.a(floatsidf.o)
 .text          0x0000000000000000        0x0 d:/psx/rj/mounriver_studio/toolchain/risc-v embedded gcc/bin/../lib/gcc/riscv-none-embed/8.2.0/rv32imacxw/ilp32\libgcc.a(addsf3.o)
 .data          0x0000000000000000        0x0 d:/psx/rj/mounriver_studio/toolchain/risc-v embedded gcc/bin/../lib/gcc/riscv-none-embed/8.2.0/rv32imacxw/ilp32\libgcc.a(addsf3.o)
 .bss           0x0000000000000000        0x0 d:/psx/rj/mounriver_studio/toolchain/risc-v embedded gcc/bin/../lib/gcc/riscv-none-embed/8.2.0/rv32imacxw/ilp32\libgcc.a(addsf3.o)
 .text.__addsf3
                0x0000000000000000      0x36e d:/psx/rj/mounriver_studio/toolchain/risc-v embedded gcc/bin/../lib/gcc/riscv-none-embed/8.2.0/rv32imacxw/ilp32\libgcc.a(addsf3.o)
 .debug_frame   0x0000000000000000       0x40 d:/psx/rj/mounriver_studio/toolchain/risc-v embedded gcc/bin/../lib/gcc/riscv-none-embed/8.2.0/rv32imacxw/ilp32\libgcc.a(addsf3.o)
 .text          0x0000000000000000        0x0 d:/psx/rj/mounriver_studio/toolchain/risc-v embedded gcc/bin/../lib/gcc/riscv-none-embed/8.2.0/rv32imacxw/ilp32\libgcc.a(divsf3.o)
 .data          0x0000000000000000        0x0 d:/psx/rj/mounriver_studio/toolchain/risc-v embedded gcc/bin/../lib/gcc/riscv-none-embed/8.2.0/rv32imacxw/ilp32\libgcc.a(divsf3.o)
 .bss           0x0000000000000000        0x0 d:/psx/rj/mounriver_studio/toolchain/risc-v embedded gcc/bin/../lib/gcc/riscv-none-embed/8.2.0/rv32imacxw/ilp32\libgcc.a(divsf3.o)
 .text          0x0000000000000000        0x0 d:/psx/rj/mounriver_studio/toolchain/risc-v embedded gcc/bin/../lib/gcc/riscv-none-embed/8.2.0/rv32imacxw/ilp32\libgcc.a(eqsf2.o)
 .data          0x0000000000000000        0x0 d:/psx/rj/mounriver_studio/toolchain/risc-v embedded gcc/bin/../lib/gcc/riscv-none-embed/8.2.0/rv32imacxw/ilp32\libgcc.a(eqsf2.o)
 .bss           0x0000000000000000        0x0 d:/psx/rj/mounriver_studio/toolchain/risc-v embedded gcc/bin/../lib/gcc/riscv-none-embed/8.2.0/rv32imacxw/ilp32\libgcc.a(eqsf2.o)
 .text.__eqsf2  0x0000000000000000       0x5c d:/psx/rj/mounriver_studio/toolchain/risc-v embedded gcc/bin/../lib/gcc/riscv-none-embed/8.2.0/rv32imacxw/ilp32\libgcc.a(eqsf2.o)
 .debug_frame   0x0000000000000000       0x20 d:/psx/rj/mounriver_studio/toolchain/risc-v embedded gcc/bin/../lib/gcc/riscv-none-embed/8.2.0/rv32imacxw/ilp32\libgcc.a(eqsf2.o)
 .text          0x0000000000000000        0x0 d:/psx/rj/mounriver_studio/toolchain/risc-v embedded gcc/bin/../lib/gcc/riscv-none-embed/8.2.0/rv32imacxw/ilp32\libgcc.a(gesf2.o)
 .data          0x0000000000000000        0x0 d:/psx/rj/mounriver_studio/toolchain/risc-v embedded gcc/bin/../lib/gcc/riscv-none-embed/8.2.0/rv32imacxw/ilp32\libgcc.a(gesf2.o)
 .bss           0x0000000000000000        0x0 d:/psx/rj/mounriver_studio/toolchain/risc-v embedded gcc/bin/../lib/gcc/riscv-none-embed/8.2.0/rv32imacxw/ilp32\libgcc.a(gesf2.o)
 .text          0x0000000000000000        0x0 d:/psx/rj/mounriver_studio/toolchain/risc-v embedded gcc/bin/../lib/gcc/riscv-none-embed/8.2.0/rv32imacxw/ilp32\libgcc.a(lesf2.o)
 .data          0x0000000000000000        0x0 d:/psx/rj/mounriver_studio/toolchain/risc-v embedded gcc/bin/../lib/gcc/riscv-none-embed/8.2.0/rv32imacxw/ilp32\libgcc.a(lesf2.o)
 .bss           0x0000000000000000        0x0 d:/psx/rj/mounriver_studio/toolchain/risc-v embedded gcc/bin/../lib/gcc/riscv-none-embed/8.2.0/rv32imacxw/ilp32\libgcc.a(lesf2.o)
 .text          0x0000000000000000        0x0 d:/psx/rj/mounriver_studio/toolchain/risc-v embedded gcc/bin/../lib/gcc/riscv-none-embed/8.2.0/rv32imacxw/ilp32\libgcc.a(mulsf3.o)
 .data          0x0000000000000000        0x0 d:/psx/rj/mounriver_studio/toolchain/risc-v embedded gcc/bin/../lib/gcc/riscv-none-embed/8.2.0/rv32imacxw/ilp32\libgcc.a(mulsf3.o)
 .bss           0x0000000000000000        0x0 d:/psx/rj/mounriver_studio/toolchain/risc-v embedded gcc/bin/../lib/gcc/riscv-none-embed/8.2.0/rv32imacxw/ilp32\libgcc.a(mulsf3.o)
 .text          0x0000000000000000        0x0 d:/psx/rj/mounriver_studio/toolchain/risc-v embedded gcc/bin/../lib/gcc/riscv-none-embed/8.2.0/rv32imacxw/ilp32\libgcc.a(subsf3.o)
 .data          0x0000000000000000        0x0 d:/psx/rj/mounriver_studio/toolchain/risc-v embedded gcc/bin/../lib/gcc/riscv-none-embed/8.2.0/rv32imacxw/ilp32\libgcc.a(subsf3.o)
 .bss           0x0000000000000000        0x0 d:/psx/rj/mounriver_studio/toolchain/risc-v embedded gcc/bin/../lib/gcc/riscv-none-embed/8.2.0/rv32imacxw/ilp32\libgcc.a(subsf3.o)
 .text          0x0000000000000000        0x0 d:/psx/rj/mounriver_studio/toolchain/risc-v embedded gcc/bin/../lib/gcc/riscv-none-embed/8.2.0/rv32imacxw/ilp32\libgcc.a(fixsfsi.o)
 .data          0x0000000000000000        0x0 d:/psx/rj/mounriver_studio/toolchain/risc-v embedded gcc/bin/../lib/gcc/riscv-none-embed/8.2.0/rv32imacxw/ilp32\libgcc.a(fixsfsi.o)
 .bss           0x0000000000000000        0x0 d:/psx/rj/mounriver_studio/toolchain/risc-v embedded gcc/bin/../lib/gcc/riscv-none-embed/8.2.0/rv32imacxw/ilp32\libgcc.a(fixsfsi.o)
 .text          0x0000000000000000        0x0 d:/psx/rj/mounriver_studio/toolchain/risc-v embedded gcc/bin/../lib/gcc/riscv-none-embed/8.2.0/rv32imacxw/ilp32\libgcc.a(fixunssfsi.o)
 .data          0x0000000000000000        0x0 d:/psx/rj/mounriver_studio/toolchain/risc-v embedded gcc/bin/../lib/gcc/riscv-none-embed/8.2.0/rv32imacxw/ilp32\libgcc.a(fixunssfsi.o)
 .bss           0x0000000000000000        0x0 d:/psx/rj/mounriver_studio/toolchain/risc-v embedded gcc/bin/../lib/gcc/riscv-none-embed/8.2.0/rv32imacxw/ilp32\libgcc.a(fixunssfsi.o)
 .text          0x0000000000000000        0x0 d:/psx/rj/mounriver_studio/toolchain/risc-v embedded gcc/bin/../lib/gcc/riscv-none-embed/8.2.0/rv32imacxw/ilp32\libgcc.a(floatsisf.o)
 .data          0x0000000000000000        0x0 d:/psx/rj/mounriver_studio/toolchain/risc-v embedded gcc/bin/../lib/gcc/riscv-none-embed/8.2.0/rv32imacxw/ilp32\libgcc.a(floatsisf.o)
 .bss           0x0000000000000000        0x0 d:/psx/rj/mounriver_studio/toolchain/risc-v embedded gcc/bin/../lib/gcc/riscv-none-embed/8.2.0/rv32imacxw/ilp32\libgcc.a(floatsisf.o)
 .text.__floatsisf
                0x0000000000000000       0xcc d:/psx/rj/mounriver_studio/toolchain/risc-v embedded gcc/bin/../lib/gcc/riscv-none-embed/8.2.0/rv32imacxw/ilp32\libgcc.a(floatsisf.o)
 .debug_frame   0x0000000000000000       0x38 d:/psx/rj/mounriver_studio/toolchain/risc-v embedded gcc/bin/../lib/gcc/riscv-none-embed/8.2.0/rv32imacxw/ilp32\libgcc.a(floatsisf.o)
 .text          0x0000000000000000        0x0 d:/psx/rj/mounriver_studio/toolchain/risc-v embedded gcc/bin/../lib/gcc/riscv-none-embed/8.2.0/rv32imacxw/ilp32\libgcc.a(floatunsisf.o)
 .data          0x0000000000000000        0x0 d:/psx/rj/mounriver_studio/toolchain/risc-v embedded gcc/bin/../lib/gcc/riscv-none-embed/8.2.0/rv32imacxw/ilp32\libgcc.a(floatunsisf.o)
 .bss           0x0000000000000000        0x0 d:/psx/rj/mounriver_studio/toolchain/risc-v embedded gcc/bin/../lib/gcc/riscv-none-embed/8.2.0/rv32imacxw/ilp32\libgcc.a(floatunsisf.o)
 .text          0x0000000000000000        0x0 d:/psx/rj/mounriver_studio/toolchain/risc-v embedded gcc/bin/../lib/gcc/riscv-none-embed/8.2.0/rv32imacxw/ilp32\libgcc.a(extendsfdf2.o)
 .data          0x0000000000000000        0x0 d:/psx/rj/mounriver_studio/toolchain/risc-v embedded gcc/bin/../lib/gcc/riscv-none-embed/8.2.0/rv32imacxw/ilp32\libgcc.a(extendsfdf2.o)
 .bss           0x0000000000000000        0x0 d:/psx/rj/mounriver_studio/toolchain/risc-v embedded gcc/bin/../lib/gcc/riscv-none-embed/8.2.0/rv32imacxw/ilp32\libgcc.a(extendsfdf2.o)
 .text          0x0000000000000000        0x0 d:/psx/rj/mounriver_studio/toolchain/risc-v embedded gcc/bin/../lib/gcc/riscv-none-embed/8.2.0/rv32imacxw/ilp32\libgcc.a(truncdfsf2.o)
 .data          0x0000000000000000        0x0 d:/psx/rj/mounriver_studio/toolchain/risc-v embedded gcc/bin/../lib/gcc/riscv-none-embed/8.2.0/rv32imacxw/ilp32\libgcc.a(truncdfsf2.o)
 .bss           0x0000000000000000        0x0 d:/psx/rj/mounriver_studio/toolchain/risc-v embedded gcc/bin/../lib/gcc/riscv-none-embed/8.2.0/rv32imacxw/ilp32\libgcc.a(truncdfsf2.o)
 .data          0x0000000000000000        0x0 d:/psx/rj/mounriver_studio/toolchain/risc-v embedded gcc/bin/../lib/gcc/riscv-none-embed/8.2.0/rv32imacxw/ilp32\libgcc.a(save-restore.o)
 .bss           0x0000000000000000        0x0 d:/psx/rj/mounriver_studio/toolchain/risc-v embedded gcc/bin/../lib/gcc/riscv-none-embed/8.2.0/rv32imacxw/ilp32\libgcc.a(save-restore.o)
 .eh_frame      0x0000000000000000       0xf8 d:/psx/rj/mounriver_studio/toolchain/risc-v embedded gcc/bin/../lib/gcc/riscv-none-embed/8.2.0/rv32imacxw/ilp32\libgcc.a(save-restore.o)
 .text          0x0000000000000000        0x0 d:/psx/rj/mounriver_studio/toolchain/risc-v embedded gcc/bin/../lib/gcc/riscv-none-embed/8.2.0/rv32imacxw/ilp32\libgcc.a(_clzsi2.o)
 .data          0x0000000000000000        0x0 d:/psx/rj/mounriver_studio/toolchain/risc-v embedded gcc/bin/../lib/gcc/riscv-none-embed/8.2.0/rv32imacxw/ilp32\libgcc.a(_clzsi2.o)
 .bss           0x0000000000000000        0x0 d:/psx/rj/mounriver_studio/toolchain/risc-v embedded gcc/bin/../lib/gcc/riscv-none-embed/8.2.0/rv32imacxw/ilp32\libgcc.a(_clzsi2.o)
 .text          0x0000000000000000        0x0 d:/psx/rj/mounriver_studio/toolchain/risc-v embedded gcc/bin/../lib/gcc/riscv-none-embed/8.2.0/rv32imacxw/ilp32\libgcc.a(_clz.o)
 .data          0x0000000000000000        0x0 d:/psx/rj/mounriver_studio/toolchain/risc-v embedded gcc/bin/../lib/gcc/riscv-none-embed/8.2.0/rv32imacxw/ilp32\libgcc.a(_clz.o)
 .bss           0x0000000000000000        0x0 d:/psx/rj/mounriver_studio/toolchain/risc-v embedded gcc/bin/../lib/gcc/riscv-none-embed/8.2.0/rv32imacxw/ilp32\libgcc.a(_clz.o)
 .text          0x0000000000000000        0x0 d:/psx/rj/mounriver_studio/toolchain/risc-v embedded gcc/bin/../lib/gcc/riscv-none-embed/8.2.0/../../../../riscv-none-embed/lib/rv32imacxw/ilp32\libg_nano.a(lib_a-memcpy.o)
 .data          0x0000000000000000        0x0 d:/psx/rj/mounriver_studio/toolchain/risc-v embedded gcc/bin/../lib/gcc/riscv-none-embed/8.2.0/../../../../riscv-none-embed/lib/rv32imacxw/ilp32\libg_nano.a(lib_a-memcpy.o)
 .bss           0x0000000000000000        0x0 d:/psx/rj/mounriver_studio/toolchain/risc-v embedded gcc/bin/../lib/gcc/riscv-none-embed/8.2.0/../../../../riscv-none-embed/lib/rv32imacxw/ilp32\libg_nano.a(lib_a-memcpy.o)
 .data          0x0000000000000000        0x0 d:/psx/rj/mounriver_studio/toolchain/risc-v embedded gcc/bin/../lib/gcc/riscv-none-embed/8.2.0/../../../../riscv-none-embed/lib/rv32imacxw/ilp32\libg_nano.a(lib_a-memset.o)
 .bss           0x0000000000000000        0x0 d:/psx/rj/mounriver_studio/toolchain/risc-v embedded gcc/bin/../lib/gcc/riscv-none-embed/8.2.0/../../../../riscv-none-embed/lib/rv32imacxw/ilp32\libg_nano.a(lib_a-memset.o)
 .text          0x0000000000000000        0x0 d:/psx/rj/mounriver_studio/toolchain/risc-v embedded gcc/bin/../lib/gcc/riscv-none-embed/8.2.0/../../../../riscv-none-embed/lib/rv32imacxw/ilp32\libg_nano.a(lib_a-printf.o)
 .data          0x0000000000000000        0x0 d:/psx/rj/mounriver_studio/toolchain/risc-v embedded gcc/bin/../lib/gcc/riscv-none-embed/8.2.0/../../../../riscv-none-embed/lib/rv32imacxw/ilp32\libg_nano.a(lib_a-printf.o)
 .bss           0x0000000000000000        0x0 d:/psx/rj/mounriver_studio/toolchain/risc-v embedded gcc/bin/../lib/gcc/riscv-none-embed/8.2.0/../../../../riscv-none-embed/lib/rv32imacxw/ilp32\libg_nano.a(lib_a-printf.o)
 .text._printf_r
                0x0000000000000000       0x40 d:/psx/rj/mounriver_studio/toolchain/risc-v embedded gcc/bin/../lib/gcc/riscv-none-embed/8.2.0/../../../../riscv-none-embed/lib/rv32imacxw/ilp32\libg_nano.a(lib_a-printf.o)
 .text          0x0000000000000000        0x0 d:/psx/rj/mounriver_studio/toolchain/risc-v embedded gcc/bin/../lib/gcc/riscv-none-embed/8.2.0/../../../../riscv-none-embed/lib/rv32imacxw/ilp32\libg_nano.a(lib_a-putchar.o)
 .data          0x0000000000000000        0x0 d:/psx/rj/mounriver_studio/toolchain/risc-v embedded gcc/bin/../lib/gcc/riscv-none-embed/8.2.0/../../../../riscv-none-embed/lib/rv32imacxw/ilp32\libg_nano.a(lib_a-putchar.o)
 .bss           0x0000000000000000        0x0 d:/psx/rj/mounriver_studio/toolchain/risc-v embedded gcc/bin/../lib/gcc/riscv-none-embed/8.2.0/../../../../riscv-none-embed/lib/rv32imacxw/ilp32\libg_nano.a(lib_a-putchar.o)
 .text._putchar_r
                0x0000000000000000       0x2c d:/psx/rj/mounriver_studio/toolchain/risc-v embedded gcc/bin/../lib/gcc/riscv-none-embed/8.2.0/../../../../riscv-none-embed/lib/rv32imacxw/ilp32\libg_nano.a(lib_a-putchar.o)
 .text.putchar  0x0000000000000000       0x38 d:/psx/rj/mounriver_studio/toolchain/risc-v embedded gcc/bin/../lib/gcc/riscv-none-embed/8.2.0/../../../../riscv-none-embed/lib/rv32imacxw/ilp32\libg_nano.a(lib_a-putchar.o)
 .debug_frame   0x0000000000000000       0x50 d:/psx/rj/mounriver_studio/toolchain/risc-v embedded gcc/bin/../lib/gcc/riscv-none-embed/8.2.0/../../../../riscv-none-embed/lib/rv32imacxw/ilp32\libg_nano.a(lib_a-putchar.o)
 .text          0x0000000000000000        0x0 d:/psx/rj/mounriver_studio/toolchain/risc-v embedded gcc/bin/../lib/gcc/riscv-none-embed/8.2.0/../../../../riscv-none-embed/lib/rv32imacxw/ilp32\libg_nano.a(lib_a-puts.o)
 .data          0x0000000000000000        0x0 d:/psx/rj/mounriver_studio/toolchain/risc-v embedded gcc/bin/../lib/gcc/riscv-none-embed/8.2.0/../../../../riscv-none-embed/lib/rv32imacxw/ilp32\libg_nano.a(lib_a-puts.o)
 .bss           0x0000000000000000        0x0 d:/psx/rj/mounriver_studio/toolchain/risc-v embedded gcc/bin/../lib/gcc/riscv-none-embed/8.2.0/../../../../riscv-none-embed/lib/rv32imacxw/ilp32\libg_nano.a(lib_a-puts.o)
 .text          0x0000000000000000        0x0 d:/psx/rj/mounriver_studio/toolchain/risc-v embedded gcc/bin/../lib/gcc/riscv-none-embed/8.2.0/../../../../riscv-none-embed/lib/rv32imacxw/ilp32\libg_nano.a(lib_a-rand.o)
 .data          0x0000000000000000        0x0 d:/psx/rj/mounriver_studio/toolchain/risc-v embedded gcc/bin/../lib/gcc/riscv-none-embed/8.2.0/../../../../riscv-none-embed/lib/rv32imacxw/ilp32\libg_nano.a(lib_a-rand.o)
 .bss           0x0000000000000000        0x0 d:/psx/rj/mounriver_studio/toolchain/risc-v embedded gcc/bin/../lib/gcc/riscv-none-embed/8.2.0/../../../../riscv-none-embed/lib/rv32imacxw/ilp32\libg_nano.a(lib_a-rand.o)
 .text.srand    0x0000000000000000       0x60 d:/psx/rj/mounriver_studio/toolchain/risc-v embedded gcc/bin/../lib/gcc/riscv-none-embed/8.2.0/../../../../riscv-none-embed/lib/rv32imacxw/ilp32\libg_nano.a(lib_a-rand.o)
 .text.rand     0x0000000000000000       0x8e d:/psx/rj/mounriver_studio/toolchain/risc-v embedded gcc/bin/../lib/gcc/riscv-none-embed/8.2.0/../../../../riscv-none-embed/lib/rv32imacxw/ilp32\libg_nano.a(lib_a-rand.o)
 .debug_frame   0x0000000000000000       0x5c d:/psx/rj/mounriver_studio/toolchain/risc-v embedded gcc/bin/../lib/gcc/riscv-none-embed/8.2.0/../../../../riscv-none-embed/lib/rv32imacxw/ilp32\libg_nano.a(lib_a-rand.o)
 .text          0x0000000000000000        0x0 d:/psx/rj/mounriver_studio/toolchain/risc-v embedded gcc/bin/../lib/gcc/riscv-none-embed/8.2.0/../../../../riscv-none-embed/lib/rv32imacxw/ilp32\libg_nano.a(lib_a-wbuf.o)
 .data          0x0000000000000000        0x0 d:/psx/rj/mounriver_studio/toolchain/risc-v embedded gcc/bin/../lib/gcc/riscv-none-embed/8.2.0/../../../../riscv-none-embed/lib/rv32imacxw/ilp32\libg_nano.a(lib_a-wbuf.o)
 .bss           0x0000000000000000        0x0 d:/psx/rj/mounriver_studio/toolchain/risc-v embedded gcc/bin/../lib/gcc/riscv-none-embed/8.2.0/../../../../riscv-none-embed/lib/rv32imacxw/ilp32\libg_nano.a(lib_a-wbuf.o)
 .text.__swbuf  0x0000000000000000       0x16 d:/psx/rj/mounriver_studio/toolchain/risc-v embedded gcc/bin/../lib/gcc/riscv-none-embed/8.2.0/../../../../riscv-none-embed/lib/rv32imacxw/ilp32\libg_nano.a(lib_a-wbuf.o)
 .text          0x0000000000000000        0x0 d:/psx/rj/mounriver_studio/toolchain/risc-v embedded gcc/bin/../lib/gcc/riscv-none-embed/8.2.0/../../../../riscv-none-embed/lib/rv32imacxw/ilp32\libg_nano.a(lib_a-wsetup.o)
 .data          0x0000000000000000        0x0 d:/psx/rj/mounriver_studio/toolchain/risc-v embedded gcc/bin/../lib/gcc/riscv-none-embed/8.2.0/../../../../riscv-none-embed/lib/rv32imacxw/ilp32\libg_nano.a(lib_a-wsetup.o)
 .bss           0x0000000000000000        0x0 d:/psx/rj/mounriver_studio/toolchain/risc-v embedded gcc/bin/../lib/gcc/riscv-none-embed/8.2.0/../../../../riscv-none-embed/lib/rv32imacxw/ilp32\libg_nano.a(lib_a-wsetup.o)
 .text          0x0000000000000000        0x0 d:/psx/rj/mounriver_studio/toolchain/risc-v embedded gcc/bin/../lib/gcc/riscv-none-embed/8.2.0/../../../../riscv-none-embed/lib/rv32imacxw/ilp32\libg_nano.a(lib_a-fflush.o)
 .data          0x0000000000000000        0x0 d:/psx/rj/mounriver_studio/toolchain/risc-v embedded gcc/bin/../lib/gcc/riscv-none-embed/8.2.0/../../../../riscv-none-embed/lib/rv32imacxw/ilp32\libg_nano.a(lib_a-fflush.o)
 .bss           0x0000000000000000        0x0 d:/psx/rj/mounriver_studio/toolchain/risc-v embedded gcc/bin/../lib/gcc/riscv-none-embed/8.2.0/../../../../riscv-none-embed/lib/rv32imacxw/ilp32\libg_nano.a(lib_a-fflush.o)
 .text.fflush   0x0000000000000000       0x30 d:/psx/rj/mounriver_studio/toolchain/risc-v embedded gcc/bin/../lib/gcc/riscv-none-embed/8.2.0/../../../../riscv-none-embed/lib/rv32imacxw/ilp32\libg_nano.a(lib_a-fflush.o)
 .text          0x0000000000000000        0x0 d:/psx/rj/mounriver_studio/toolchain/risc-v embedded gcc/bin/../lib/gcc/riscv-none-embed/8.2.0/../../../../riscv-none-embed/lib/rv32imacxw/ilp32\libg_nano.a(lib_a-findfp.o)
 .data          0x0000000000000000        0x0 d:/psx/rj/mounriver_studio/toolchain/risc-v embedded gcc/bin/../lib/gcc/riscv-none-embed/8.2.0/../../../../riscv-none-embed/lib/rv32imacxw/ilp32\libg_nano.a(lib_a-findfp.o)
 .bss           0x0000000000000000        0x0 d:/psx/rj/mounriver_studio/toolchain/risc-v embedded gcc/bin/../lib/gcc/riscv-none-embed/8.2.0/../../../../riscv-none-embed/lib/rv32imacxw/ilp32\libg_nano.a(lib_a-findfp.o)
 .text.__fp_lock
                0x0000000000000000        0x4 d:/psx/rj/mounriver_studio/toolchain/risc-v embedded gcc/bin/../lib/gcc/riscv-none-embed/8.2.0/../../../../riscv-none-embed/lib/rv32imacxw/ilp32\libg_nano.a(lib_a-findfp.o)
 .text.__fp_unlock
                0x0000000000000000        0x4 d:/psx/rj/mounriver_studio/toolchain/risc-v embedded gcc/bin/../lib/gcc/riscv-none-embed/8.2.0/../../../../riscv-none-embed/lib/rv32imacxw/ilp32\libg_nano.a(lib_a-findfp.o)
 .text._cleanup
                0x0000000000000000       0x12 d:/psx/rj/mounriver_studio/toolchain/risc-v embedded gcc/bin/../lib/gcc/riscv-none-embed/8.2.0/../../../../riscv-none-embed/lib/rv32imacxw/ilp32\libg_nano.a(lib_a-findfp.o)
 .text.__sfp_lock_acquire
                0x0000000000000000        0x2 d:/psx/rj/mounriver_studio/toolchain/risc-v embedded gcc/bin/../lib/gcc/riscv-none-embed/8.2.0/../../../../riscv-none-embed/lib/rv32imacxw/ilp32\libg_nano.a(lib_a-findfp.o)
 .text.__sfp_lock_release
                0x0000000000000000        0x2 d:/psx/rj/mounriver_studio/toolchain/risc-v embedded gcc/bin/../lib/gcc/riscv-none-embed/8.2.0/../../../../riscv-none-embed/lib/rv32imacxw/ilp32\libg_nano.a(lib_a-findfp.o)
 .text.__sinit_lock_acquire
                0x0000000000000000        0x2 d:/psx/rj/mounriver_studio/toolchain/risc-v embedded gcc/bin/../lib/gcc/riscv-none-embed/8.2.0/../../../../riscv-none-embed/lib/rv32imacxw/ilp32\libg_nano.a(lib_a-findfp.o)
 .text.__sinit_lock_release
                0x0000000000000000        0x2 d:/psx/rj/mounriver_studio/toolchain/risc-v embedded gcc/bin/../lib/gcc/riscv-none-embed/8.2.0/../../../../riscv-none-embed/lib/rv32imacxw/ilp32\libg_nano.a(lib_a-findfp.o)
 .text.__fp_lock_all
                0x0000000000000000       0x1a d:/psx/rj/mounriver_studio/toolchain/risc-v embedded gcc/bin/../lib/gcc/riscv-none-embed/8.2.0/../../../../riscv-none-embed/lib/rv32imacxw/ilp32\libg_nano.a(lib_a-findfp.o)
 .text.__fp_unlock_all
                0x0000000000000000       0x1a d:/psx/rj/mounriver_studio/toolchain/risc-v embedded gcc/bin/../lib/gcc/riscv-none-embed/8.2.0/../../../../riscv-none-embed/lib/rv32imacxw/ilp32\libg_nano.a(lib_a-findfp.o)
 .text          0x0000000000000000        0x0 d:/psx/rj/mounriver_studio/toolchain/risc-v embedded gcc/bin/../lib/gcc/riscv-none-embed/8.2.0/../../../../riscv-none-embed/lib/rv32imacxw/ilp32\libg_nano.a(lib_a-fwalk.o)
 .data          0x0000000000000000        0x0 d:/psx/rj/mounriver_studio/toolchain/risc-v embedded gcc/bin/../lib/gcc/riscv-none-embed/8.2.0/../../../../riscv-none-embed/lib/rv32imacxw/ilp32\libg_nano.a(lib_a-fwalk.o)
 .bss           0x0000000000000000        0x0 d:/psx/rj/mounriver_studio/toolchain/risc-v embedded gcc/bin/../lib/gcc/riscv-none-embed/8.2.0/../../../../riscv-none-embed/lib/rv32imacxw/ilp32\libg_nano.a(lib_a-fwalk.o)
 .text._fwalk   0x0000000000000000       0x60 d:/psx/rj/mounriver_studio/toolchain/risc-v embedded gcc/bin/../lib/gcc/riscv-none-embed/8.2.0/../../../../riscv-none-embed/lib/rv32imacxw/ilp32\libg_nano.a(lib_a-fwalk.o)
 .text          0x0000000000000000        0x0 d:/psx/rj/mounriver_studio/toolchain/risc-v embedded gcc/bin/../lib/gcc/riscv-none-embed/8.2.0/../../../../riscv-none-embed/lib/rv32imacxw/ilp32\libg_nano.a(lib_a-impure.o)
 .data          0x0000000000000000        0x0 d:/psx/rj/mounriver_studio/toolchain/risc-v embedded gcc/bin/../lib/gcc/riscv-none-embed/8.2.0/../../../../riscv-none-embed/lib/rv32imacxw/ilp32\libg_nano.a(lib_a-impure.o)
 .bss           0x0000000000000000        0x0 d:/psx/rj/mounriver_studio/toolchain/risc-v embedded gcc/bin/../lib/gcc/riscv-none-embed/8.2.0/../../../../riscv-none-embed/lib/rv32imacxw/ilp32\libg_nano.a(lib_a-impure.o)
 .text          0x0000000000000000        0x0 d:/psx/rj/mounriver_studio/toolchain/risc-v embedded gcc/bin/../lib/gcc/riscv-none-embed/8.2.0/../../../../riscv-none-embed/lib/rv32imacxw/ilp32\libg_nano.a(lib_a-makebuf.o)
 .data          0x0000000000000000        0x0 d:/psx/rj/mounriver_studio/toolchain/risc-v embedded gcc/bin/../lib/gcc/riscv-none-embed/8.2.0/../../../../riscv-none-embed/lib/rv32imacxw/ilp32\libg_nano.a(lib_a-makebuf.o)
 .bss           0x0000000000000000        0x0 d:/psx/rj/mounriver_studio/toolchain/risc-v embedded gcc/bin/../lib/gcc/riscv-none-embed/8.2.0/../../../../riscv-none-embed/lib/rv32imacxw/ilp32\libg_nano.a(lib_a-makebuf.o)
 .text          0x0000000000000000        0x0 d:/psx/rj/mounriver_studio/toolchain/risc-v embedded gcc/bin/../lib/gcc/riscv-none-embed/8.2.0/../../../../riscv-none-embed/lib/rv32imacxw/ilp32\libg_nano.a(lib_a-malloc.o)
 .data          0x0000000000000000        0x0 d:/psx/rj/mounriver_studio/toolchain/risc-v embedded gcc/bin/../lib/gcc/riscv-none-embed/8.2.0/../../../../riscv-none-embed/lib/rv32imacxw/ilp32\libg_nano.a(lib_a-malloc.o)
 .bss           0x0000000000000000        0x0 d:/psx/rj/mounriver_studio/toolchain/risc-v embedded gcc/bin/../lib/gcc/riscv-none-embed/8.2.0/../../../../riscv-none-embed/lib/rv32imacxw/ilp32\libg_nano.a(lib_a-malloc.o)
 .text.malloc   0x0000000000000000       0x14 d:/psx/rj/mounriver_studio/toolchain/risc-v embedded gcc/bin/../lib/gcc/riscv-none-embed/8.2.0/../../../../riscv-none-embed/lib/rv32imacxw/ilp32\libg_nano.a(lib_a-malloc.o)
 .text.free     0x0000000000000000       0x14 d:/psx/rj/mounriver_studio/toolchain/risc-v embedded gcc/bin/../lib/gcc/riscv-none-embed/8.2.0/../../../../riscv-none-embed/lib/rv32imacxw/ilp32\libg_nano.a(lib_a-malloc.o)
 .debug_frame   0x0000000000000000       0x30 d:/psx/rj/mounriver_studio/toolchain/risc-v embedded gcc/bin/../lib/gcc/riscv-none-embed/8.2.0/../../../../riscv-none-embed/lib/rv32imacxw/ilp32\libg_nano.a(lib_a-malloc.o)
 .text          0x0000000000000000        0x0 d:/psx/rj/mounriver_studio/toolchain/risc-v embedded gcc/bin/../lib/gcc/riscv-none-embed/8.2.0/../../../../riscv-none-embed/lib/rv32imacxw/ilp32\libg_nano.a(lib_a-nano-freer.o)
 .data          0x0000000000000000        0x0 d:/psx/rj/mounriver_studio/toolchain/risc-v embedded gcc/bin/../lib/gcc/riscv-none-embed/8.2.0/../../../../riscv-none-embed/lib/rv32imacxw/ilp32\libg_nano.a(lib_a-nano-freer.o)
 .bss           0x0000000000000000        0x0 d:/psx/rj/mounriver_studio/toolchain/risc-v embedded gcc/bin/../lib/gcc/riscv-none-embed/8.2.0/../../../../riscv-none-embed/lib/rv32imacxw/ilp32\libg_nano.a(lib_a-nano-freer.o)
 .text          0x0000000000000000        0x0 d:/psx/rj/mounriver_studio/toolchain/risc-v embedded gcc/bin/../lib/gcc/riscv-none-embed/8.2.0/../../../../riscv-none-embed/lib/rv32imacxw/ilp32\libg_nano.a(lib_a-nano-mallocr.o)
 .data          0x0000000000000000        0x0 d:/psx/rj/mounriver_studio/toolchain/risc-v embedded gcc/bin/../lib/gcc/riscv-none-embed/8.2.0/../../../../riscv-none-embed/lib/rv32imacxw/ilp32\libg_nano.a(lib_a-nano-mallocr.o)
 .bss           0x0000000000000000        0x0 d:/psx/rj/mounriver_studio/toolchain/risc-v embedded gcc/bin/../lib/gcc/riscv-none-embed/8.2.0/../../../../riscv-none-embed/lib/rv32imacxw/ilp32\libg_nano.a(lib_a-nano-mallocr.o)
 .text          0x0000000000000000        0x0 d:/psx/rj/mounriver_studio/toolchain/risc-v embedded gcc/bin/../lib/gcc/riscv-none-embed/8.2.0/../../../../riscv-none-embed/lib/rv32imacxw/ilp32\libg_nano.a(lib_a-nano-vfprintf.o)
 .data          0x0000000000000000        0x0 d:/psx/rj/mounriver_studio/toolchain/risc-v embedded gcc/bin/../lib/gcc/riscv-none-embed/8.2.0/../../../../riscv-none-embed/lib/rv32imacxw/ilp32\libg_nano.a(lib_a-nano-vfprintf.o)
 .bss           0x0000000000000000        0x0 d:/psx/rj/mounriver_studio/toolchain/risc-v embedded gcc/bin/../lib/gcc/riscv-none-embed/8.2.0/../../../../riscv-none-embed/lib/rv32imacxw/ilp32\libg_nano.a(lib_a-nano-vfprintf.o)
 .text.__sprint_r
                0x0000000000000000       0x2c d:/psx/rj/mounriver_studio/toolchain/risc-v embedded gcc/bin/../lib/gcc/riscv-none-embed/8.2.0/../../../../riscv-none-embed/lib/rv32imacxw/ilp32\libg_nano.a(lib_a-nano-vfprintf.o)
 .text.vfprintf
                0x0000000000000000       0x18 d:/psx/rj/mounriver_studio/toolchain/risc-v embedded gcc/bin/../lib/gcc/riscv-none-embed/8.2.0/../../../../riscv-none-embed/lib/rv32imacxw/ilp32\libg_nano.a(lib_a-nano-vfprintf.o)
 .text          0x0000000000000000        0x0 d:/psx/rj/mounriver_studio/toolchain/risc-v embedded gcc/bin/../lib/gcc/riscv-none-embed/8.2.0/../../../../riscv-none-embed/lib/rv32imacxw/ilp32\libg_nano.a(lib_a-nano-vfprintf_i.o)
 .data          0x0000000000000000        0x0 d:/psx/rj/mounriver_studio/toolchain/risc-v embedded gcc/bin/../lib/gcc/riscv-none-embed/8.2.0/../../../../riscv-none-embed/lib/rv32imacxw/ilp32\libg_nano.a(lib_a-nano-vfprintf_i.o)
 .bss           0x0000000000000000        0x0 d:/psx/rj/mounriver_studio/toolchain/risc-v embedded gcc/bin/../lib/gcc/riscv-none-embed/8.2.0/../../../../riscv-none-embed/lib/rv32imacxw/ilp32\libg_nano.a(lib_a-nano-vfprintf_i.o)
 .text          0x0000000000000000        0x0 d:/psx/rj/mounriver_studio/toolchain/risc-v embedded gcc/bin/../lib/gcc/riscv-none-embed/8.2.0/../../../../riscv-none-embed/lib/rv32imacxw/ilp32\libg_nano.a(lib_a-putc.o)
 .data          0x0000000000000000        0x0 d:/psx/rj/mounriver_studio/toolchain/risc-v embedded gcc/bin/../lib/gcc/riscv-none-embed/8.2.0/../../../../riscv-none-embed/lib/rv32imacxw/ilp32\libg_nano.a(lib_a-putc.o)
 .bss           0x0000000000000000        0x0 d:/psx/rj/mounriver_studio/toolchain/risc-v embedded gcc/bin/../lib/gcc/riscv-none-embed/8.2.0/../../../../riscv-none-embed/lib/rv32imacxw/ilp32\libg_nano.a(lib_a-putc.o)
 .text._putc_r  0x0000000000000000       0x8c d:/psx/rj/mounriver_studio/toolchain/risc-v embedded gcc/bin/../lib/gcc/riscv-none-embed/8.2.0/../../../../riscv-none-embed/lib/rv32imacxw/ilp32\libg_nano.a(lib_a-putc.o)
 .text.putc     0x0000000000000000       0x16 d:/psx/rj/mounriver_studio/toolchain/risc-v embedded gcc/bin/../lib/gcc/riscv-none-embed/8.2.0/../../../../riscv-none-embed/lib/rv32imacxw/ilp32\libg_nano.a(lib_a-putc.o)
 .debug_frame   0x0000000000000000       0x4c d:/psx/rj/mounriver_studio/toolchain/risc-v embedded gcc/bin/../lib/gcc/riscv-none-embed/8.2.0/../../../../riscv-none-embed/lib/rv32imacxw/ilp32\libg_nano.a(lib_a-putc.o)
 .text          0x0000000000000000        0x0 d:/psx/rj/mounriver_studio/toolchain/risc-v embedded gcc/bin/../lib/gcc/riscv-none-embed/8.2.0/../../../../riscv-none-embed/lib/rv32imacxw/ilp32\libg_nano.a(lib_a-sbrkr.o)
 .data          0x0000000000000000        0x0 d:/psx/rj/mounriver_studio/toolchain/risc-v embedded gcc/bin/../lib/gcc/riscv-none-embed/8.2.0/../../../../riscv-none-embed/lib/rv32imacxw/ilp32\libg_nano.a(lib_a-sbrkr.o)
 .bss           0x0000000000000000        0x0 d:/psx/rj/mounriver_studio/toolchain/risc-v embedded gcc/bin/../lib/gcc/riscv-none-embed/8.2.0/../../../../riscv-none-embed/lib/rv32imacxw/ilp32\libg_nano.a(lib_a-sbrkr.o)
 .text          0x0000000000000000        0x0 d:/psx/rj/mounriver_studio/toolchain/risc-v embedded gcc/bin/../lib/gcc/riscv-none-embed/8.2.0/../../../../riscv-none-embed/lib/rv32imacxw/ilp32\libg_nano.a(lib_a-stdio.o)
 .data          0x0000000000000000        0x0 d:/psx/rj/mounriver_studio/toolchain/risc-v embedded gcc/bin/../lib/gcc/riscv-none-embed/8.2.0/../../../../riscv-none-embed/lib/rv32imacxw/ilp32\libg_nano.a(lib_a-stdio.o)
 .bss           0x0000000000000000        0x0 d:/psx/rj/mounriver_studio/toolchain/risc-v embedded gcc/bin/../lib/gcc/riscv-none-embed/8.2.0/../../../../riscv-none-embed/lib/rv32imacxw/ilp32\libg_nano.a(lib_a-stdio.o)
 .text.__seofread
                0x0000000000000000        0x4 d:/psx/rj/mounriver_studio/toolchain/risc-v embedded gcc/bin/../lib/gcc/riscv-none-embed/8.2.0/../../../../riscv-none-embed/lib/rv32imacxw/ilp32\libg_nano.a(lib_a-stdio.o)
 .text          0x0000000000000000        0x0 d:/psx/rj/mounriver_studio/toolchain/risc-v embedded gcc/bin/../lib/gcc/riscv-none-embed/8.2.0/../../../../riscv-none-embed/lib/rv32imacxw/ilp32\libg_nano.a(lib_a-writer.o)
 .data          0x0000000000000000        0x0 d:/psx/rj/mounriver_studio/toolchain/risc-v embedded gcc/bin/../lib/gcc/riscv-none-embed/8.2.0/../../../../riscv-none-embed/lib/rv32imacxw/ilp32\libg_nano.a(lib_a-writer.o)
 .bss           0x0000000000000000        0x0 d:/psx/rj/mounriver_studio/toolchain/risc-v embedded gcc/bin/../lib/gcc/riscv-none-embed/8.2.0/../../../../riscv-none-embed/lib/rv32imacxw/ilp32\libg_nano.a(lib_a-writer.o)
 .text          0x0000000000000000        0x0 d:/psx/rj/mounriver_studio/toolchain/risc-v embedded gcc/bin/../lib/gcc/riscv-none-embed/8.2.0/../../../../riscv-none-embed/lib/rv32imacxw/ilp32\libg_nano.a(lib_a-closer.o)
 .data          0x0000000000000000        0x0 d:/psx/rj/mounriver_studio/toolchain/risc-v embedded gcc/bin/../lib/gcc/riscv-none-embed/8.2.0/../../../../riscv-none-embed/lib/rv32imacxw/ilp32\libg_nano.a(lib_a-closer.o)
 .bss           0x0000000000000000        0x0 d:/psx/rj/mounriver_studio/toolchain/risc-v embedded gcc/bin/../lib/gcc/riscv-none-embed/8.2.0/../../../../riscv-none-embed/lib/rv32imacxw/ilp32\libg_nano.a(lib_a-closer.o)
 .text          0x0000000000000000        0x0 d:/psx/rj/mounriver_studio/toolchain/risc-v embedded gcc/bin/../lib/gcc/riscv-none-embed/8.2.0/../../../../riscv-none-embed/lib/rv32imacxw/ilp32\libg_nano.a(lib_a-fstatr.o)
 .data          0x0000000000000000        0x0 d:/psx/rj/mounriver_studio/toolchain/risc-v embedded gcc/bin/../lib/gcc/riscv-none-embed/8.2.0/../../../../riscv-none-embed/lib/rv32imacxw/ilp32\libg_nano.a(lib_a-fstatr.o)
 .bss           0x0000000000000000        0x0 d:/psx/rj/mounriver_studio/toolchain/risc-v embedded gcc/bin/../lib/gcc/riscv-none-embed/8.2.0/../../../../riscv-none-embed/lib/rv32imacxw/ilp32\libg_nano.a(lib_a-fstatr.o)
 .text          0x0000000000000000        0x0 d:/psx/rj/mounriver_studio/toolchain/risc-v embedded gcc/bin/../lib/gcc/riscv-none-embed/8.2.0/../../../../riscv-none-embed/lib/rv32imacxw/ilp32\libg_nano.a(lib_a-fvwrite.o)
 .data          0x0000000000000000        0x0 d:/psx/rj/mounriver_studio/toolchain/risc-v embedded gcc/bin/../lib/gcc/riscv-none-embed/8.2.0/../../../../riscv-none-embed/lib/rv32imacxw/ilp32\libg_nano.a(lib_a-fvwrite.o)
 .bss           0x0000000000000000        0x0 d:/psx/rj/mounriver_studio/toolchain/risc-v embedded gcc/bin/../lib/gcc/riscv-none-embed/8.2.0/../../../../riscv-none-embed/lib/rv32imacxw/ilp32\libg_nano.a(lib_a-fvwrite.o)
 .text.__sfvwrite_r
                0x0000000000000000      0x306 d:/psx/rj/mounriver_studio/toolchain/risc-v embedded gcc/bin/../lib/gcc/riscv-none-embed/8.2.0/../../../../riscv-none-embed/lib/rv32imacxw/ilp32\libg_nano.a(lib_a-fvwrite.o)
 .debug_frame   0x0000000000000000       0x60 d:/psx/rj/mounriver_studio/toolchain/risc-v embedded gcc/bin/../lib/gcc/riscv-none-embed/8.2.0/../../../../riscv-none-embed/lib/rv32imacxw/ilp32\libg_nano.a(lib_a-fvwrite.o)
 .text          0x0000000000000000        0x0 d:/psx/rj/mounriver_studio/toolchain/risc-v embedded gcc/bin/../lib/gcc/riscv-none-embed/8.2.0/../../../../riscv-none-embed/lib/rv32imacxw/ilp32\libg_nano.a(lib_a-isattyr.o)
 .data          0x0000000000000000        0x0 d:/psx/rj/mounriver_studio/toolchain/risc-v embedded gcc/bin/../lib/gcc/riscv-none-embed/8.2.0/../../../../riscv-none-embed/lib/rv32imacxw/ilp32\libg_nano.a(lib_a-isattyr.o)
 .bss           0x0000000000000000        0x0 d:/psx/rj/mounriver_studio/toolchain/risc-v embedded gcc/bin/../lib/gcc/riscv-none-embed/8.2.0/../../../../riscv-none-embed/lib/rv32imacxw/ilp32\libg_nano.a(lib_a-isattyr.o)
 .text          0x0000000000000000        0x0 d:/psx/rj/mounriver_studio/toolchain/risc-v embedded gcc/bin/../lib/gcc/riscv-none-embed/8.2.0/../../../../riscv-none-embed/lib/rv32imacxw/ilp32\libg_nano.a(lib_a-lseekr.o)
 .data          0x0000000000000000        0x0 d:/psx/rj/mounriver_studio/toolchain/risc-v embedded gcc/bin/../lib/gcc/riscv-none-embed/8.2.0/../../../../riscv-none-embed/lib/rv32imacxw/ilp32\libg_nano.a(lib_a-lseekr.o)
 .bss           0x0000000000000000        0x0 d:/psx/rj/mounriver_studio/toolchain/risc-v embedded gcc/bin/../lib/gcc/riscv-none-embed/8.2.0/../../../../riscv-none-embed/lib/rv32imacxw/ilp32\libg_nano.a(lib_a-lseekr.o)
 .text          0x0000000000000000        0x0 d:/psx/rj/mounriver_studio/toolchain/risc-v embedded gcc/bin/../lib/gcc/riscv-none-embed/8.2.0/../../../../riscv-none-embed/lib/rv32imacxw/ilp32\libg_nano.a(lib_a-memchr.o)
 .data          0x0000000000000000        0x0 d:/psx/rj/mounriver_studio/toolchain/risc-v embedded gcc/bin/../lib/gcc/riscv-none-embed/8.2.0/../../../../riscv-none-embed/lib/rv32imacxw/ilp32\libg_nano.a(lib_a-memchr.o)
 .bss           0x0000000000000000        0x0 d:/psx/rj/mounriver_studio/toolchain/risc-v embedded gcc/bin/../lib/gcc/riscv-none-embed/8.2.0/../../../../riscv-none-embed/lib/rv32imacxw/ilp32\libg_nano.a(lib_a-memchr.o)
 .text          0x0000000000000000        0x0 d:/psx/rj/mounriver_studio/toolchain/risc-v embedded gcc/bin/../lib/gcc/riscv-none-embed/8.2.0/../../../../riscv-none-embed/lib/rv32imacxw/ilp32\libg_nano.a(lib_a-memmove.o)
 .data          0x0000000000000000        0x0 d:/psx/rj/mounriver_studio/toolchain/risc-v embedded gcc/bin/../lib/gcc/riscv-none-embed/8.2.0/../../../../riscv-none-embed/lib/rv32imacxw/ilp32\libg_nano.a(lib_a-memmove.o)
 .bss           0x0000000000000000        0x0 d:/psx/rj/mounriver_studio/toolchain/risc-v embedded gcc/bin/../lib/gcc/riscv-none-embed/8.2.0/../../../../riscv-none-embed/lib/rv32imacxw/ilp32\libg_nano.a(lib_a-memmove.o)
 .text.memmove  0x0000000000000000       0x46 d:/psx/rj/mounriver_studio/toolchain/risc-v embedded gcc/bin/../lib/gcc/riscv-none-embed/8.2.0/../../../../riscv-none-embed/lib/rv32imacxw/ilp32\libg_nano.a(lib_a-memmove.o)
 .debug_frame   0x0000000000000000       0x20 d:/psx/rj/mounriver_studio/toolchain/risc-v embedded gcc/bin/../lib/gcc/riscv-none-embed/8.2.0/../../../../riscv-none-embed/lib/rv32imacxw/ilp32\libg_nano.a(lib_a-memmove.o)
 .text          0x0000000000000000        0x0 d:/psx/rj/mounriver_studio/toolchain/risc-v embedded gcc/bin/../lib/gcc/riscv-none-embed/8.2.0/../../../../riscv-none-embed/lib/rv32imacxw/ilp32\libg_nano.a(lib_a-mlock.o)
 .data          0x0000000000000000        0x0 d:/psx/rj/mounriver_studio/toolchain/risc-v embedded gcc/bin/../lib/gcc/riscv-none-embed/8.2.0/../../../../riscv-none-embed/lib/rv32imacxw/ilp32\libg_nano.a(lib_a-mlock.o)
 .bss           0x0000000000000000        0x0 d:/psx/rj/mounriver_studio/toolchain/risc-v embedded gcc/bin/../lib/gcc/riscv-none-embed/8.2.0/../../../../riscv-none-embed/lib/rv32imacxw/ilp32\libg_nano.a(lib_a-mlock.o)
 .text          0x0000000000000000        0x0 d:/psx/rj/mounriver_studio/toolchain/risc-v embedded gcc/bin/../lib/gcc/riscv-none-embed/8.2.0/../../../../riscv-none-embed/lib/rv32imacxw/ilp32\libg_nano.a(lib_a-nano-reallocr.o)
 .data          0x0000000000000000        0x0 d:/psx/rj/mounriver_studio/toolchain/risc-v embedded gcc/bin/../lib/gcc/riscv-none-embed/8.2.0/../../../../riscv-none-embed/lib/rv32imacxw/ilp32\libg_nano.a(lib_a-nano-reallocr.o)
 .bss           0x0000000000000000        0x0 d:/psx/rj/mounriver_studio/toolchain/risc-v embedded gcc/bin/../lib/gcc/riscv-none-embed/8.2.0/../../../../riscv-none-embed/lib/rv32imacxw/ilp32\libg_nano.a(lib_a-nano-reallocr.o)
 .text._realloc_r
                0x0000000000000000       0x72 d:/psx/rj/mounriver_studio/toolchain/risc-v embedded gcc/bin/../lib/gcc/riscv-none-embed/8.2.0/../../../../riscv-none-embed/lib/rv32imacxw/ilp32\libg_nano.a(lib_a-nano-reallocr.o)
 .debug_frame   0x0000000000000000       0x40 d:/psx/rj/mounriver_studio/toolchain/risc-v embedded gcc/bin/../lib/gcc/riscv-none-embed/8.2.0/../../../../riscv-none-embed/lib/rv32imacxw/ilp32\libg_nano.a(lib_a-nano-reallocr.o)
 .text          0x0000000000000000        0x0 d:/psx/rj/mounriver_studio/toolchain/risc-v embedded gcc/bin/../lib/gcc/riscv-none-embed/8.2.0/../../../../riscv-none-embed/lib/rv32imacxw/ilp32\libg_nano.a(lib_a-readr.o)
 .data          0x0000000000000000        0x0 d:/psx/rj/mounriver_studio/toolchain/risc-v embedded gcc/bin/../lib/gcc/riscv-none-embed/8.2.0/../../../../riscv-none-embed/lib/rv32imacxw/ilp32\libg_nano.a(lib_a-readr.o)
 .bss           0x0000000000000000        0x0 d:/psx/rj/mounriver_studio/toolchain/risc-v embedded gcc/bin/../lib/gcc/riscv-none-embed/8.2.0/../../../../riscv-none-embed/lib/rv32imacxw/ilp32\libg_nano.a(lib_a-readr.o)
 .text          0x0000000000000000        0x0 d:/psx/rj/mounriver_studio/toolchain/risc-v embedded gcc/bin/../lib/gcc/riscv-none-embed/8.2.0/../../../../riscv-none-embed/lib/rv32imacxw/ilp32\libg_nano.a(lib_a-reent.o)
 .data          0x0000000000000000        0x0 d:/psx/rj/mounriver_studio/toolchain/risc-v embedded gcc/bin/../lib/gcc/riscv-none-embed/8.2.0/../../../../riscv-none-embed/lib/rv32imacxw/ilp32\libg_nano.a(lib_a-reent.o)
 .bss           0x0000000000000000        0x0 d:/psx/rj/mounriver_studio/toolchain/risc-v embedded gcc/bin/../lib/gcc/riscv-none-embed/8.2.0/../../../../riscv-none-embed/lib/rv32imacxw/ilp32\libg_nano.a(lib_a-reent.o)
 .text.cleanup_glue
                0x0000000000000000       0x2c d:/psx/rj/mounriver_studio/toolchain/risc-v embedded gcc/bin/../lib/gcc/riscv-none-embed/8.2.0/../../../../riscv-none-embed/lib/rv32imacxw/ilp32\libg_nano.a(lib_a-reent.o)
 .text._reclaim_reent
                0x0000000000000000      0x10c d:/psx/rj/mounriver_studio/toolchain/risc-v embedded gcc/bin/../lib/gcc/riscv-none-embed/8.2.0/../../../../riscv-none-embed/lib/rv32imacxw/ilp32\libg_nano.a(lib_a-reent.o)
 .text          0x0000000000000000        0x0 d:/psx/rj/mounriver_studio/toolchain/risc-v embedded gcc/bin/../lib/gcc/riscv-none-embed/8.2.0/../../../../riscv-none-embed/lib/rv32imacxw/ilp32\libg_nano.a(lib_a-nano-msizer.o)
 .data          0x0000000000000000        0x0 d:/psx/rj/mounriver_studio/toolchain/risc-v embedded gcc/bin/../lib/gcc/riscv-none-embed/8.2.0/../../../../riscv-none-embed/lib/rv32imacxw/ilp32\libg_nano.a(lib_a-nano-msizer.o)
 .bss           0x0000000000000000        0x0 d:/psx/rj/mounriver_studio/toolchain/risc-v embedded gcc/bin/../lib/gcc/riscv-none-embed/8.2.0/../../../../riscv-none-embed/lib/rv32imacxw/ilp32\libg_nano.a(lib_a-nano-msizer.o)
 .text._malloc_usable_size_r
                0x0000000000000000       0x14 d:/psx/rj/mounriver_studio/toolchain/risc-v embedded gcc/bin/../lib/gcc/riscv-none-embed/8.2.0/../../../../riscv-none-embed/lib/rv32imacxw/ilp32\libg_nano.a(lib_a-nano-msizer.o)
 .debug_frame   0x0000000000000000       0x20 d:/psx/rj/mounriver_studio/toolchain/risc-v embedded gcc/bin/../lib/gcc/riscv-none-embed/8.2.0/../../../../riscv-none-embed/lib/rv32imacxw/ilp32\libg_nano.a(lib_a-nano-msizer.o)
 .text          0x0000000000000000        0x0 d:/psx/rj/mounriver_studio/toolchain/risc-v embedded gcc/bin/../lib/gcc/riscv-none-embed/8.2.0/../../../../riscv-none-embed/lib/rv32imacxw/ilp32\libnosys.a(close.o)
 .data          0x0000000000000000        0x0 d:/psx/rj/mounriver_studio/toolchain/risc-v embedded gcc/bin/../lib/gcc/riscv-none-embed/8.2.0/../../../../riscv-none-embed/lib/rv32imacxw/ilp32\libnosys.a(close.o)
 .bss           0x0000000000000000        0x0 d:/psx/rj/mounriver_studio/toolchain/risc-v embedded gcc/bin/../lib/gcc/riscv-none-embed/8.2.0/../../../../riscv-none-embed/lib/rv32imacxw/ilp32\libnosys.a(close.o)
 .text          0x0000000000000000        0x0 d:/psx/rj/mounriver_studio/toolchain/risc-v embedded gcc/bin/../lib/gcc/riscv-none-embed/8.2.0/../../../../riscv-none-embed/lib/rv32imacxw/ilp32\libnosys.a(fstat.o)
 .data          0x0000000000000000        0x0 d:/psx/rj/mounriver_studio/toolchain/risc-v embedded gcc/bin/../lib/gcc/riscv-none-embed/8.2.0/../../../../riscv-none-embed/lib/rv32imacxw/ilp32\libnosys.a(fstat.o)
 .bss           0x0000000000000000        0x0 d:/psx/rj/mounriver_studio/toolchain/risc-v embedded gcc/bin/../lib/gcc/riscv-none-embed/8.2.0/../../../../riscv-none-embed/lib/rv32imacxw/ilp32\libnosys.a(fstat.o)
 .text          0x0000000000000000        0x0 d:/psx/rj/mounriver_studio/toolchain/risc-v embedded gcc/bin/../lib/gcc/riscv-none-embed/8.2.0/../../../../riscv-none-embed/lib/rv32imacxw/ilp32\libnosys.a(isatty.o)
 .data          0x0000000000000000        0x0 d:/psx/rj/mounriver_studio/toolchain/risc-v embedded gcc/bin/../lib/gcc/riscv-none-embed/8.2.0/../../../../riscv-none-embed/lib/rv32imacxw/ilp32\libnosys.a(isatty.o)
 .bss           0x0000000000000000        0x0 d:/psx/rj/mounriver_studio/toolchain/risc-v embedded gcc/bin/../lib/gcc/riscv-none-embed/8.2.0/../../../../riscv-none-embed/lib/rv32imacxw/ilp32\libnosys.a(isatty.o)
 .text          0x0000000000000000        0x0 d:/psx/rj/mounriver_studio/toolchain/risc-v embedded gcc/bin/../lib/gcc/riscv-none-embed/8.2.0/../../../../riscv-none-embed/lib/rv32imacxw/ilp32\libnosys.a(lseek.o)
 .data          0x0000000000000000        0x0 d:/psx/rj/mounriver_studio/toolchain/risc-v embedded gcc/bin/../lib/gcc/riscv-none-embed/8.2.0/../../../../riscv-none-embed/lib/rv32imacxw/ilp32\libnosys.a(lseek.o)
 .bss           0x0000000000000000        0x0 d:/psx/rj/mounriver_studio/toolchain/risc-v embedded gcc/bin/../lib/gcc/riscv-none-embed/8.2.0/../../../../riscv-none-embed/lib/rv32imacxw/ilp32\libnosys.a(lseek.o)
 .text          0x0000000000000000        0x0 d:/psx/rj/mounriver_studio/toolchain/risc-v embedded gcc/bin/../lib/gcc/riscv-none-embed/8.2.0/../../../../riscv-none-embed/lib/rv32imacxw/ilp32\libnosys.a(read.o)
 .data          0x0000000000000000        0x0 d:/psx/rj/mounriver_studio/toolchain/risc-v embedded gcc/bin/../lib/gcc/riscv-none-embed/8.2.0/../../../../riscv-none-embed/lib/rv32imacxw/ilp32\libnosys.a(read.o)
 .bss           0x0000000000000000        0x0 d:/psx/rj/mounriver_studio/toolchain/risc-v embedded gcc/bin/../lib/gcc/riscv-none-embed/8.2.0/../../../../riscv-none-embed/lib/rv32imacxw/ilp32\libnosys.a(read.o)

Memory Configuration

Name             Origin             Length             Attributes
FLASH            0x0000000000000000 0x0000000000010000 xr
RAM              0x0000000020000000 0x0000000000005000 xrw
*default*        0x0000000000000000 0xffffffffffffffff

Linker script and memory map

LOAD ./User/ch32l103_it.o
LOAD ./User/main.o
LOAD ./User/system_ch32l103.o
LOAD ./Startup/startup_ch32l103.o
LOAD ./Peripheral/src/ch32l103_adc.o
LOAD ./Peripheral/src/ch32l103_bkp.o
LOAD ./Peripheral/src/ch32l103_can.o
LOAD ./Peripheral/src/ch32l103_crc.o
LOAD ./Peripheral/src/ch32l103_dbgmcu.o
LOAD ./Peripheral/src/ch32l103_dma.o
LOAD ./Peripheral/src/ch32l103_exti.o
LOAD ./Peripheral/src/ch32l103_flash.o
LOAD ./Peripheral/src/ch32l103_gpio.o
LOAD ./Peripheral/src/ch32l103_i2c.o
LOAD ./Peripheral/src/ch32l103_iwdg.o
LOAD ./Peripheral/src/ch32l103_lptim.o
LOAD ./Peripheral/src/ch32l103_misc.o
LOAD ./Peripheral/src/ch32l103_opa.o
LOAD ./Peripheral/src/ch32l103_pwr.o
LOAD ./Peripheral/src/ch32l103_rcc.o
LOAD ./Peripheral/src/ch32l103_rtc.o
LOAD ./Peripheral/src/ch32l103_spi.o
LOAD ./Peripheral/src/ch32l103_tim.o
LOAD ./Peripheral/src/ch32l103_usart.o
LOAD ./Peripheral/src/ch32l103_wwdg.o
LOAD ./Hardware/src/adc.o
LOAD ./Hardware/src/flash.o
LOAD ./Hardware/src/gpio.o
LOAD ./Hardware/src/pwm.o
LOAD ./Hardware/src/rs485.o
LOAD ./Hardware/src/tim.o
LOAD ./Drivers/TimeSliceOffset/timeSliceOffset.o
LOAD ./Drivers/RingQueue/ring_queue.o
LOAD ./Debug/debug.o
LOAD ./Core/core_riscv.o
LOAD ./App/src/collect_Conversion.o
LOAD ./App/src/inflash.o
LOAD ./App/src/mppt_control.o
LOAD ./App/src/sl_protocol.o
LOAD ./App/src/task.o
LOAD ./App/src/uart_dev.o
LOAD d:/psx/rj/mounriver_studio/toolchain/risc-v embedded gcc/bin/../lib/gcc/riscv-none-embed/8.2.0/../../../../riscv-none-embed/lib/rv32imacxw/ilp32\libm.a
LOAD d:/psx/rj/mounriver_studio/toolchain/risc-v embedded gcc/bin/../lib/gcc/riscv-none-embed/8.2.0/rv32imacxw/ilp32\libgcc.a
LOAD d:/psx/rj/mounriver_studio/toolchain/risc-v embedded gcc/bin/../lib/gcc/riscv-none-embed/8.2.0/../../../../riscv-none-embed/lib/rv32imacxw/ilp32\libg_nano.a
LOAD d:/psx/rj/mounriver_studio/toolchain/risc-v embedded gcc/bin/../lib/gcc/riscv-none-embed/8.2.0/../../../../riscv-none-embed/lib/rv32imacxw/ilp32\libc_nano.a
LOAD d:/psx/rj/mounriver_studio/toolchain/risc-v embedded gcc/bin/../lib/gcc/riscv-none-embed/8.2.0/rv32imacxw/ilp32\libgcc.a
START GROUP
LOAD d:/psx/rj/mounriver_studio/toolchain/risc-v embedded gcc/bin/../lib/gcc/riscv-none-embed/8.2.0/rv32imacxw/ilp32\libgcc.a
LOAD d:/psx/rj/mounriver_studio/toolchain/risc-v embedded gcc/bin/../lib/gcc/riscv-none-embed/8.2.0/../../../../riscv-none-embed/lib/rv32imacxw/ilp32\libc_nano.a
LOAD d:/psx/rj/mounriver_studio/toolchain/risc-v embedded gcc/bin/../lib/gcc/riscv-none-embed/8.2.0/../../../../riscv-none-embed/lib/rv32imacxw/ilp32\libnosys.a
END GROUP
START GROUP
LOAD d:/psx/rj/mounriver_studio/toolchain/risc-v embedded gcc/bin/../lib/gcc/riscv-none-embed/8.2.0/rv32imacxw/ilp32\libgcc.a
LOAD d:/psx/rj/mounriver_studio/toolchain/risc-v embedded gcc/bin/../lib/gcc/riscv-none-embed/8.2.0/../../../../riscv-none-embed/lib/rv32imacxw/ilp32\libc_nano.a
LOAD d:/psx/rj/mounriver_studio/toolchain/risc-v embedded gcc/bin/../lib/gcc/riscv-none-embed/8.2.0/../../../../riscv-none-embed/lib/rv32imacxw/ilp32\libnosys.a
END GROUP
                0x0000000000000800                __stack_size = 0x800
                [!provide]                        PROVIDE (_stack_size = __stack_size)

.init           0x0000000000000000        0x4
                0x0000000000000000                _sinit = .
                0x0000000000000000                . = ALIGN (0x4)
 *(SORT_NONE(.init))
 .init          0x0000000000000000        0x4 ./Startup/startup_ch32l103.o
                0x0000000000000000                _start
                0x0000000000000004                . = ALIGN (0x4)
                0x0000000000000004                _einit = .

.vector         0x0000000000000004      0x13c
 *(.vector)
 .vector        0x0000000000000004      0x114 ./Startup/startup_ch32l103.o
                0x0000000000000140                . = ALIGN (0x40)
 *fill*         0x0000000000000118       0x28 

.text           0x0000000000000140     0x5aac
                0x0000000000000140                . = ALIGN (0x4)
 *(.text)
 .text          0x0000000000000140       0x60 d:/psx/rj/mounriver_studio/toolchain/risc-v embedded gcc/bin/../lib/gcc/riscv-none-embed/8.2.0/rv32imacxw/ilp32\libgcc.a(save-restore.o)
                0x0000000000000140                __riscv_save_12
                0x0000000000000148                __riscv_save_9
                0x0000000000000148                __riscv_save_11
                0x0000000000000148                __riscv_save_10
                0x0000000000000148                __riscv_save_8
                0x0000000000000156                __riscv_save_4
                0x0000000000000156                __riscv_save_6
                0x0000000000000156                __riscv_save_5
                0x0000000000000156                __riscv_save_7
                0x0000000000000170                __riscv_save_3
                0x0000000000000170                __riscv_save_2
                0x0000000000000170                __riscv_save_1
                0x0000000000000170                __riscv_save_0
                0x000000000000017c                __riscv_restore_12
                0x0000000000000180                __riscv_restore_11
                0x0000000000000180                __riscv_restore_9
                0x0000000000000180                __riscv_restore_10
                0x0000000000000180                __riscv_restore_8
                0x000000000000018a                __riscv_restore_5
                0x000000000000018a                __riscv_restore_7
                0x000000000000018a                __riscv_restore_6
                0x000000000000018a                __riscv_restore_4
                0x0000000000000194                __riscv_restore_3
                0x0000000000000194                __riscv_restore_0
                0x0000000000000194                __riscv_restore_2
                0x0000000000000194                __riscv_restore_1
 .text          0x00000000000001a0       0xa8 d:/psx/rj/mounriver_studio/toolchain/risc-v embedded gcc/bin/../lib/gcc/riscv-none-embed/8.2.0/../../../../riscv-none-embed/lib/rv32imacxw/ilp32\libg_nano.a(lib_a-memset.o)
                0x00000000000001a0                memset
 *(.text.*)
 .text.NMI_Handler
                0x0000000000000248        0x2 ./User/ch32l103_it.o
                0x0000000000000248                NMI_Handler
 .text.HardFault_Handler
                0x000000000000024a        0x2 ./User/ch32l103_it.o
                0x000000000000024a                HardFault_Handler
 .text.startup.main
                0x000000000000024c       0x4a ./User/main.o
                0x000000000000024c                main
 .text.SystemInit
                0x0000000000000296      0x106 ./User/system_ch32l103.o
                0x0000000000000296                SystemInit
 .text.SystemCoreClockUpdate
                0x000000000000039c       0xa4 ./User/system_ch32l103.o
                0x000000000000039c                SystemCoreClockUpdate
 .text.vector_handler
                0x0000000000000440        0x2 ./Startup/startup_ch32l103.o
                0x0000000000000440                TIM1_CC_IRQHandler
                0x0000000000000440                USBPD_IRQHandler
                0x0000000000000440                PVD_IRQHandler
                0x0000000000000440                EXTI3_IRQHandler
                0x0000000000000440                USBFS_IRQHandler
                0x0000000000000440                EXTI0_IRQHandler
                0x0000000000000440                I2C2_EV_IRQHandler
                0x0000000000000440                LPTIM_IRQHandler
                0x0000000000000440                Break_Point_Handler
                0x0000000000000440                SPI1_IRQHandler
                0x0000000000000440                TAMPER_IRQHandler
                0x0000000000000440                Ecall_M_Mode_Handler
                0x0000000000000440                DMA1_Channel4_IRQHandler
                0x0000000000000440                RTC_IRQHandler
                0x0000000000000440                DMA1_Channel7_IRQHandler
                0x0000000000000440                CAN1_RX1_IRQHandler
                0x0000000000000440                USBPDWakeUp_IRQHandler
                0x0000000000000440                TIM4_IRQHandler
                0x0000000000000440                I2C1_EV_IRQHandler
                0x0000000000000440                DMA1_Channel6_IRQHandler
                0x0000000000000440                RCC_IRQHandler
                0x0000000000000440                TIM1_TRG_COM_IRQHandler
                0x0000000000000440                ADC_IRQHandler
                0x0000000000000440                DMA1_Channel8_IRQHandler
                0x0000000000000440                EXTI9_5_IRQHandler
                0x0000000000000440                SPI2_IRQHandler
                0x0000000000000440                DMA1_Channel5_IRQHandler
                0x0000000000000440                EXTI4_IRQHandler
                0x0000000000000440                USB_LP_CAN1_RX0_IRQHandler
                0x0000000000000440                USB_HP_CAN1_TX_IRQHandler
                0x0000000000000440                CMPWakeUp_IRQHandler
                0x0000000000000440                DMA1_Channel3_IRQHandler
                0x0000000000000440                LPTIMWakeUp_IRQHandler
                0x0000000000000440                WWDG_IRQHandler
                0x0000000000000440                Ecall_U_Mode_Handler
                0x0000000000000440                SW_Handler
                0x0000000000000440                TIM1_BRK_IRQHandler
                0x0000000000000440                OPA_IRQHandler
                0x0000000000000440                EXTI1_IRQHandler
                0x0000000000000440                RTCAlarm_IRQHandler
                0x0000000000000440                USART2_IRQHandler
                0x0000000000000440                I2C2_ER_IRQHandler
                0x0000000000000440                DMA1_Channel2_IRQHandler
                0x0000000000000440                CAN1_SCE_IRQHandler
                0x0000000000000440                FLASH_IRQHandler
                0x0000000000000440                USBFSWakeUp_IRQHandler
                0x0000000000000440                USART1_IRQHandler
                0x0000000000000440                I2C1_ER_IRQHandler
                0x0000000000000440                TKeyWakeUp_IRQHandler
 .text.handle_reset
                0x0000000000000442       0x86 ./Startup/startup_ch32l103.o
                0x0000000000000442                handle_reset
 .text.ADC_DeInit
                0x00000000000004c8       0x28 ./Peripheral/src/ch32l103_adc.o
                0x00000000000004c8                ADC_DeInit
 .text.ADC_Init
                0x00000000000004f0       0x56 ./Peripheral/src/ch32l103_adc.o
                0x00000000000004f0                ADC_Init
 .text.ADC_Cmd  0x0000000000000546       0x10 ./Peripheral/src/ch32l103_adc.o
                0x0000000000000546                ADC_Cmd
 .text.ADC_DMACmd
                0x0000000000000556       0x12 ./Peripheral/src/ch32l103_adc.o
                0x0000000000000556                ADC_DMACmd
 .text.ADC_ResetCalibration
                0x0000000000000568        0xa ./Peripheral/src/ch32l103_adc.o
                0x0000000000000568                ADC_ResetCalibration
 .text.ADC_GetResetCalibrationStatus
                0x0000000000000572        0x8 ./Peripheral/src/ch32l103_adc.o
                0x0000000000000572                ADC_GetResetCalibrationStatus
 .text.ADC_StartCalibration
                0x000000000000057a        0xa ./Peripheral/src/ch32l103_adc.o
                0x000000000000057a                ADC_StartCalibration
 .text.ADC_GetCalibrationStatus
                0x0000000000000584        0x8 ./Peripheral/src/ch32l103_adc.o
                0x0000000000000584                ADC_GetCalibrationStatus
 .text.ADC_SoftwareStartConvCmd
                0x000000000000058c       0x18 ./Peripheral/src/ch32l103_adc.o
                0x000000000000058c                ADC_SoftwareStartConvCmd
 .text.ADC_RegularChannelConfig
                0x00000000000005a4       0xb8 ./Peripheral/src/ch32l103_adc.o
                0x00000000000005a4                ADC_RegularChannelConfig
 .text.ADC_GetConversionValue
                0x000000000000065c        0x8 ./Peripheral/src/ch32l103_adc.o
                0x000000000000065c                ADC_GetConversionValue
 .text.ADC_GetFlagStatus
                0x0000000000000664        0xa ./Peripheral/src/ch32l103_adc.o
                0x0000000000000664                ADC_GetFlagStatus
 .text.ADC_BufferCmd
                0x000000000000066e       0x18 ./Peripheral/src/ch32l103_adc.o
                0x000000000000066e                ADC_BufferCmd
 .text.ADC_DutyDelayCmd
                0x0000000000000686       0x12 ./Peripheral/src/ch32l103_adc.o
                0x0000000000000686                ADC_DutyDelayCmd
 .text.ADC_FIFO_Cmd
                0x0000000000000698       0x12 ./Peripheral/src/ch32l103_adc.o
                0x0000000000000698                ADC_FIFO_Cmd
 .text.ADC_Sample_ModeConfig
                0x00000000000006aa       0x10 ./Peripheral/src/ch32l103_adc.o
                0x00000000000006aa                ADC_Sample_ModeConfig
 .text.Get_CalibrationValue
                0x00000000000006ba      0x1d4 ./Peripheral/src/ch32l103_adc.o
                0x00000000000006ba                Get_CalibrationValue
 .text.DBGMCU_GetCHIPID
                0x000000000000088e        0x6 ./Peripheral/src/ch32l103_dbgmcu.o
                0x000000000000088e                DBGMCU_GetCHIPID
 .text.DMA_DeInit
                0x0000000000000894       0xa2 ./Peripheral/src/ch32l103_dma.o
                0x0000000000000894                DMA_DeInit
 .text.DMA_Init
                0x0000000000000936       0x38 ./Peripheral/src/ch32l103_dma.o
                0x0000000000000936                DMA_Init
 .text.DMA_Cmd  0x000000000000096e       0x14 ./Peripheral/src/ch32l103_dma.o
                0x000000000000096e                DMA_Cmd
 .text.DMA_ITConfig
                0x0000000000000982       0x12 ./Peripheral/src/ch32l103_dma.o
                0x0000000000000982                DMA_ITConfig
 .text.DMA_GetFlagStatus
                0x0000000000000994        0xe ./Peripheral/src/ch32l103_dma.o
                0x0000000000000994                DMA_GetFlagStatus
 .text.DMA_GetITStatus
                0x00000000000009a2        0xa ./Peripheral/src/ch32l103_dma.o
                0x00000000000009a2                DMA_GetITStatus
 .text.DMA_ClearITPendingBit
                0x00000000000009ac        0x8 ./Peripheral/src/ch32l103_dma.o
                0x00000000000009ac                DMA_ClearITPendingBit
 .text.EXTI_Init
                0x00000000000009b4       0x6a ./Peripheral/src/ch32l103_exti.o
                0x00000000000009b4                EXTI_Init
 .text.EXTI_GetITStatus
                0x0000000000000a1e       0x1e ./Peripheral/src/ch32l103_exti.o
                0x0000000000000a1e                EXTI_GetITStatus
 .text.EXTI_ClearITPendingBit
                0x0000000000000a3c        0xa ./Peripheral/src/ch32l103_exti.o
                0x0000000000000a3c                EXTI_ClearITPendingBit
 .text.GPIO_Init
                0x0000000000000a46       0xc0 ./Peripheral/src/ch32l103_gpio.o
                0x0000000000000a46                GPIO_Init
 .text.GPIO_ReadInputDataBit
                0x0000000000000b06        0xa ./Peripheral/src/ch32l103_gpio.o
                0x0000000000000b06                GPIO_ReadInputDataBit
 .text.GPIO_ReadOutputDataBit
                0x0000000000000b10        0xa ./Peripheral/src/ch32l103_gpio.o
                0x0000000000000b10                GPIO_ReadOutputDataBit
 .text.GPIO_SetBits
                0x0000000000000b1a        0x4 ./Peripheral/src/ch32l103_gpio.o
                0x0000000000000b1a                GPIO_SetBits
 .text.GPIO_WriteBit
                0x0000000000000b1e        0xa ./Peripheral/src/ch32l103_gpio.o
                0x0000000000000b1e                GPIO_WriteBit
 .text.GPIO_PinRemapConfig
                0x0000000000000b28      0x12c ./Peripheral/src/ch32l103_gpio.o
                0x0000000000000b28                GPIO_PinRemapConfig
 .text.GPIO_EXTILineConfig
                0x0000000000000c54       0x2c ./Peripheral/src/ch32l103_gpio.o
                0x0000000000000c54                GPIO_EXTILineConfig
 .text.GPIO_IPD_Unused
                0x0000000000000c80      0x190 ./Peripheral/src/ch32l103_gpio.o
                0x0000000000000c80                GPIO_IPD_Unused
 .text.NVIC_PriorityGroupConfig
                0x0000000000000e10        0x6 ./Peripheral/src/ch32l103_misc.o
                0x0000000000000e10                NVIC_PriorityGroupConfig
 .text.NVIC_Init
                0x0000000000000e16       0x54 ./Peripheral/src/ch32l103_misc.o
                0x0000000000000e16                NVIC_Init
 .text.RCC_ADCCLKConfig
                0x0000000000000e6a       0x14 ./Peripheral/src/ch32l103_rcc.o
                0x0000000000000e6a                RCC_ADCCLKConfig
 .text.RCC_GetClocksFreq
                0x0000000000000e7e       0xd6 ./Peripheral/src/ch32l103_rcc.o
                0x0000000000000e7e                RCC_GetClocksFreq
 .text.RCC_HBPeriphClockCmd
                0x0000000000000f54       0x1e ./Peripheral/src/ch32l103_rcc.o
                0x0000000000000f54                RCC_HBPeriphClockCmd
 .text.RCC_PB2PeriphClockCmd
                0x0000000000000f72       0x1e ./Peripheral/src/ch32l103_rcc.o
                0x0000000000000f72                RCC_PB2PeriphClockCmd
 .text.RCC_PB1PeriphClockCmd
                0x0000000000000f90       0x1e ./Peripheral/src/ch32l103_rcc.o
                0x0000000000000f90                RCC_PB1PeriphClockCmd
 .text.RCC_PB2PeriphResetCmd
                0x0000000000000fae       0x1e ./Peripheral/src/ch32l103_rcc.o
                0x0000000000000fae                RCC_PB2PeriphResetCmd
 .text.SPI_Init
                0x0000000000000fcc       0x32 ./Peripheral/src/ch32l103_spi.o
                0x0000000000000fcc                SPI_Init
 .text.SPI_Cmd  0x0000000000000ffe       0x1a ./Peripheral/src/ch32l103_spi.o
                0x0000000000000ffe                SPI_Cmd
 .text.SPI_I2S_SendData
                0x0000000000001018        0x4 ./Peripheral/src/ch32l103_spi.o
                0x0000000000001018                SPI_I2S_SendData
 .text.SPI_I2S_ReceiveData
                0x000000000000101c        0x4 ./Peripheral/src/ch32l103_spi.o
                0x000000000000101c                SPI_I2S_ReceiveData
 .text.SPI_I2S_GetFlagStatus
                0x0000000000001020        0xa ./Peripheral/src/ch32l103_spi.o
                0x0000000000001020                SPI_I2S_GetFlagStatus
 .text.TIM_TimeBaseInit
                0x000000000000102a       0x76 ./Peripheral/src/ch32l103_tim.o
                0x000000000000102a                TIM_TimeBaseInit
 .text.TIM_OC1Init
                0x00000000000010a0       0x7c ./Peripheral/src/ch32l103_tim.o
                0x00000000000010a0                TIM_OC1Init
 .text.TIM_OC4Init
                0x000000000000111c       0x7c ./Peripheral/src/ch32l103_tim.o
                0x000000000000111c                TIM_OC4Init
 .text.TIM_Cmd  0x0000000000001198       0x18 ./Peripheral/src/ch32l103_tim.o
                0x0000000000001198                TIM_Cmd
 .text.TIM_CtrlPWMOutputs
                0x00000000000011b0       0x16 ./Peripheral/src/ch32l103_tim.o
                0x00000000000011b0                TIM_CtrlPWMOutputs
 .text.TIM_ITConfig
                0x00000000000011c6       0x12 ./Peripheral/src/ch32l103_tim.o
                0x00000000000011c6                TIM_ITConfig
 .text.TIM_ARRPreloadConfig
                0x00000000000011d8       0x1a ./Peripheral/src/ch32l103_tim.o
                0x00000000000011d8                TIM_ARRPreloadConfig
 .text.TIM_OC1PreloadConfig
                0x00000000000011f2        0xe ./Peripheral/src/ch32l103_tim.o
                0x00000000000011f2                TIM_OC1PreloadConfig
 .text.TIM_OC4PreloadConfig
                0x0000000000001200       0x16 ./Peripheral/src/ch32l103_tim.o
                0x0000000000001200                TIM_OC4PreloadConfig
 .text.TIM_SetCompare4
                0x0000000000001216       0x16 ./Peripheral/src/ch32l103_tim.o
                0x0000000000001216                TIM_SetCompare4
 .text.TIM_GetITStatus
                0x000000000000122c       0x18 ./Peripheral/src/ch32l103_tim.o
                0x000000000000122c                TIM_GetITStatus
 .text.TIM_ClearITPendingBit
                0x0000000000001244        0xc ./Peripheral/src/ch32l103_tim.o
                0x0000000000001244                TIM_ClearITPendingBit
 .text.USART_Init
                0x0000000000001250       0xba ./Peripheral/src/ch32l103_usart.o
                0x0000000000001250                USART_Init
 .text.USART_Cmd
                0x000000000000130a       0x16 ./Peripheral/src/ch32l103_usart.o
                0x000000000000130a                USART_Cmd
 .text.USART_ITConfig
                0x0000000000001320       0x36 ./Peripheral/src/ch32l103_usart.o
                0x0000000000001320                USART_ITConfig
 .text.USART_SendData
                0x0000000000001356        0x8 ./Peripheral/src/ch32l103_usart.o
                0x0000000000001356                USART_SendData
 .text.USART_ReceiveData
                0x000000000000135e        0x8 ./Peripheral/src/ch32l103_usart.o
                0x000000000000135e                USART_ReceiveData
 .text.USART_GetFlagStatus
                0x0000000000001366        0xa ./Peripheral/src/ch32l103_usart.o
                0x0000000000001366                USART_GetFlagStatus
 .text.USART_GetITStatus
                0x0000000000001370       0x3c ./Peripheral/src/ch32l103_usart.o
                0x0000000000001370                USART_GetITStatus
 .text.ADC_all_Init
                0x00000000000013ac       0xf0 ./Hardware/src/adc.o
                0x00000000000013ac                ADC_all_Init
 .text.DMA_Tx_Init
                0x000000000000149c       0x94 ./Hardware/src/adc.o
                0x000000000000149c                DMA_Tx_Init
 .text.TIM1_Init1
                0x0000000000001530       0x7e ./Hardware/src/adc.o
                0x0000000000001530                TIM1_Init1
 .text.ADC_TIM_DMA_Init
                0x00000000000015ae      0x10e ./Hardware/src/adc.o
                0x00000000000015ae                ADC_TIM_DMA_Init
 .text.DMA1_Channel1_IRQHandler
                0x00000000000016bc       0x48 ./Hardware/src/adc.o
                0x00000000000016bc                DMA1_Channel1_IRQHandler
 .text.SPI_Flash_Init
                0x0000000000001704       0xac ./Hardware/src/flash.o
                0x0000000000001704                SPI_Flash_Init
 .text.SPI_ReadWriteByte
                0x00000000000017b0       0x62 ./Hardware/src/flash.o
                0x00000000000017b0                SPI_ReadWriteByte
 .text.SPI_Flash_Read
                0x0000000000001812       0x68 ./Hardware/src/flash.o
                0x0000000000001812                SPI_Flash_Read
 .text.RUN_LED_Init
                0x000000000000187a       0x38 ./Hardware/src/gpio.o
                0x000000000000187a                RUN_LED_Init
 .text.WDI_INPUT_Init
                0x00000000000018b2       0x32 ./Hardware/src/gpio.o
                0x00000000000018b2                WDI_INPUT_Init
 .text.POW_OUT_CON_Init
                0x00000000000018e4       0x3e ./Hardware/src/gpio.o
                0x00000000000018e4                POW_OUT_CON_Init
 .text.DSG_PROT_Init
                0x0000000000001922       0x5a ./Hardware/src/gpio.o
                0x0000000000001922                DSG_PROT_Init
 .text.EXTI2_IRQHandler
                0x000000000000197c       0x3e ./Hardware/src/gpio.o
                0x000000000000197c                EXTI2_IRQHandler
 .text.WORK_VOLT_INT_Init
                0x00000000000019ba       0x5a ./Hardware/src/gpio.o
                0x00000000000019ba                WORK_VOLT_INT_Init
 .text.EXTI15_10_IRQHandler
                0x0000000000001a14       0x34 ./Hardware/src/gpio.o
                0x0000000000001a14                EXTI15_10_IRQHandler
 .text.PWM_GPIO_Configuration
                0x0000000000001a48       0x48 ./Hardware/src/pwm.o
                0x0000000000001a48                PWM_GPIO_Configuration
 .text.PWM_TIM_Configuration
                0x0000000000001a90       0x6c ./Hardware/src/pwm.o
                0x0000000000001a90                PWM_TIM_Configuration
 .text.Set_duty_ratio
                0x0000000000001afc       0x86 ./Hardware/src/pwm.o
                0x0000000000001afc                Set_duty_ratio
 .text.GW_485_Init
                0x0000000000001b82       0xb2 ./Hardware/src/rs485.o
                0x0000000000001b82                GW_485_Init
 .text.BAT_485_Init
                0x0000000000001c34       0xbe ./Hardware/src/rs485.o
                0x0000000000001c34                BAT_485_Init
 .text.USART3_IRQHandler
                0x0000000000001cf2       0x46 ./Hardware/src/rs485.o
                0x0000000000001cf2                USART3_IRQHandler
 .text.USART4_IRQHandler
                0x0000000000001d38       0x46 ./Hardware/src/rs485.o
                0x0000000000001d38                USART4_IRQHandler
 .text.TIM3_IRQHandler
                0x0000000000001d7e       0x28 ./Hardware/src/tim.o
                0x0000000000001d7e                TIM3_IRQHandler
 .text.TIM2_Int_Init
                0x0000000000001da6       0x58 ./Hardware/src/tim.o
                0x0000000000001da6                TIM2_Int_Init
 .text.TIM2_Init
                0x0000000000001dfe       0x2e ./Hardware/src/tim.o
                0x0000000000001dfe                TIM2_Init
 .text.TIM2_IRQHandler
                0x0000000000001e2c       0x1c ./Hardware/src/tim.o
                0x0000000000001e2c                TIM2_IRQHandler
 .text.SysTick_Handler
                0x0000000000001e48        0xe ./Hardware/src/tim.o
                0x0000000000001e48                SysTick_Handler
 .text.TIM1_UP_IRQHandler
                0x0000000000001e56       0x32 ./Hardware/src/tim.o
                0x0000000000001e56                TIM1_UP_IRQHandler
 .text.TimeSliceOffset_Register
                0x0000000000001e88       0x3e ./Drivers/TimeSliceOffset/timeSliceOffset.o
                0x0000000000001e88                TimeSliceOffset_Register
 .text.TimeSliceOffset_Unregister
                0x0000000000001ec6       0x2e ./Drivers/TimeSliceOffset/timeSliceOffset.o
                0x0000000000001ec6                TimeSliceOffset_Unregister
 .text.TimeSliceOffset_Start
                0x0000000000001ef4       0x22 ./Drivers/TimeSliceOffset/timeSliceOffset.o
                0x0000000000001ef4                TimeSliceOffset_Start
 .text.TimeSliceOffset_Produce
                0x0000000000001f16       0x28 ./Drivers/TimeSliceOffset/timeSliceOffset.o
                0x0000000000001f16                TimeSliceOffset_Produce
 .text.InitRingQueue
                0x0000000000001f3e       0x10 ./Drivers/RingQueue/ring_queue.o
                0x0000000000001f3e                InitRingQueue
 .text.InRingQueue
                0x0000000000001f4e       0x2c ./Drivers/RingQueue/ring_queue.o
                0x0000000000001f4e                InRingQueue
 .text.Delay_Init
                0x0000000000001f7a       0x20 ./Debug/debug.o
                0x0000000000001f7a                Delay_Init
 .text.USART_Printf_Init
                0x0000000000001f9a       0x5a ./Debug/debug.o
                0x0000000000001f9a                USART_Printf_Init
 .text._write   0x0000000000001ff4       0x3e ./Debug/debug.o
                0x0000000000001ff4                _write
 .text._sbrk    0x0000000000002032       0x26 ./Debug/debug.o
                0x0000000000002032                _sbrk
 .text.get_adcDmaTim_middleAverageFilter
                0x0000000000002058       0xe6 ./App/src/collect_Conversion.o
 .text.Get_ConversionVal
                0x000000000000213e       0x2a ./App/src/collect_Conversion.o
                0x000000000000213e                Get_ConversionVal
 .text.middleAverageFilter
                0x0000000000002168       0x92 ./App/src/collect_Conversion.o
 .text.get_CHG_CURR
                0x00000000000021fa       0x1c ./App/src/collect_Conversion.o
                0x00000000000021fa                get_CHG_CURR
 .text.get_PV_VOLT_OUT
                0x0000000000002216        0x6 ./App/src/collect_Conversion.o
                0x0000000000002216                get_PV_VOLT_OUT
 .text.get_DSG_CURR
                0x000000000000221c       0x1c ./App/src/collect_Conversion.o
                0x000000000000221c                get_DSG_CURR
 .text.get_PV_VOLT_IN
                0x0000000000002238       0x1c ./App/src/collect_Conversion.o
                0x0000000000002238                get_PV_VOLT_IN
 .text.get_MOSFET_Temper
                0x0000000000002254       0x56 ./App/src/collect_Conversion.o
                0x0000000000002254                get_MOSFET_Temper
 .text.read_config_info
                0x00000000000022aa       0x86 ./App/src/inflash.o
                0x00000000000022aa                read_config_info
 .text.test     0x0000000000002330       0xe6 ./App/src/mppt_control.o
                0x0000000000002330                test
 .text.Task_wdi
                0x0000000000002416       0x52 ./App/src/task.o
                0x0000000000002416                Task_wdi
 .text.Task_RunLED
                0x0000000000002468       0x46 ./App/src/task.o
                0x0000000000002468                Task_RunLED
 .text.Task_outputAgain
                0x00000000000024ae       0x66 ./App/src/task.o
                0x00000000000024ae                Task_outputAgain
 .text.Task_excessiveLoad
                0x0000000000002514       0xdc ./App/src/task.o
                0x0000000000002514                Task_excessiveLoad
 .text.g_Mppt_Para_Init
                0x00000000000025f0      0x1c6 ./App/src/task.o
                0x00000000000025f0                g_Mppt_Para_Init
 .text.task_Init
                0x00000000000027b6       0x44 ./App/src/task.o
                0x00000000000027b6                task_Init
 .text.hardware_Init
                0x00000000000027fa       0x44 ./App/src/task.o
                0x00000000000027fa                hardware_Init
 .text.uart_dev_init
                0x000000000000283e       0x52 ./App/src/uart_dev.o
                0x000000000000283e                uart_dev_init
 .text.__gedf2  0x0000000000002890       0xae d:/psx/rj/mounriver_studio/toolchain/risc-v embedded gcc/bin/../lib/gcc/riscv-none-embed/8.2.0/rv32imacxw/ilp32\libgcc.a(gedf2.o)
                0x0000000000002890                __gedf2
                0x0000000000002890                __gtdf2
 .text.__ledf2  0x000000000000293e       0xb6 d:/psx/rj/mounriver_studio/toolchain/risc-v embedded gcc/bin/../lib/gcc/riscv-none-embed/8.2.0/rv32imacxw/ilp32\libgcc.a(ledf2.o)
                0x000000000000293e                __ledf2
                0x000000000000293e                __ltdf2
 .text.__muldf3
                0x00000000000029f4      0x4b8 d:/psx/rj/mounriver_studio/toolchain/risc-v embedded gcc/bin/../lib/gcc/riscv-none-embed/8.2.0/rv32imacxw/ilp32\libgcc.a(muldf3.o)
                0x00000000000029f4                __muldf3
 .text.__subdf3
                0x0000000000002eac      0x73e d:/psx/rj/mounriver_studio/toolchain/risc-v embedded gcc/bin/../lib/gcc/riscv-none-embed/8.2.0/rv32imacxw/ilp32\libgcc.a(subdf3.o)
                0x0000000000002eac                __subdf3
 .text.__floatsidf
                0x00000000000035ea       0x72 d:/psx/rj/mounriver_studio/toolchain/risc-v embedded gcc/bin/../lib/gcc/riscv-none-embed/8.2.0/rv32imacxw/ilp32\libgcc.a(floatsidf.o)
                0x00000000000035ea                __floatsidf
 .text.__divsf3
                0x000000000000365c      0x2b2 d:/psx/rj/mounriver_studio/toolchain/risc-v embedded gcc/bin/../lib/gcc/riscv-none-embed/8.2.0/rv32imacxw/ilp32\libgcc.a(divsf3.o)
                0x000000000000365c                __divsf3
 .text.__gesf2  0x000000000000390e       0x86 d:/psx/rj/mounriver_studio/toolchain/risc-v embedded gcc/bin/../lib/gcc/riscv-none-embed/8.2.0/rv32imacxw/ilp32\libgcc.a(gesf2.o)
                0x000000000000390e                __gesf2
                0x000000000000390e                __gtsf2
 .text.__lesf2  0x0000000000003994       0x8c d:/psx/rj/mounriver_studio/toolchain/risc-v embedded gcc/bin/../lib/gcc/riscv-none-embed/8.2.0/rv32imacxw/ilp32\libgcc.a(lesf2.o)
                0x0000000000003994                __ltsf2
                0x0000000000003994                __lesf2
 .text.__mulsf3
                0x0000000000003a20      0x294 d:/psx/rj/mounriver_studio/toolchain/risc-v embedded gcc/bin/../lib/gcc/riscv-none-embed/8.2.0/rv32imacxw/ilp32\libgcc.a(mulsf3.o)
                0x0000000000003a20                __mulsf3
 .text.__subsf3
                0x0000000000003cb4      0x388 d:/psx/rj/mounriver_studio/toolchain/risc-v embedded gcc/bin/../lib/gcc/riscv-none-embed/8.2.0/rv32imacxw/ilp32\libgcc.a(subsf3.o)
                0x0000000000003cb4                __subsf3
 .text.__fixsfsi
                0x000000000000403c       0x62 d:/psx/rj/mounriver_studio/toolchain/risc-v embedded gcc/bin/../lib/gcc/riscv-none-embed/8.2.0/rv32imacxw/ilp32\libgcc.a(fixsfsi.o)
                0x000000000000403c                __fixsfsi
 .text.__fixunssfsi
                0x000000000000409e       0x56 d:/psx/rj/mounriver_studio/toolchain/risc-v embedded gcc/bin/../lib/gcc/riscv-none-embed/8.2.0/rv32imacxw/ilp32\libgcc.a(fixunssfsi.o)
                0x000000000000409e                __fixunssfsi
 .text.__floatunsisf
                0x00000000000040f4       0xce d:/psx/rj/mounriver_studio/toolchain/risc-v embedded gcc/bin/../lib/gcc/riscv-none-embed/8.2.0/rv32imacxw/ilp32\libgcc.a(floatunsisf.o)
                0x00000000000040f4                __floatunsisf
 .text.__extendsfdf2
                0x00000000000041c2       0xac d:/psx/rj/mounriver_studio/toolchain/risc-v embedded gcc/bin/../lib/gcc/riscv-none-embed/8.2.0/rv32imacxw/ilp32\libgcc.a(extendsfdf2.o)
                0x00000000000041c2                __extendsfdf2
 .text.__truncdfsf2
                0x000000000000426e      0x16a d:/psx/rj/mounriver_studio/toolchain/risc-v embedded gcc/bin/../lib/gcc/riscv-none-embed/8.2.0/rv32imacxw/ilp32\libgcc.a(truncdfsf2.o)
                0x000000000000426e                __truncdfsf2
 .text.__clzsi2
                0x00000000000043d8       0x6e d:/psx/rj/mounriver_studio/toolchain/risc-v embedded gcc/bin/../lib/gcc/riscv-none-embed/8.2.0/rv32imacxw/ilp32\libgcc.a(_clzsi2.o)
                0x00000000000043d8                __clzsi2
 .text.memcpy   0x0000000000004446       0xb2 d:/psx/rj/mounriver_studio/toolchain/risc-v embedded gcc/bin/../lib/gcc/riscv-none-embed/8.2.0/../../../../riscv-none-embed/lib/rv32imacxw/ilp32\libg_nano.a(lib_a-memcpy.o)
                0x0000000000004446                memcpy
 .text.printf   0x00000000000044f8       0x40 d:/psx/rj/mounriver_studio/toolchain/risc-v embedded gcc/bin/../lib/gcc/riscv-none-embed/8.2.0/../../../../riscv-none-embed/lib/rv32imacxw/ilp32\libg_nano.a(lib_a-printf.o)
                0x00000000000044f8                iprintf
                0x00000000000044f8                printf
 .text._puts_r  0x0000000000004538       0xd4 d:/psx/rj/mounriver_studio/toolchain/risc-v embedded gcc/bin/../lib/gcc/riscv-none-embed/8.2.0/../../../../riscv-none-embed/lib/rv32imacxw/ilp32\libg_nano.a(lib_a-puts.o)
                0x0000000000004538                _puts_r
 .text.puts     0x000000000000460c        0xc d:/psx/rj/mounriver_studio/toolchain/risc-v embedded gcc/bin/../lib/gcc/riscv-none-embed/8.2.0/../../../../riscv-none-embed/lib/rv32imacxw/ilp32\libg_nano.a(lib_a-puts.o)
                0x000000000000460c                puts
 .text.__swbuf_r
                0x0000000000004618       0xbc d:/psx/rj/mounriver_studio/toolchain/risc-v embedded gcc/bin/../lib/gcc/riscv-none-embed/8.2.0/../../../../riscv-none-embed/lib/rv32imacxw/ilp32\libg_nano.a(lib_a-wbuf.o)
                0x0000000000004618                __swbuf_r
 .text.__swsetup_r
                0x00000000000046d4       0xfc d:/psx/rj/mounriver_studio/toolchain/risc-v embedded gcc/bin/../lib/gcc/riscv-none-embed/8.2.0/../../../../riscv-none-embed/lib/rv32imacxw/ilp32\libg_nano.a(lib_a-wsetup.o)
                0x00000000000046d4                __swsetup_r
 .text.__sflush_r
                0x00000000000047d0      0x130 d:/psx/rj/mounriver_studio/toolchain/risc-v embedded gcc/bin/../lib/gcc/riscv-none-embed/8.2.0/../../../../riscv-none-embed/lib/rv32imacxw/ilp32\libg_nano.a(lib_a-fflush.o)
                0x00000000000047d0                __sflush_r
 .text._fflush_r
                0x0000000000004900       0x66 d:/psx/rj/mounriver_studio/toolchain/risc-v embedded gcc/bin/../lib/gcc/riscv-none-embed/8.2.0/../../../../riscv-none-embed/lib/rv32imacxw/ilp32\libg_nano.a(lib_a-fflush.o)
                0x0000000000004900                _fflush_r
 .text.std      0x0000000000004966       0x66 d:/psx/rj/mounriver_studio/toolchain/risc-v embedded gcc/bin/../lib/gcc/riscv-none-embed/8.2.0/../../../../riscv-none-embed/lib/rv32imacxw/ilp32\libg_nano.a(lib_a-findfp.o)
 .text._cleanup_r
                0x00000000000049cc        0xa d:/psx/rj/mounriver_studio/toolchain/risc-v embedded gcc/bin/../lib/gcc/riscv-none-embed/8.2.0/../../../../riscv-none-embed/lib/rv32imacxw/ilp32\libg_nano.a(lib_a-findfp.o)
                0x00000000000049cc                _cleanup_r
 .text.__sfmoreglue
                0x00000000000049d6       0x46 d:/psx/rj/mounriver_studio/toolchain/risc-v embedded gcc/bin/../lib/gcc/riscv-none-embed/8.2.0/../../../../riscv-none-embed/lib/rv32imacxw/ilp32\libg_nano.a(lib_a-findfp.o)
                0x00000000000049d6                __sfmoreglue
 .text.__sinit  0x0000000000004a1c       0x6c d:/psx/rj/mounriver_studio/toolchain/risc-v embedded gcc/bin/../lib/gcc/riscv-none-embed/8.2.0/../../../../riscv-none-embed/lib/rv32imacxw/ilp32\libg_nano.a(lib_a-findfp.o)
                0x0000000000004a1c                __sinit
 .text.__sfp    0x0000000000004a88       0xa0 d:/psx/rj/mounriver_studio/toolchain/risc-v embedded gcc/bin/../lib/gcc/riscv-none-embed/8.2.0/../../../../riscv-none-embed/lib/rv32imacxw/ilp32\libg_nano.a(lib_a-findfp.o)
                0x0000000000004a88                __sfp
 .text._fwalk_reent
                0x0000000000004b28       0x6a d:/psx/rj/mounriver_studio/toolchain/risc-v embedded gcc/bin/../lib/gcc/riscv-none-embed/8.2.0/../../../../riscv-none-embed/lib/rv32imacxw/ilp32\libg_nano.a(lib_a-fwalk.o)
                0x0000000000004b28                _fwalk_reent
 .text.__swhatbuf_r
                0x0000000000004b92       0x58 d:/psx/rj/mounriver_studio/toolchain/risc-v embedded gcc/bin/../lib/gcc/riscv-none-embed/8.2.0/../../../../riscv-none-embed/lib/rv32imacxw/ilp32\libg_nano.a(lib_a-makebuf.o)
                0x0000000000004b92                __swhatbuf_r
 .text.__smakebuf_r
                0x0000000000004bea       0x92 d:/psx/rj/mounriver_studio/toolchain/risc-v embedded gcc/bin/../lib/gcc/riscv-none-embed/8.2.0/../../../../riscv-none-embed/lib/rv32imacxw/ilp32\libg_nano.a(lib_a-makebuf.o)
                0x0000000000004bea                __smakebuf_r
 .text._free_r  0x0000000000004c7c       0xa8 d:/psx/rj/mounriver_studio/toolchain/risc-v embedded gcc/bin/../lib/gcc/riscv-none-embed/8.2.0/../../../../riscv-none-embed/lib/rv32imacxw/ilp32\libg_nano.a(lib_a-nano-freer.o)
                0x0000000000004c7c                _free_r
 .text._malloc_r
                0x0000000000004d24       0xd4 d:/psx/rj/mounriver_studio/toolchain/risc-v embedded gcc/bin/../lib/gcc/riscv-none-embed/8.2.0/../../../../riscv-none-embed/lib/rv32imacxw/ilp32\libg_nano.a(lib_a-nano-mallocr.o)
                0x0000000000004d24                _malloc_r
 .text.__sfputc_r
                0x0000000000004df8       0x28 d:/psx/rj/mounriver_studio/toolchain/risc-v embedded gcc/bin/../lib/gcc/riscv-none-embed/8.2.0/../../../../riscv-none-embed/lib/rv32imacxw/ilp32\libg_nano.a(lib_a-nano-vfprintf.o)
 .text.__sfputs_r
                0x0000000000004e20       0x42 d:/psx/rj/mounriver_studio/toolchain/risc-v embedded gcc/bin/../lib/gcc/riscv-none-embed/8.2.0/../../../../riscv-none-embed/lib/rv32imacxw/ilp32\libg_nano.a(lib_a-nano-vfprintf.o)
                0x0000000000004e20                __sfputs_r
 .text._vfprintf_r
                0x0000000000004e62      0x288 d:/psx/rj/mounriver_studio/toolchain/risc-v embedded gcc/bin/../lib/gcc/riscv-none-embed/8.2.0/../../../../riscv-none-embed/lib/rv32imacxw/ilp32\libg_nano.a(lib_a-nano-vfprintf.o)
                0x0000000000004e62                _vfprintf_r
                0x0000000000004e62                _vfiprintf_r
 .text._printf_common
                0x00000000000050ea      0x10c d:/psx/rj/mounriver_studio/toolchain/risc-v embedded gcc/bin/../lib/gcc/riscv-none-embed/8.2.0/../../../../riscv-none-embed/lib/rv32imacxw/ilp32\libg_nano.a(lib_a-nano-vfprintf_i.o)
                0x00000000000050ea                _printf_common
 .text._printf_i
                0x00000000000051f6      0x2a2 d:/psx/rj/mounriver_studio/toolchain/risc-v embedded gcc/bin/../lib/gcc/riscv-none-embed/8.2.0/../../../../riscv-none-embed/lib/rv32imacxw/ilp32\libg_nano.a(lib_a-nano-vfprintf_i.o)
                0x00000000000051f6                _printf_i
 .text._sbrk_r  0x0000000000005498       0x2a d:/psx/rj/mounriver_studio/toolchain/risc-v embedded gcc/bin/../lib/gcc/riscv-none-embed/8.2.0/../../../../riscv-none-embed/lib/rv32imacxw/ilp32\libg_nano.a(lib_a-sbrkr.o)
                0x0000000000005498                _sbrk_r
 .text.__sread  0x00000000000054c2       0x2c d:/psx/rj/mounriver_studio/toolchain/risc-v embedded gcc/bin/../lib/gcc/riscv-none-embed/8.2.0/../../../../riscv-none-embed/lib/rv32imacxw/ilp32\libg_nano.a(lib_a-stdio.o)
                0x00000000000054c2                __sread
 .text.__swrite
                0x00000000000054ee       0x48 d:/psx/rj/mounriver_studio/toolchain/risc-v embedded gcc/bin/../lib/gcc/riscv-none-embed/8.2.0/../../../../riscv-none-embed/lib/rv32imacxw/ilp32\libg_nano.a(lib_a-stdio.o)
                0x00000000000054ee                __swrite
 .text.__sseek  0x0000000000005536       0x30 d:/psx/rj/mounriver_studio/toolchain/risc-v embedded gcc/bin/../lib/gcc/riscv-none-embed/8.2.0/../../../../riscv-none-embed/lib/rv32imacxw/ilp32\libg_nano.a(lib_a-stdio.o)
                0x0000000000005536                __sseek
 .text.__sclose
                0x0000000000005566        0x6 d:/psx/rj/mounriver_studio/toolchain/risc-v embedded gcc/bin/../lib/gcc/riscv-none-embed/8.2.0/../../../../riscv-none-embed/lib/rv32imacxw/ilp32\libg_nano.a(lib_a-stdio.o)
                0x0000000000005566                __sclose
 .text._write_r
                0x000000000000556c       0x2e d:/psx/rj/mounriver_studio/toolchain/risc-v embedded gcc/bin/../lib/gcc/riscv-none-embed/8.2.0/../../../../riscv-none-embed/lib/rv32imacxw/ilp32\libg_nano.a(lib_a-writer.o)
                0x000000000000556c                _write_r
 .text._close_r
                0x000000000000559a       0x28 d:/psx/rj/mounriver_studio/toolchain/risc-v embedded gcc/bin/../lib/gcc/riscv-none-embed/8.2.0/../../../../riscv-none-embed/lib/rv32imacxw/ilp32\libg_nano.a(lib_a-closer.o)
                0x000000000000559a                _close_r
 .text._fstat_r
                0x00000000000055c2       0x2a d:/psx/rj/mounriver_studio/toolchain/risc-v embedded gcc/bin/../lib/gcc/riscv-none-embed/8.2.0/../../../../riscv-none-embed/lib/rv32imacxw/ilp32\libg_nano.a(lib_a-fstatr.o)
                0x00000000000055c2                _fstat_r
 .text._isatty_r
                0x00000000000055ec       0x28 d:/psx/rj/mounriver_studio/toolchain/risc-v embedded gcc/bin/../lib/gcc/riscv-none-embed/8.2.0/../../../../riscv-none-embed/lib/rv32imacxw/ilp32\libg_nano.a(lib_a-isattyr.o)
                0x00000000000055ec                _isatty_r
 .text._lseek_r
                0x0000000000005614       0x2c d:/psx/rj/mounriver_studio/toolchain/risc-v embedded gcc/bin/../lib/gcc/riscv-none-embed/8.2.0/../../../../riscv-none-embed/lib/rv32imacxw/ilp32\libg_nano.a(lib_a-lseekr.o)
                0x0000000000005614                _lseek_r
 .text.memchr   0x0000000000005640       0x18 d:/psx/rj/mounriver_studio/toolchain/risc-v embedded gcc/bin/../lib/gcc/riscv-none-embed/8.2.0/../../../../riscv-none-embed/lib/rv32imacxw/ilp32\libg_nano.a(lib_a-memchr.o)
                0x0000000000005640                memchr
 .text.__malloc_lock
                0x0000000000005658        0x2 d:/psx/rj/mounriver_studio/toolchain/risc-v embedded gcc/bin/../lib/gcc/riscv-none-embed/8.2.0/../../../../riscv-none-embed/lib/rv32imacxw/ilp32\libg_nano.a(lib_a-mlock.o)
                0x0000000000005658                __malloc_lock
 .text.__malloc_unlock
                0x000000000000565a        0x2 d:/psx/rj/mounriver_studio/toolchain/risc-v embedded gcc/bin/../lib/gcc/riscv-none-embed/8.2.0/../../../../riscv-none-embed/lib/rv32imacxw/ilp32\libg_nano.a(lib_a-mlock.o)
                0x000000000000565a                __malloc_unlock
 .text._read_r  0x000000000000565c       0x2c d:/psx/rj/mounriver_studio/toolchain/risc-v embedded gcc/bin/../lib/gcc/riscv-none-embed/8.2.0/../../../../riscv-none-embed/lib/rv32imacxw/ilp32\libg_nano.a(lib_a-readr.o)
                0x000000000000565c                _read_r
 .text._close   0x0000000000005688        0xc d:/psx/rj/mounriver_studio/toolchain/risc-v embedded gcc/bin/../lib/gcc/riscv-none-embed/8.2.0/../../../../riscv-none-embed/lib/rv32imacxw/ilp32\libnosys.a(close.o)
                0x0000000000005688                _close
 .text._fstat   0x0000000000005694        0xc d:/psx/rj/mounriver_studio/toolchain/risc-v embedded gcc/bin/../lib/gcc/riscv-none-embed/8.2.0/../../../../riscv-none-embed/lib/rv32imacxw/ilp32\libnosys.a(fstat.o)
                0x0000000000005694                _fstat
 .text._isatty  0x00000000000056a0        0xc d:/psx/rj/mounriver_studio/toolchain/risc-v embedded gcc/bin/../lib/gcc/riscv-none-embed/8.2.0/../../../../riscv-none-embed/lib/rv32imacxw/ilp32\libnosys.a(isatty.o)
                0x00000000000056a0                _isatty
 .text._lseek   0x00000000000056ac        0xc d:/psx/rj/mounriver_studio/toolchain/risc-v embedded gcc/bin/../lib/gcc/riscv-none-embed/8.2.0/../../../../riscv-none-embed/lib/rv32imacxw/ilp32\libnosys.a(lseek.o)
                0x00000000000056ac                _lseek
 .text._read    0x00000000000056b8        0xc d:/psx/rj/mounriver_studio/toolchain/risc-v embedded gcc/bin/../lib/gcc/riscv-none-embed/8.2.0/../../../../riscv-none-embed/lib/rv32imacxw/ilp32\libnosys.a(read.o)
                0x00000000000056b8                _read
 *(.rodata)
 *(.rodata*)
 *fill*         0x00000000000056c4        0x0 
 .rodata.main.str1.4
                0x00000000000056c4       0x1e ./User/main.o
 *fill*         0x00000000000056e2        0x2 
 .rodata.ADC_all_Init.str1.4
                0x00000000000056e4       0x17 ./Hardware/src/adc.o
 *fill*         0x00000000000056fb        0x1 
 .rodata.DMA1_Channel1_IRQHandler.str1.4
                0x00000000000056fc        0x9 ./Hardware/src/adc.o
 *fill*         0x0000000000005705        0x3 
 .rodata.Set_duty_ratio.cst4
                0x0000000000005708        0xc ./Hardware/src/pwm.o
 *fill*         0x0000000000005714        0x4 
 .rodata.Set_duty_ratio.cst8
                0x0000000000005718       0x10 ./Hardware/src/pwm.o
 .rodata.TIM1_UP_IRQHandler.str1.4
                0x0000000000005728        0xd ./Hardware/src/tim.o
 *fill*         0x0000000000005735        0x3 
 .rodata.get_CHG_CURR.cst4
                0x0000000000005738        0x4 ./App/src/collect_Conversion.o
 *fill*         0x000000000000573c        0x4 
 .rodata.get_MOSFET_Temper.cst8
                0x0000000000005740       0x10 ./App/src/collect_Conversion.o
 .rodata.get_PV_VOLT_IN.cst4
                0x0000000000005750        0x4 ./App/src/collect_Conversion.o
 .rodata.mosTemperADC
                0x0000000000005754      0x1e2 ./App/src/collect_Conversion.o
                0x0000000000005754                mosTemperADC
 *fill*         0x0000000000005936        0x2 
 .rodata.mppt_readJust.cst4
                0x0000000000005938        0x8 ./App/src/mppt_control.o
 .rodata.test.str1.4
                0x0000000000005940        0x9 ./App/src/mppt_control.o
 .rodata.Task_impedanceCalculation.cst4
                0x0000000000005940        0x4 ./App/src/task.o
                                          0x8 (size before relaxing)
 .rodata.Task_startMpptControl.cst4
                0x0000000000005944        0x4 ./App/src/task.o
                                          0x8 (size before relaxing)
 .rodata.g_Mppt_Para_Init.cst4
                0x0000000000005948        0x4 ./App/src/task.o
 .rodata.hardware_Init.cst4
                0x000000000000594c        0x4 ./App/src/task.o
 .rodata.__muldf3
                0x0000000000005950       0x40 d:/psx/rj/mounriver_studio/toolchain/risc-v embedded gcc/bin/../lib/gcc/riscv-none-embed/8.2.0/rv32imacxw/ilp32\libgcc.a(muldf3.o)
 .rodata.__divsf3
                0x0000000000005990       0x80 d:/psx/rj/mounriver_studio/toolchain/risc-v embedded gcc/bin/../lib/gcc/riscv-none-embed/8.2.0/rv32imacxw/ilp32\libgcc.a(divsf3.o)
 .rodata.__mulsf3
                0x0000000000005a10       0x40 d:/psx/rj/mounriver_studio/toolchain/risc-v embedded gcc/bin/../lib/gcc/riscv-none-embed/8.2.0/rv32imacxw/ilp32\libgcc.a(mulsf3.o)
 .rodata.__clz_tab
                0x0000000000005a50      0x100 d:/psx/rj/mounriver_studio/toolchain/risc-v embedded gcc/bin/../lib/gcc/riscv-none-embed/8.2.0/rv32imacxw/ilp32\libgcc.a(_clz.o)
                0x0000000000005a50                __clz_tab
 .rodata.__sf_fake_stderr
                0x0000000000005b50       0x20 d:/psx/rj/mounriver_studio/toolchain/risc-v embedded gcc/bin/../lib/gcc/riscv-none-embed/8.2.0/../../../../riscv-none-embed/lib/rv32imacxw/ilp32\libg_nano.a(lib_a-findfp.o)
                0x0000000000005b50                __sf_fake_stderr
 .rodata.__sf_fake_stdin
                0x0000000000005b70       0x20 d:/psx/rj/mounriver_studio/toolchain/risc-v embedded gcc/bin/../lib/gcc/riscv-none-embed/8.2.0/../../../../riscv-none-embed/lib/rv32imacxw/ilp32\libg_nano.a(lib_a-findfp.o)
                0x0000000000005b70                __sf_fake_stdin
 .rodata.__sf_fake_stdout
                0x0000000000005b90       0x20 d:/psx/rj/mounriver_studio/toolchain/risc-v embedded gcc/bin/../lib/gcc/riscv-none-embed/8.2.0/../../../../riscv-none-embed/lib/rv32imacxw/ilp32\libg_nano.a(lib_a-findfp.o)
                0x0000000000005b90                __sf_fake_stdout
 .rodata._vfprintf_r.str1.4
                0x0000000000005bb0       0x13 d:/psx/rj/mounriver_studio/toolchain/risc-v embedded gcc/bin/../lib/gcc/riscv-none-embed/8.2.0/../../../../riscv-none-embed/lib/rv32imacxw/ilp32\libg_nano.a(lib_a-nano-vfprintf.o)
 *fill*         0x0000000000005bc3        0x1 
 .rodata._printf_i.str1.4
                0x0000000000005bc4       0x28 d:/psx/rj/mounriver_studio/toolchain/risc-v embedded gcc/bin/../lib/gcc/riscv-none-embed/8.2.0/../../../../riscv-none-embed/lib/rv32imacxw/ilp32\libg_nano.a(lib_a-nano-vfprintf_i.o)
                                         0x25 (size before relaxing)
 *(.gnu.linkonce.t.*)
                0x0000000000005bec                . = ALIGN (0x4)

.rela.dyn       0x0000000000005bec        0x0
 .rela.init     0x0000000000005bec        0x0 ./User/ch32l103_it.o
 .rela.vector   0x0000000000005bec        0x0 ./User/ch32l103_it.o
 .rela.text.handle_reset
                0x0000000000005bec        0x0 ./User/ch32l103_it.o
 .rela.text._sbrk
                0x0000000000005bec        0x0 ./User/ch32l103_it.o
 .rela.sdata.curbrk.5007
                0x0000000000005bec        0x0 ./User/ch32l103_it.o
 .rela.text._vfprintf_r
                0x0000000000005bec        0x0 ./User/ch32l103_it.o
 .rela.text._sbrk_r
                0x0000000000005bec        0x0 ./User/ch32l103_it.o
 .rela.text._write_r
                0x0000000000005bec        0x0 ./User/ch32l103_it.o
 .rela.text._close_r
                0x0000000000005bec        0x0 ./User/ch32l103_it.o
 .rela.text._fstat_r
                0x0000000000005bec        0x0 ./User/ch32l103_it.o
 .rela.text._isatty_r
                0x0000000000005bec        0x0 ./User/ch32l103_it.o
 .rela.text._lseek_r
                0x0000000000005bec        0x0 ./User/ch32l103_it.o
 .rela.text._read_r
                0x0000000000005bec        0x0 ./User/ch32l103_it.o
 .rela.text._close
                0x0000000000005bec        0x0 ./User/ch32l103_it.o
 .rela.text._fstat
                0x0000000000005bec        0x0 ./User/ch32l103_it.o
 .rela.text._isatty
                0x0000000000005bec        0x0 ./User/ch32l103_it.o
 .rela.text._lseek
                0x0000000000005bec        0x0 ./User/ch32l103_it.o
 .rela.text._read
                0x0000000000005bec        0x0 ./User/ch32l103_it.o

.fini           0x0000000000005bec        0x0
 *(SORT_NONE(.fini))
                0x0000000000005bec                . = ALIGN (0x4)
                [!provide]                        PROVIDE (_etext = .)
                [!provide]                        PROVIDE (_eitcm = .)

.preinit_array  0x0000000000005bec        0x0
                [!provide]                        PROVIDE (__preinit_array_start = .)
 *(.preinit_array)
                [!provide]                        PROVIDE (__preinit_array_end = .)

.init_array     0x0000000000005bec        0x0
                [!provide]                        PROVIDE (__init_array_start = .)
 *(SORT_BY_INIT_PRIORITY(.init_array.*) SORT_BY_INIT_PRIORITY(.ctors.*))
 *(.init_array EXCLUDE_FILE(*crtend?.o *crtend.o *crtbegin?.o *crtbegin.o) .ctors)
                [!provide]                        PROVIDE (__init_array_end = .)

.fini_array     0x0000000000005bec        0x0
                [!provide]                        PROVIDE (__fini_array_start = .)
 *(SORT_BY_INIT_PRIORITY(.fini_array.*) SORT_BY_INIT_PRIORITY(.dtors.*))
 *(.fini_array EXCLUDE_FILE(*crtend?.o *crtend.o *crtbegin?.o *crtbegin.o) .dtors)
                [!provide]                        PROVIDE (__fini_array_end = .)

.ctors
 *crtbegin.o(.ctors)
 *crtbegin?.o(.ctors)
 *(EXCLUDE_FILE(*crtend?.o *crtend.o) .ctors)
 *(SORT_BY_NAME(.ctors.*))
 *(.ctors)

.dtors
 *crtbegin.o(.dtors)
 *crtbegin?.o(.dtors)
 *(EXCLUDE_FILE(*crtend?.o *crtend.o) .dtors)
 *(SORT_BY_NAME(.dtors.*))
 *(.dtors)

.dalign         0x0000000020000000        0x0 load address 0x0000000000005bec
                0x0000000020000000                . = ALIGN (0x4)
                0x0000000020000000                PROVIDE (_data_vma = .)

.dlalign        0x0000000000005bec        0x0
                0x0000000000005bec                . = ALIGN (0x4)
                0x0000000000005bec                PROVIDE (_data_lma = .)

.data           0x0000000020000000      0x118 load address 0x0000000000005bec
 *(.gnu.linkonce.r.*)
 *(.data .data.*)
 .data.HBPrescTable
                0x0000000020000000       0x10 ./User/system_ch32l103.o
                0x0000000020000000                HBPrescTable
 .data.PBHBPrescTable
                0x0000000020000010       0x10 ./Peripheral/src/ch32l103_rcc.o
 .data.g_slConfigInfo
                0x0000000020000020       0x32 ./App/src/inflash.o
                0x0000000020000020                g_slConfigInfo
 *fill*         0x0000000020000052        0x2 
 .data.defaultValue
                0x0000000020000054        0xe ./App/src/sl_protocol.o
                0x0000000020000054                defaultValue
 *fill*         0x0000000020000062        0x2 
 .data.uart_devices
                0x0000000020000064       0x38 ./App/src/uart_dev.o
                0x0000000020000064                uart_devices
 .data.impure_data
                0x000000002000009c       0x60 d:/psx/rj/mounriver_studio/toolchain/risc-v embedded gcc/bin/../lib/gcc/riscv-none-embed/8.2.0/../../../../riscv-none-embed/lib/rv32imacxw/ilp32\libg_nano.a(lib_a-impure.o)
 *(.gnu.linkonce.d.*)
                0x0000000020000100                . = ALIGN (0x8)
 *fill*         0x00000000200000fc        0x4 
                0x0000000020000900                PROVIDE (__global_pointer$ = (. + 0x800))
 *(.sdata .sdata.*)
 .sdata.SystemCoreClock
                0x0000000020000100        0x4 ./User/system_ch32l103.o
                0x0000000020000100                SystemCoreClock
 .sdata.ADCPrescTable
                0x0000000020000104        0x4 ./Peripheral/src/ch32l103_rcc.o
 .sdata.curbrk.5007
                0x0000000020000108        0x4 ./Debug/debug.o
 .sdata.g_duty_ratio
                0x000000002000010c        0x4 ./App/src/mppt_control.o
                0x000000002000010c                g_duty_ratio
 .sdata._impure_ptr
                0x0000000020000110        0x4 d:/psx/rj/mounriver_studio/toolchain/risc-v embedded gcc/bin/../lib/gcc/riscv-none-embed/8.2.0/../../../../riscv-none-embed/lib/rv32imacxw/ilp32\libg_nano.a(lib_a-impure.o)
                0x0000000020000110                _impure_ptr
 *(.sdata2.*)
 .sdata2._global_impure_ptr
                0x0000000020000114        0x4 d:/psx/rj/mounriver_studio/toolchain/risc-v embedded gcc/bin/../lib/gcc/riscv-none-embed/8.2.0/../../../../riscv-none-embed/lib/rv32imacxw/ilp32\libg_nano.a(lib_a-impure.o)
                0x0000000020000114                _global_impure_ptr
 *(.gnu.linkonce.s.*)
                0x0000000020000118                . = ALIGN (0x8)
 *(.srodata.cst16)
 *(.srodata.cst8)
 *(.srodata.cst4)
 *(.srodata.cst2)
 *(.srodata .srodata.*)
                0x0000000020000118                . = ALIGN (0x4)
                0x0000000020000118                PROVIDE (_edata = .)

.bss            0x0000000020000118      0x514 load address 0x0000000000005d04
                0x0000000020000118                . = ALIGN (0x4)
                0x0000000020000118                PROVIDE (_sbss = .)
 *(.sbss*)
 .sbss.ADC_Trim
                0x0000000020000118        0x2 ./Peripheral/src/ch32l103_gpio.o
                0x0000000020000118                ADC_Trim
 *fill*         0x000000002000011a        0x2 
 .sbss.CHIPID   0x000000002000011c        0x4 ./Peripheral/src/ch32l103_gpio.o
                0x000000002000011c                CHIPID
 .sbss.OPA_Trim
                0x0000000020000120        0x4 ./Peripheral/src/ch32l103_gpio.o
                0x0000000020000120                OPA_Trim
 .sbss.TS_Val   0x0000000020000124        0x4 ./Peripheral/src/ch32l103_gpio.o
                0x0000000020000124                TS_Val
 .sbss.NVIC_Priority_Group
                0x0000000020000128        0x4 ./Peripheral/src/ch32l103_misc.o
                0x0000000020000128                NVIC_Priority_Group
 .sbss.ADC_ConvertedValue
                0x000000002000012c        0x6 ./Hardware/src/adc.o
                0x000000002000012c                ADC_ConvertedValue
 .sbss.Calibrattion_Val
                0x0000000020000132        0x2 ./Hardware/src/adc.o
                0x0000000020000132                Calibrattion_Val
 .sbss.USART3_Rbuffer
                0x0000000020000134        0x1 ./Hardware/src/rs485.o
                0x0000000020000134                USART3_Rbuffer
 *fill*         0x0000000020000135        0x3 
 .sbss.USART4_Rbuffer
                0x0000000020000138        0x1 ./Hardware/src/rs485.o
                0x0000000020000138                USART4_Rbuffer
 *fill*         0x0000000020000139        0x3 
 .sbss.pTimeSliceList
                0x000000002000013c        0x4 ./Drivers/TimeSliceOffset/timeSliceOffset.o
 .sbss.p_ms     0x0000000020000140        0x2 ./Debug/debug.o
 .sbss.p_us     0x0000000020000142        0x2 ./Debug/debug.o
 .sbss.excessiveLoadFlag
                0x0000000020000144        0x1 ./App/src/task.o
                0x0000000020000144                excessiveLoadFlag
 .sbss.flag.6438
                0x0000000020000145        0x1 ./App/src/task.o
 *fill*         0x0000000020000146        0x2 
 .sbss.g_impedance
                0x0000000020000148        0x4 ./App/src/task.o
                0x0000000020000148                g_impedance
 .sbss.g_impedanceStart
                0x000000002000014c        0x1 ./App/src/task.o
                0x000000002000014c                g_impedanceStart
 .sbss.num.6439
                0x000000002000014d        0x1 ./App/src/task.o
 .sbss.num.6502
                0x000000002000014e        0x1 ./App/src/task.o
 .sbss.num.6508
                0x000000002000014f        0x1 ./App/src/task.o
 .sbss.numLong.6509
                0x0000000020000150        0x2 ./App/src/task.o
 .sbss.outputAgainFlag
                0x0000000020000152        0x1 ./App/src/task.o
                0x0000000020000152                outputAgainFlag
 *fill*         0x0000000020000153        0x1 
 .sbss.temp.6461
                0x0000000020000154        0x4 ./App/src/task.o
 .sbss.g_bat485_uart3_handle
                0x0000000020000158        0x4 ./App/src/uart_dev.o
                0x0000000020000158                g_bat485_uart3_handle
 .sbss.g_gw485_uart4_handle
                0x000000002000015c        0x4 ./App/src/uart_dev.o
                0x000000002000015c                g_gw485_uart4_handle
 .sbss.__malloc_free_list
                0x0000000020000160        0x4 d:/psx/rj/mounriver_studio/toolchain/risc-v embedded gcc/bin/../lib/gcc/riscv-none-embed/8.2.0/../../../../riscv-none-embed/lib/rv32imacxw/ilp32\libg_nano.a(lib_a-nano-mallocr.o)
                0x0000000020000160                __malloc_free_list
 .sbss.__malloc_sbrk_start
                0x0000000020000164        0x4 d:/psx/rj/mounriver_studio/toolchain/risc-v embedded gcc/bin/../lib/gcc/riscv-none-embed/8.2.0/../../../../riscv-none-embed/lib/rv32imacxw/ilp32\libg_nano.a(lib_a-nano-mallocr.o)
                0x0000000020000164                __malloc_sbrk_start
 *(.gnu.linkonce.sb.*)
 *(.bss*)
 .bss.g_adcData
                0x0000000020000168      0x25a ./Hardware/src/adc.o
                0x0000000020000168                g_adcData
 *fill*         0x00000000200003c2        0x2 
 .bss.g_Mppt_Para
                0x00000000200003c4       0x2d ./App/src/sl_protocol.o
                0x00000000200003c4                g_Mppt_Para
 *fill*         0x00000000200003f1        0x3 
 .bss.m_excessiveLoad
                0x00000000200003f4       0x10 ./App/src/task.o
                0x00000000200003f4                m_excessiveLoad
 .bss.m_outputAgain
                0x0000000020000404       0x10 ./App/src/task.o
                0x0000000020000404                m_outputAgain
 .bss.m_runled  0x0000000020000414       0x10 ./App/src/task.o
                0x0000000020000414                m_runled
 .bss.m_wdi     0x0000000020000424       0x10 ./App/src/task.o
                0x0000000020000424                m_wdi
 .bss.bat485_in_buff
                0x0000000020000434       0xc8 ./App/src/uart_dev.o
 .bss.gw485_in_buff
                0x00000000200004fc      0x12c ./App/src/uart_dev.o
 *(.gnu.linkonce.b.*)
 *(COMMON*)
 COMMON         0x0000000020000628        0x4 d:/psx/rj/mounriver_studio/toolchain/risc-v embedded gcc/bin/../lib/gcc/riscv-none-embed/8.2.0/../../../../riscv-none-embed/lib/rv32imacxw/ilp32\libg_nano.a(lib_a-reent.o)
                0x0000000020000628                errno
                0x000000002000062c                . = ALIGN (0x4)
                0x000000002000062c                PROVIDE (_ebss = .)
                0x000000002000062c                PROVIDE (_end = _ebss)
                [!provide]                        PROVIDE (end = .)

.stack          0x0000000020004800      0x800
                0x0000000020004800                PROVIDE (_heap_end = .)
                0x0000000020004800                . = ALIGN (0x4)
                [!provide]                        PROVIDE (_susrstack = .)
                0x0000000020005000                . = (. + __stack_size)
 *fill*         0x0000000020004800      0x800 
                0x0000000020005000                PROVIDE (_eusrstack = .)
OUTPUT(mppt_Nos_V0.4.elf elf32-littleriscv)

.debug_info     0x0000000000000000    0x23059
 .debug_info    0x0000000000000000      0x9aa ./User/ch32l103_it.o
 .debug_info    0x00000000000009aa      0xca3 ./User/main.o
 .debug_info    0x000000000000164d      0xc5f ./User/system_ch32l103.o
 .debug_info    0x00000000000022ac       0x22 ./Startup/startup_ch32l103.o
 .debug_info    0x00000000000022ce     0x1b9e ./Peripheral/src/ch32l103_adc.o
 .debug_info    0x0000000000003e6c      0xadc ./Peripheral/src/ch32l103_dbgmcu.o
 .debug_info    0x0000000000004948      0xd4c ./Peripheral/src/ch32l103_dma.o
 .debug_info    0x0000000000005694      0xc55 ./Peripheral/src/ch32l103_exti.o
 .debug_info    0x00000000000062e9     0x125d ./Peripheral/src/ch32l103_gpio.o
 .debug_info    0x0000000000007546      0xed8 ./Peripheral/src/ch32l103_misc.o
 .debug_info    0x000000000000841e     0x12a5 ./Peripheral/src/ch32l103_rcc.o
 .debug_info    0x00000000000096c3     0x1118 ./Peripheral/src/ch32l103_spi.o
 .debug_info    0x000000000000a7db     0x2ac7 ./Peripheral/src/ch32l103_tim.o
 .debug_info    0x000000000000d2a2     0x13e4 ./Peripheral/src/ch32l103_usart.o
 .debug_info    0x000000000000e686     0x1cbf ./Hardware/src/adc.o
 .debug_info    0x0000000000010345     0x1a36 ./Hardware/src/flash.o
 .debug_info    0x0000000000011d7b     0x14cc ./Hardware/src/gpio.o
 .debug_info    0x0000000000013247     0x10cf ./Hardware/src/pwm.o
 .debug_info    0x0000000000014316     0x14ab ./Hardware/src/rs485.o
 .debug_info    0x00000000000157c1     0x1954 ./Hardware/src/tim.o
 .debug_info    0x0000000000017115      0xb61 ./Drivers/TimeSliceOffset/timeSliceOffset.o
 .debug_info    0x0000000000017c76      0xa9c ./Drivers/RingQueue/ring_queue.o
 .debug_info    0x0000000000018712      0xf18 ./Debug/debug.o
 .debug_info    0x000000000001962a     0x1318 ./App/src/collect_Conversion.o
 .debug_info    0x000000000001a942      0xe24 ./App/src/inflash.o
 .debug_info    0x000000000001b766     0x197f ./App/src/mppt_control.o
 .debug_info    0x000000000001d0e5     0x284a ./App/src/sl_protocol.o
 .debug_info    0x000000000001f92f     0x235f ./App/src/task.o
 .debug_info    0x0000000000021c8e     0x13cb ./App/src/uart_dev.o

.debug_abbrev   0x0000000000000000     0x5ae3
 .debug_abbrev  0x0000000000000000      0x1cf ./User/ch32l103_it.o
 .debug_abbrev  0x00000000000001cf      0x238 ./User/main.o
 .debug_abbrev  0x0000000000000407      0x2d7 ./User/system_ch32l103.o
 .debug_abbrev  0x00000000000006de       0x12 ./Startup/startup_ch32l103.o
 .debug_abbrev  0x00000000000006f0      0x44a ./Peripheral/src/ch32l103_adc.o
 .debug_abbrev  0x0000000000000b3a      0x2f7 ./Peripheral/src/ch32l103_dbgmcu.o
 .debug_abbrev  0x0000000000000e31      0x302 ./Peripheral/src/ch32l103_dma.o
 .debug_abbrev  0x0000000000001133      0x2da ./Peripheral/src/ch32l103_exti.o
 .debug_abbrev  0x000000000000140d      0x347 ./Peripheral/src/ch32l103_gpio.o
 .debug_abbrev  0x0000000000001754      0x2ea ./Peripheral/src/ch32l103_misc.o
 .debug_abbrev  0x0000000000001a3e      0x351 ./Peripheral/src/ch32l103_rcc.o
 .debug_abbrev  0x0000000000001d8f      0x303 ./Peripheral/src/ch32l103_spi.o
 .debug_abbrev  0x0000000000002092      0x418 ./Peripheral/src/ch32l103_tim.o
 .debug_abbrev  0x00000000000024aa      0x312 ./Peripheral/src/ch32l103_usart.o
 .debug_abbrev  0x00000000000027bc      0x310 ./Hardware/src/adc.o
 .debug_abbrev  0x0000000000002acc      0x3e4 ./Hardware/src/flash.o
 .debug_abbrev  0x0000000000002eb0      0x289 ./Hardware/src/gpio.o
 .debug_abbrev  0x0000000000003139      0x2b9 ./Hardware/src/pwm.o
 .debug_abbrev  0x00000000000033f2      0x2e3 ./Hardware/src/rs485.o
 .debug_abbrev  0x00000000000036d5      0x3a4 ./Hardware/src/tim.o
 .debug_abbrev  0x0000000000003a79      0x279 ./Drivers/TimeSliceOffset/timeSliceOffset.o
 .debug_abbrev  0x0000000000003cf2      0x23a ./Drivers/RingQueue/ring_queue.o
 .debug_abbrev  0x0000000000003f2c      0x2d7 ./Debug/debug.o
 .debug_abbrev  0x0000000000004203      0x475 ./App/src/collect_Conversion.o
 .debug_abbrev  0x0000000000004678      0x28f ./App/src/inflash.o
 .debug_abbrev  0x0000000000004907      0x45c ./App/src/mppt_control.o
 .debug_abbrev  0x0000000000004d63      0x532 ./App/src/sl_protocol.o
 .debug_abbrev  0x0000000000005295      0x447 ./App/src/task.o
 .debug_abbrev  0x00000000000056dc      0x407 ./App/src/uart_dev.o

.debug_aranges  0x0000000000000000      0xf98
 .debug_aranges
                0x0000000000000000       0x28 ./User/ch32l103_it.o
 .debug_aranges
                0x0000000000000028       0x20 ./User/main.o
 .debug_aranges
                0x0000000000000048       0x28 ./User/system_ch32l103.o
 .debug_aranges
                0x0000000000000070       0x30 ./Startup/startup_ch32l103.o
 .debug_aranges
                0x00000000000000a0      0x190 ./Peripheral/src/ch32l103_adc.o
 .debug_aranges
                0x0000000000000230       0x48 ./Peripheral/src/ch32l103_dbgmcu.o
 .debug_aranges
                0x0000000000000278       0x60 ./Peripheral/src/ch32l103_dma.o
 .debug_aranges
                0x00000000000002d8       0x50 ./Peripheral/src/ch32l103_exti.o
 .debug_aranges
                0x0000000000000328       0xa8 ./Peripheral/src/ch32l103_gpio.o
 .debug_aranges
                0x00000000000003d0       0x28 ./Peripheral/src/ch32l103_misc.o
 .debug_aranges
                0x00000000000003f8      0x130 ./Peripheral/src/ch32l103_rcc.o
 .debug_aranges
                0x0000000000000528       0xc0 ./Peripheral/src/ch32l103_spi.o
 .debug_aranges
                0x00000000000005e8      0x2e0 ./Peripheral/src/ch32l103_tim.o
 .debug_aranges
                0x00000000000008c8      0x100 ./Peripheral/src/ch32l103_usart.o
 .debug_aranges
                0x00000000000009c8       0x48 ./Hardware/src/adc.o
 .debug_aranges
                0x0000000000000a10       0xa0 ./Hardware/src/flash.o
 .debug_aranges
                0x0000000000000ab0       0x68 ./Hardware/src/gpio.o
 .debug_aranges
                0x0000000000000b18       0x30 ./Hardware/src/pwm.o
 .debug_aranges
                0x0000000000000b48       0x48 ./Hardware/src/rs485.o
 .debug_aranges
                0x0000000000000b90       0x70 ./Hardware/src/tim.o
 .debug_aranges
                0x0000000000000c00       0x38 ./Drivers/TimeSliceOffset/timeSliceOffset.o
 .debug_aranges
                0x0000000000000c38       0x40 ./Drivers/RingQueue/ring_queue.o
 .debug_aranges
                0x0000000000000c78       0x48 ./Debug/debug.o
 .debug_aranges
                0x0000000000000cc0       0x70 ./App/src/collect_Conversion.o
 .debug_aranges
                0x0000000000000d30       0x30 ./App/src/inflash.o
 .debug_aranges
                0x0000000000000d60       0x78 ./App/src/mppt_control.o
 .debug_aranges
                0x0000000000000dd8       0xa8 ./App/src/sl_protocol.o
 .debug_aranges
                0x0000000000000e80       0x98 ./App/src/task.o
 .debug_aranges
                0x0000000000000f18       0x80 ./App/src/uart_dev.o

.debug_ranges   0x0000000000000000     0x11b0
 .debug_ranges  0x0000000000000000       0x18 ./User/ch32l103_it.o
 .debug_ranges  0x0000000000000018       0x10 ./User/main.o
 .debug_ranges  0x0000000000000028       0x48 ./User/system_ch32l103.o
 .debug_ranges  0x0000000000000070       0x28 ./Startup/startup_ch32l103.o
 .debug_ranges  0x0000000000000098      0x1b8 ./Peripheral/src/ch32l103_adc.o
 .debug_ranges  0x0000000000000250       0x50 ./Peripheral/src/ch32l103_dbgmcu.o
 .debug_ranges  0x00000000000002a0       0x50 ./Peripheral/src/ch32l103_dma.o
 .debug_ranges  0x00000000000002f0       0x40 ./Peripheral/src/ch32l103_exti.o
 .debug_ranges  0x0000000000000330       0x98 ./Peripheral/src/ch32l103_gpio.o
 .debug_ranges  0x00000000000003c8       0x48 ./Peripheral/src/ch32l103_misc.o
 .debug_ranges  0x0000000000000410      0x120 ./Peripheral/src/ch32l103_rcc.o
 .debug_ranges  0x0000000000000530       0xb0 ./Peripheral/src/ch32l103_spi.o
 .debug_ranges  0x00000000000005e0      0x300 ./Peripheral/src/ch32l103_tim.o
 .debug_ranges  0x00000000000008e0       0xf0 ./Peripheral/src/ch32l103_usart.o
 .debug_ranges  0x00000000000009d0       0x38 ./Hardware/src/adc.o
 .debug_ranges  0x0000000000000a08       0xb0 ./Hardware/src/flash.o
 .debug_ranges  0x0000000000000ab8       0x58 ./Hardware/src/gpio.o
 .debug_ranges  0x0000000000000b10       0x20 ./Hardware/src/pwm.o
 .debug_ranges  0x0000000000000b30       0x38 ./Hardware/src/rs485.o
 .debug_ranges  0x0000000000000b68       0x78 ./Hardware/src/tim.o
 .debug_ranges  0x0000000000000be0       0x90 ./Drivers/TimeSliceOffset/timeSliceOffset.o
 .debug_ranges  0x0000000000000c70       0x30 ./Drivers/RingQueue/ring_queue.o
 .debug_ranges  0x0000000000000ca0       0x38 ./Debug/debug.o
 .debug_ranges  0x0000000000000cd8       0x98 ./App/src/collect_Conversion.o
 .debug_ranges  0x0000000000000d70       0x20 ./App/src/inflash.o
 .debug_ranges  0x0000000000000d90       0x98 ./App/src/mppt_control.o
 .debug_ranges  0x0000000000000e28      0x230 ./App/src/sl_protocol.o
 .debug_ranges  0x0000000000001058       0xa0 ./App/src/task.o
 .debug_ranges  0x00000000000010f8       0xb8 ./App/src/uart_dev.o

.debug_line     0x0000000000000000    0x152fa
 .debug_line    0x0000000000000000      0x22f ./User/ch32l103_it.o
 .debug_line    0x000000000000022f      0x340 ./User/main.o
 .debug_line    0x000000000000056f      0x6cf ./User/system_ch32l103.o
 .debug_line    0x0000000000000c3e      0x11e ./Startup/startup_ch32l103.o
 .debug_line    0x0000000000000d5c     0x1cea ./Peripheral/src/ch32l103_adc.o
 .debug_line    0x0000000000002a46      0x34d ./Peripheral/src/ch32l103_dbgmcu.o
 .debug_line    0x0000000000002d93      0x76b ./Peripheral/src/ch32l103_dma.o
 .debug_line    0x00000000000034fe      0x580 ./Peripheral/src/ch32l103_exti.o
 .debug_line    0x0000000000003a7e     0x1249 ./Peripheral/src/ch32l103_gpio.o
 .debug_line    0x0000000000004cc7      0x387 ./Peripheral/src/ch32l103_misc.o
 .debug_line    0x000000000000504e     0x118b ./Peripheral/src/ch32l103_rcc.o
 .debug_line    0x00000000000061d9      0xa01 ./Peripheral/src/ch32l103_spi.o
 .debug_line    0x0000000000006bda     0x3218 ./Peripheral/src/ch32l103_tim.o
 .debug_line    0x0000000000009df2      0xf51 ./Peripheral/src/ch32l103_usart.o
 .debug_line    0x000000000000ad43      0xb5a ./Hardware/src/adc.o
 .debug_line    0x000000000000b89d      0xd9e ./Hardware/src/flash.o
 .debug_line    0x000000000000c63b      0xaa9 ./Hardware/src/gpio.o
 .debug_line    0x000000000000d0e4      0x4fb ./Hardware/src/pwm.o
 .debug_line    0x000000000000d5df      0x8a6 ./Hardware/src/rs485.o
 .debug_line    0x000000000000de85      0x91a ./Hardware/src/tim.o
 .debug_line    0x000000000000e79f      0x58c ./Drivers/TimeSliceOffset/timeSliceOffset.o
 .debug_line    0x000000000000ed2b      0x3c0 ./Drivers/RingQueue/ring_queue.o
 .debug_line    0x000000000000f0eb      0x696 ./Debug/debug.o
 .debug_line    0x000000000000f781      0xa89 ./App/src/collect_Conversion.o
 .debug_line    0x000000000001020a      0x5a8 ./App/src/inflash.o
 .debug_line    0x00000000000107b2      0xff9 ./App/src/mppt_control.o
 .debug_line    0x00000000000117ab     0x1907 ./App/src/sl_protocol.o
 .debug_line    0x00000000000130b2     0x19e6 ./App/src/task.o
 .debug_line    0x0000000000014a98      0x862 ./App/src/uart_dev.o

.debug_str      0x0000000000000000     0x4e18
 .debug_str     0x0000000000000000      0x53e ./User/ch32l103_it.o
                                        0x5c2 (size before relaxing)
 .debug_str     0x000000000000053e      0x2f3 ./User/main.o
                                        0x8a8 (size before relaxing)
 .debug_str     0x0000000000000831      0x124 ./User/system_ch32l103.o
                                        0x6fc (size before relaxing)
 .debug_str     0x0000000000000955       0x2a ./Startup/startup_ch32l103.o
                                         0x3e (size before relaxing)
 .debug_str     0x000000000000097f      0x6d7 ./Peripheral/src/ch32l103_adc.o
                                        0xd19 (size before relaxing)
 .debug_str     0x0000000000001056       0x7e ./Peripheral/src/ch32l103_dbgmcu.o
                                        0x652 (size before relaxing)
 .debug_str     0x00000000000010d4      0x1fc ./Peripheral/src/ch32l103_dma.o
                                        0x7eb (size before relaxing)
 .debug_str     0x00000000000012d0      0x1ae ./Peripheral/src/ch32l103_exti.o
                                        0x799 (size before relaxing)
 .debug_str     0x000000000000147e      0x367 ./Peripheral/src/ch32l103_gpio.o
                                        0x976 (size before relaxing)
 .debug_str     0x00000000000017e5      0x4f1 ./Peripheral/src/ch32l103_misc.o
                                        0xadc (size before relaxing)
 .debug_str     0x0000000000001cd6      0x3d2 ./Peripheral/src/ch32l103_rcc.o
                                        0xab3 (size before relaxing)
 .debug_str     0x00000000000020a8      0x2b1 ./Peripheral/src/ch32l103_spi.o
                                        0x95c (size before relaxing)
 .debug_str     0x0000000000002359      0xbdb ./Peripheral/src/ch32l103_tim.o
                                       0x12c1 (size before relaxing)
 .debug_str     0x0000000000002f34      0x401 ./Peripheral/src/ch32l103_usart.o
                                        0xb0c (size before relaxing)
 .debug_str     0x0000000000003335      0x19b ./Hardware/src/adc.o
                                       0x12c7 (size before relaxing)
 .debug_str     0x00000000000034d0      0x222 ./Hardware/src/flash.o
                                        0xb11 (size before relaxing)
 .debug_str     0x00000000000036f2       0xe5 ./Hardware/src/gpio.o
                                        0xf79 (size before relaxing)
 .debug_str     0x00000000000037d7       0x6e ./Hardware/src/pwm.o
                                        0xa88 (size before relaxing)
 .debug_str     0x0000000000003845      0x14b ./Hardware/src/rs485.o
                                        0xe4a (size before relaxing)
 .debug_str     0x0000000000003990      0x124 ./Hardware/src/tim.o
                                       0x1028 (size before relaxing)
 .debug_str     0x0000000000003ab4       0x7b ./Drivers/TimeSliceOffset/timeSliceOffset.o
                                        0x6eb (size before relaxing)
 .debug_str     0x0000000000003b2f       0x65 ./Drivers/RingQueue/ring_queue.o
                                        0x5e7 (size before relaxing)
 .debug_str     0x0000000000003b94       0x41 ./Debug/debug.o
                                        0x8e4 (size before relaxing)
 .debug_str     0x0000000000003bd5      0x16f ./App/src/collect_Conversion.o
                                        0x98f (size before relaxing)
 .debug_str     0x0000000000003d44      0x264 ./App/src/inflash.o
                                        0x9f7 (size before relaxing)
 .debug_str     0x0000000000003fa8      0x29e ./App/src/mppt_control.o
                                       0x1065 (size before relaxing)
 .debug_str     0x0000000000004246      0x897 ./App/src/sl_protocol.o
                                       0x169f (size before relaxing)
 .debug_str     0x0000000000004add      0x25c ./App/src/task.o
                                       0x148c (size before relaxing)
 .debug_str     0x0000000000004d39       0xdf ./App/src/uart_dev.o
                                        0xad7 (size before relaxing)

.comment        0x0000000000000000       0x33
 .comment       0x0000000000000000       0x33 ./User/ch32l103_it.o
                                         0x34 (size before relaxing)
 .comment       0x0000000000000033       0x34 ./User/main.o
 .comment       0x0000000000000033       0x34 ./User/system_ch32l103.o
 .comment       0x0000000000000033       0x34 ./Peripheral/src/ch32l103_adc.o
 .comment       0x0000000000000033       0x34 ./Peripheral/src/ch32l103_dbgmcu.o
 .comment       0x0000000000000033       0x34 ./Peripheral/src/ch32l103_dma.o
 .comment       0x0000000000000033       0x34 ./Peripheral/src/ch32l103_exti.o
 .comment       0x0000000000000033       0x34 ./Peripheral/src/ch32l103_gpio.o
 .comment       0x0000000000000033       0x34 ./Peripheral/src/ch32l103_misc.o
 .comment       0x0000000000000033       0x34 ./Peripheral/src/ch32l103_rcc.o
 .comment       0x0000000000000033       0x34 ./Peripheral/src/ch32l103_spi.o
 .comment       0x0000000000000033       0x34 ./Peripheral/src/ch32l103_tim.o
 .comment       0x0000000000000033       0x34 ./Peripheral/src/ch32l103_usart.o
 .comment       0x0000000000000033       0x34 ./Hardware/src/adc.o
 .comment       0x0000000000000033       0x34 ./Hardware/src/flash.o
 .comment       0x0000000000000033       0x34 ./Hardware/src/gpio.o
 .comment       0x0000000000000033       0x34 ./Hardware/src/pwm.o
 .comment       0x0000000000000033       0x34 ./Hardware/src/rs485.o
 .comment       0x0000000000000033       0x34 ./Hardware/src/tim.o
 .comment       0x0000000000000033       0x34 ./Drivers/TimeSliceOffset/timeSliceOffset.o
 .comment       0x0000000000000033       0x34 ./Drivers/RingQueue/ring_queue.o
 .comment       0x0000000000000033       0x34 ./Debug/debug.o
 .comment       0x0000000000000033       0x34 ./App/src/collect_Conversion.o
 .comment       0x0000000000000033       0x34 ./App/src/inflash.o
 .comment       0x0000000000000033       0x34 ./App/src/mppt_control.o
 .comment       0x0000000000000033       0x34 ./App/src/sl_protocol.o
 .comment       0x0000000000000033       0x34 ./App/src/task.o
 .comment       0x0000000000000033       0x34 ./App/src/uart_dev.o

.debug_frame    0x0000000000000000     0x3230
 .debug_frame   0x0000000000000000       0x30 ./User/ch32l103_it.o
 .debug_frame   0x0000000000000030       0x2c ./User/main.o
 .debug_frame   0x000000000000005c       0x48 ./User/system_ch32l103.o
 .debug_frame   0x00000000000000a4      0x334 ./Peripheral/src/ch32l103_adc.o
 .debug_frame   0x00000000000003d8       0x70 ./Peripheral/src/ch32l103_dbgmcu.o
 .debug_frame   0x0000000000000448       0xcc ./Peripheral/src/ch32l103_dma.o
 .debug_frame   0x0000000000000514       0x90 ./Peripheral/src/ch32l103_exti.o
 .debug_frame   0x00000000000005a4      0x160 ./Peripheral/src/ch32l103_gpio.o
 .debug_frame   0x0000000000000704       0x30 ./Peripheral/src/ch32l103_misc.o
 .debug_frame   0x0000000000000734      0x254 ./Peripheral/src/ch32l103_rcc.o
 .debug_frame   0x0000000000000988      0x16c ./Peripheral/src/ch32l103_spi.o
 .debug_frame   0x0000000000000af4      0x634 ./Peripheral/src/ch32l103_tim.o
 .debug_frame   0x0000000000001128      0x204 ./Peripheral/src/ch32l103_usart.o
 .debug_frame   0x000000000000132c       0xe4 ./Hardware/src/adc.o
 .debug_frame   0x0000000000001410      0x274 ./Hardware/src/flash.o
 .debug_frame   0x0000000000001684      0x150 ./Hardware/src/gpio.o
 .debug_frame   0x00000000000017d4       0x84 ./Hardware/src/pwm.o
 .debug_frame   0x0000000000001858       0xd8 ./Hardware/src/rs485.o
 .debug_frame   0x0000000000001930      0x144 ./Hardware/src/tim.o
 .debug_frame   0x0000000000001a74       0x5c ./Drivers/TimeSliceOffset/timeSliceOffset.o
 .debug_frame   0x0000000000001ad0       0x60 ./Drivers/RingQueue/ring_queue.o
 .debug_frame   0x0000000000001b30       0x9c ./Debug/debug.o
 .debug_frame   0x0000000000001bcc      0x13c ./App/src/collect_Conversion.o
 .debug_frame   0x0000000000001d08       0x78 ./App/src/inflash.o
 .debug_frame   0x0000000000001d80      0x1e8 ./App/src/mppt_control.o
 .debug_frame   0x0000000000001f68      0x280 ./App/src/sl_protocol.o
 .debug_frame   0x00000000000021e8      0x258 ./App/src/task.o
 .debug_frame   0x0000000000002440      0x194 ./App/src/uart_dev.o
 .debug_frame   0x00000000000025d4       0x20 d:/psx/rj/mounriver_studio/toolchain/risc-v embedded gcc/bin/../lib/gcc/riscv-none-embed/8.2.0/rv32imacxw/ilp32\libgcc.a(gedf2.o)
 .debug_frame   0x00000000000025f4       0x20 d:/psx/rj/mounriver_studio/toolchain/risc-v embedded gcc/bin/../lib/gcc/riscv-none-embed/8.2.0/rv32imacxw/ilp32\libgcc.a(ledf2.o)
 .debug_frame   0x0000000000002614       0x54 d:/psx/rj/mounriver_studio/toolchain/risc-v embedded gcc/bin/../lib/gcc/riscv-none-embed/8.2.0/rv32imacxw/ilp32\libgcc.a(muldf3.o)
 .debug_frame   0x0000000000002668       0x44 d:/psx/rj/mounriver_studio/toolchain/risc-v embedded gcc/bin/../lib/gcc/riscv-none-embed/8.2.0/rv32imacxw/ilp32\libgcc.a(subdf3.o)
 .debug_frame   0x00000000000026ac       0x38 d:/psx/rj/mounriver_studio/toolchain/risc-v embedded gcc/bin/../lib/gcc/riscv-none-embed/8.2.0/rv32imacxw/ilp32\libgcc.a(floatsidf.o)
 .debug_frame   0x00000000000026e4       0x50 d:/psx/rj/mounriver_studio/toolchain/risc-v embedded gcc/bin/../lib/gcc/riscv-none-embed/8.2.0/rv32imacxw/ilp32\libgcc.a(divsf3.o)
 .debug_frame   0x0000000000002734       0x20 d:/psx/rj/mounriver_studio/toolchain/risc-v embedded gcc/bin/../lib/gcc/riscv-none-embed/8.2.0/rv32imacxw/ilp32\libgcc.a(gesf2.o)
 .debug_frame   0x0000000000002754       0x20 d:/psx/rj/mounriver_studio/toolchain/risc-v embedded gcc/bin/../lib/gcc/riscv-none-embed/8.2.0/rv32imacxw/ilp32\libgcc.a(lesf2.o)
 .debug_frame   0x0000000000002774       0x50 d:/psx/rj/mounriver_studio/toolchain/risc-v embedded gcc/bin/../lib/gcc/riscv-none-embed/8.2.0/rv32imacxw/ilp32\libgcc.a(mulsf3.o)
 .debug_frame   0x00000000000027c4       0x3c d:/psx/rj/mounriver_studio/toolchain/risc-v embedded gcc/bin/../lib/gcc/riscv-none-embed/8.2.0/rv32imacxw/ilp32\libgcc.a(subsf3.o)
 .debug_frame   0x0000000000002800       0x20 d:/psx/rj/mounriver_studio/toolchain/risc-v embedded gcc/bin/../lib/gcc/riscv-none-embed/8.2.0/rv32imacxw/ilp32\libgcc.a(fixsfsi.o)
 .debug_frame   0x0000000000002820       0x20 d:/psx/rj/mounriver_studio/toolchain/risc-v embedded gcc/bin/../lib/gcc/riscv-none-embed/8.2.0/rv32imacxw/ilp32\libgcc.a(fixunssfsi.o)
 .debug_frame   0x0000000000002840       0x44 d:/psx/rj/mounriver_studio/toolchain/risc-v embedded gcc/bin/../lib/gcc/riscv-none-embed/8.2.0/rv32imacxw/ilp32\libgcc.a(floatunsisf.o)
 .debug_frame   0x0000000000002884       0x38 d:/psx/rj/mounriver_studio/toolchain/risc-v embedded gcc/bin/../lib/gcc/riscv-none-embed/8.2.0/rv32imacxw/ilp32\libgcc.a(extendsfdf2.o)
 .debug_frame   0x00000000000028bc       0x20 d:/psx/rj/mounriver_studio/toolchain/risc-v embedded gcc/bin/../lib/gcc/riscv-none-embed/8.2.0/rv32imacxw/ilp32\libgcc.a(truncdfsf2.o)
 .debug_frame   0x00000000000028dc       0x20 d:/psx/rj/mounriver_studio/toolchain/risc-v embedded gcc/bin/../lib/gcc/riscv-none-embed/8.2.0/rv32imacxw/ilp32\libgcc.a(_clzsi2.o)
 .debug_frame   0x00000000000028fc       0x20 d:/psx/rj/mounriver_studio/toolchain/risc-v embedded gcc/bin/../lib/gcc/riscv-none-embed/8.2.0/../../../../riscv-none-embed/lib/rv32imacxw/ilp32\libg_nano.a(lib_a-memcpy.o)
 .debug_frame   0x000000000000291c       0x54 d:/psx/rj/mounriver_studio/toolchain/risc-v embedded gcc/bin/../lib/gcc/riscv-none-embed/8.2.0/../../../../riscv-none-embed/lib/rv32imacxw/ilp32\libg_nano.a(lib_a-printf.o)
 .debug_frame   0x0000000000002970       0x54 d:/psx/rj/mounriver_studio/toolchain/risc-v embedded gcc/bin/../lib/gcc/riscv-none-embed/8.2.0/../../../../riscv-none-embed/lib/rv32imacxw/ilp32\libg_nano.a(lib_a-puts.o)
 .debug_frame   0x00000000000029c4       0x50 d:/psx/rj/mounriver_studio/toolchain/risc-v embedded gcc/bin/../lib/gcc/riscv-none-embed/8.2.0/../../../../riscv-none-embed/lib/rv32imacxw/ilp32\libg_nano.a(lib_a-wbuf.o)
 .debug_frame   0x0000000000002a14       0x3c d:/psx/rj/mounriver_studio/toolchain/risc-v embedded gcc/bin/../lib/gcc/riscv-none-embed/8.2.0/../../../../riscv-none-embed/lib/rv32imacxw/ilp32\libg_nano.a(lib_a-wsetup.o)
 .debug_frame   0x0000000000002a50       0x7c d:/psx/rj/mounriver_studio/toolchain/risc-v embedded gcc/bin/../lib/gcc/riscv-none-embed/8.2.0/../../../../riscv-none-embed/lib/rv32imacxw/ilp32\libg_nano.a(lib_a-fflush.o)
 .debug_frame   0x0000000000002acc      0x148 d:/psx/rj/mounriver_studio/toolchain/risc-v embedded gcc/bin/../lib/gcc/riscv-none-embed/8.2.0/../../../../riscv-none-embed/lib/rv32imacxw/ilp32\libg_nano.a(lib_a-findfp.o)
 .debug_frame   0x0000000000002c14       0x88 d:/psx/rj/mounriver_studio/toolchain/risc-v embedded gcc/bin/../lib/gcc/riscv-none-embed/8.2.0/../../../../riscv-none-embed/lib/rv32imacxw/ilp32\libg_nano.a(lib_a-fwalk.o)
 .debug_frame   0x0000000000002c9c       0x64 d:/psx/rj/mounriver_studio/toolchain/risc-v embedded gcc/bin/../lib/gcc/riscv-none-embed/8.2.0/../../../../riscv-none-embed/lib/rv32imacxw/ilp32\libg_nano.a(lib_a-makebuf.o)
 .debug_frame   0x0000000000002d00       0x40 d:/psx/rj/mounriver_studio/toolchain/risc-v embedded gcc/bin/../lib/gcc/riscv-none-embed/8.2.0/../../../../riscv-none-embed/lib/rv32imacxw/ilp32\libg_nano.a(lib_a-nano-freer.o)
 .debug_frame   0x0000000000002d40       0x40 d:/psx/rj/mounriver_studio/toolchain/risc-v embedded gcc/bin/../lib/gcc/riscv-none-embed/8.2.0/../../../../riscv-none-embed/lib/rv32imacxw/ilp32\libg_nano.a(lib_a-nano-mallocr.o)
 .debug_frame   0x0000000000002d80       0xd0 d:/psx/rj/mounriver_studio/toolchain/risc-v embedded gcc/bin/../lib/gcc/riscv-none-embed/8.2.0/../../../../riscv-none-embed/lib/rv32imacxw/ilp32\libg_nano.a(lib_a-nano-vfprintf.o)
 .debug_frame   0x0000000000002e50       0x8c d:/psx/rj/mounriver_studio/toolchain/risc-v embedded gcc/bin/../lib/gcc/riscv-none-embed/8.2.0/../../../../riscv-none-embed/lib/rv32imacxw/ilp32\libg_nano.a(lib_a-nano-vfprintf_i.o)
 .debug_frame   0x0000000000002edc       0x30 d:/psx/rj/mounriver_studio/toolchain/risc-v embedded gcc/bin/../lib/gcc/riscv-none-embed/8.2.0/../../../../riscv-none-embed/lib/rv32imacxw/ilp32\libg_nano.a(lib_a-sbrkr.o)
 .debug_frame   0x0000000000002f0c       0xa4 d:/psx/rj/mounriver_studio/toolchain/risc-v embedded gcc/bin/../lib/gcc/riscv-none-embed/8.2.0/../../../../riscv-none-embed/lib/rv32imacxw/ilp32\libg_nano.a(lib_a-stdio.o)
 .debug_frame   0x0000000000002fb0       0x30 d:/psx/rj/mounriver_studio/toolchain/risc-v embedded gcc/bin/../lib/gcc/riscv-none-embed/8.2.0/../../../../riscv-none-embed/lib/rv32imacxw/ilp32\libg_nano.a(lib_a-writer.o)
 .debug_frame   0x0000000000002fe0       0x30 d:/psx/rj/mounriver_studio/toolchain/risc-v embedded gcc/bin/../lib/gcc/riscv-none-embed/8.2.0/../../../../riscv-none-embed/lib/rv32imacxw/ilp32\libg_nano.a(lib_a-closer.o)
 .debug_frame   0x0000000000003010       0x30 d:/psx/rj/mounriver_studio/toolchain/risc-v embedded gcc/bin/../lib/gcc/riscv-none-embed/8.2.0/../../../../riscv-none-embed/lib/rv32imacxw/ilp32\libg_nano.a(lib_a-fstatr.o)
 .debug_frame   0x0000000000003040       0x30 d:/psx/rj/mounriver_studio/toolchain/risc-v embedded gcc/bin/../lib/gcc/riscv-none-embed/8.2.0/../../../../riscv-none-embed/lib/rv32imacxw/ilp32\libg_nano.a(lib_a-isattyr.o)
 .debug_frame   0x0000000000003070       0x30 d:/psx/rj/mounriver_studio/toolchain/risc-v embedded gcc/bin/../lib/gcc/riscv-none-embed/8.2.0/../../../../riscv-none-embed/lib/rv32imacxw/ilp32\libg_nano.a(lib_a-lseekr.o)
 .debug_frame   0x00000000000030a0       0x20 d:/psx/rj/mounriver_studio/toolchain/risc-v embedded gcc/bin/../lib/gcc/riscv-none-embed/8.2.0/../../../../riscv-none-embed/lib/rv32imacxw/ilp32\libg_nano.a(lib_a-memchr.o)
 .debug_frame   0x00000000000030c0       0x30 d:/psx/rj/mounriver_studio/toolchain/risc-v embedded gcc/bin/../lib/gcc/riscv-none-embed/8.2.0/../../../../riscv-none-embed/lib/rv32imacxw/ilp32\libg_nano.a(lib_a-mlock.o)
 .debug_frame   0x00000000000030f0       0x30 d:/psx/rj/mounriver_studio/toolchain/risc-v embedded gcc/bin/../lib/gcc/riscv-none-embed/8.2.0/../../../../riscv-none-embed/lib/rv32imacxw/ilp32\libg_nano.a(lib_a-readr.o)
 .debug_frame   0x0000000000003120       0x70 d:/psx/rj/mounriver_studio/toolchain/risc-v embedded gcc/bin/../lib/gcc/riscv-none-embed/8.2.0/../../../../riscv-none-embed/lib/rv32imacxw/ilp32\libg_nano.a(lib_a-reent.o)
 .debug_frame   0x0000000000003190       0x20 d:/psx/rj/mounriver_studio/toolchain/risc-v embedded gcc/bin/../lib/gcc/riscv-none-embed/8.2.0/../../../../riscv-none-embed/lib/rv32imacxw/ilp32\libnosys.a(close.o)
 .debug_frame   0x00000000000031b0       0x20 d:/psx/rj/mounriver_studio/toolchain/risc-v embedded gcc/bin/../lib/gcc/riscv-none-embed/8.2.0/../../../../riscv-none-embed/lib/rv32imacxw/ilp32\libnosys.a(fstat.o)
 .debug_frame   0x00000000000031d0       0x20 d:/psx/rj/mounriver_studio/toolchain/risc-v embedded gcc/bin/../lib/gcc/riscv-none-embed/8.2.0/../../../../riscv-none-embed/lib/rv32imacxw/ilp32\libnosys.a(isatty.o)
 .debug_frame   0x00000000000031f0       0x20 d:/psx/rj/mounriver_studio/toolchain/risc-v embedded gcc/bin/../lib/gcc/riscv-none-embed/8.2.0/../../../../riscv-none-embed/lib/rv32imacxw/ilp32\libnosys.a(lseek.o)
 .debug_frame   0x0000000000003210       0x20 d:/psx/rj/mounriver_studio/toolchain/risc-v embedded gcc/bin/../lib/gcc/riscv-none-embed/8.2.0/../../../../riscv-none-embed/lib/rv32imacxw/ilp32\libnosys.a(read.o)

.debug_loc      0x0000000000000000     0x6aba
 .debug_loc     0x0000000000000000       0xac ./User/system_ch32l103.o
 .debug_loc     0x00000000000000ac      0xc10 ./Peripheral/src/ch32l103_adc.o
 .debug_loc     0x0000000000000cbc       0x7c ./Peripheral/src/ch32l103_dbgmcu.o
 .debug_loc     0x0000000000000d38      0x155 ./Peripheral/src/ch32l103_dma.o
 .debug_loc     0x0000000000000e8d      0x181 ./Peripheral/src/ch32l103_exti.o
 .debug_loc     0x000000000000100e      0x896 ./Peripheral/src/ch32l103_gpio.o
 .debug_loc     0x00000000000018a4       0x2d ./Peripheral/src/ch32l103_misc.o
 .debug_loc     0x00000000000018d1      0x797 ./Peripheral/src/ch32l103_rcc.o
 .debug_loc     0x0000000000002068      0x437 ./Peripheral/src/ch32l103_spi.o
 .debug_loc     0x000000000000249f     0x1a0f ./Peripheral/src/ch32l103_tim.o
 .debug_loc     0x0000000000003eae      0x757 ./Peripheral/src/ch32l103_usart.o
 .debug_loc     0x0000000000004605       0xa2 ./Hardware/src/adc.o
 .debug_loc     0x00000000000046a7      0x466 ./Hardware/src/flash.o
 .debug_loc     0x0000000000004b0d       0x5b ./Hardware/src/pwm.o
 .debug_loc     0x0000000000004b68      0x142 ./Hardware/src/rs485.o
 .debug_loc     0x0000000000004caa      0x206 ./Hardware/src/tim.o
 .debug_loc     0x0000000000004eb0      0x128 ./Drivers/TimeSliceOffset/timeSliceOffset.o
 .debug_loc     0x0000000000004fd8       0xd7 ./Drivers/RingQueue/ring_queue.o
 .debug_loc     0x00000000000050af      0x1c7 ./Debug/debug.o
 .debug_loc     0x0000000000005276      0x472 ./App/src/collect_Conversion.o
 .debug_loc     0x00000000000056e8       0x3f ./App/src/inflash.o
 .debug_loc     0x0000000000005727      0x2df ./App/src/mppt_control.o
 .debug_loc     0x0000000000005a06      0xd1e ./App/src/sl_protocol.o
 .debug_loc     0x0000000000006724       0x71 ./App/src/task.o
 .debug_loc     0x0000000000006795      0x325 ./App/src/uart_dev.o

.stab           0x0000000000000000       0x84
 .stab          0x0000000000000000       0x24 d:/psx/rj/mounriver_studio/toolchain/risc-v embedded gcc/bin/../lib/gcc/riscv-none-embed/8.2.0/../../../../riscv-none-embed/lib/rv32imacxw/ilp32\libnosys.a(close.o)
 .stab          0x0000000000000024       0x18 d:/psx/rj/mounriver_studio/toolchain/risc-v embedded gcc/bin/../lib/gcc/riscv-none-embed/8.2.0/../../../../riscv-none-embed/lib/rv32imacxw/ilp32\libnosys.a(fstat.o)
                                         0x24 (size before relaxing)
 .stab          0x000000000000003c       0x18 d:/psx/rj/mounriver_studio/toolchain/risc-v embedded gcc/bin/../lib/gcc/riscv-none-embed/8.2.0/../../../../riscv-none-embed/lib/rv32imacxw/ilp32\libnosys.a(isatty.o)
                                         0x24 (size before relaxing)
 .stab          0x0000000000000054       0x18 d:/psx/rj/mounriver_studio/toolchain/risc-v embedded gcc/bin/../lib/gcc/riscv-none-embed/8.2.0/../../../../riscv-none-embed/lib/rv32imacxw/ilp32\libnosys.a(lseek.o)
                                         0x24 (size before relaxing)
 .stab          0x000000000000006c       0x18 d:/psx/rj/mounriver_studio/toolchain/risc-v embedded gcc/bin/../lib/gcc/riscv-none-embed/8.2.0/../../../../riscv-none-embed/lib/rv32imacxw/ilp32\libnosys.a(read.o)
                                         0x24 (size before relaxing)

.stabstr        0x0000000000000000      0x117
 .stabstr       0x0000000000000000      0x117 d:/psx/rj/mounriver_studio/toolchain/risc-v embedded gcc/bin/../lib/gcc/riscv-none-embed/8.2.0/../../../../riscv-none-embed/lib/rv32imacxw/ilp32\libnosys.a(close.o)
